:100000000C943E0D0C9400000C9400000C94000025
:100010000C9400000C9400000C9400000C949A6165
:100020000C9400000C9400000C948B150C940000B0
:100030000C9400000C9400000C9400000C94000040
:100040000C9446150C9400000C94505E0C94000027
:100050000C948C5E0C9400000C9400000C94000036
:100060000C9400000C9400000C9400000C94000010
:100070000C9400000C9400000C94F55F0C940000AC
:100080000C9438610C9400000C94000000000100F6
:100090000200040008001000200040008000000161
:1000A0000002000400080010002000400080000151
:1000B0000204081020408000B803C10B801000002B
:1000C000BC03C10B821F0000C603C10B81030000EB
:1000D000CE03C10B01040300D803C20B01060500C7
:1000E000E203C40B01800000EE03CB0B020F000003
:1000F000F603C50B020F0000FE03C70B020FD01260
:100100000604C90B011000001004190C01100000B6
:100110001A04CA0B000100002204CD0B01080100E3
:100120002C04CE0B030801003A04CF0B0307000098
:100130004204E50B017F3F004C04E40B0104000086
:100140005604D00B030400005E04E30B01641E00A0
:100150006A04D10B000100007604D20B00010000FC
:100160008204E20B010200008E04D30B00010000A8
:100170009C04D40B020F0000A804D60B020FE70367
:10018000B204180C0163000010051A0C01100000E5
:100190001A051B0C01020200BE04D80B0308010063
:1001A000C404D90B03080000CA04DA0B03080000DA
:1001B000D004DB0B03080000D604DC0B03080000AE
:1001C000DC04DD0B03080000E204DE0B0308000082
:1001D000E804E60B040A2E00F004F00B040A2E00DB
:1001E000F804FA0B040A2E000005040C040A2E0081
:1001F00008050E0C040A2E0000000000FF0000009D
:10020000220500022A0504043005080736050C05FE
:1002100036058C063C0580094405100B4C05500C36
:10022000560540035E05140A6805180870051C0190
:1002300000000002280060009800D0000801400182
:10024000210C58002D0B2D002B0B2B004D0A4D00BF
:10025000808182838400002188898A8B8C8D8E8F97
:10026000310B312041424300320B322044454600DD
:10027000330B3320474849004D0A4D000000000071
:10028000340B34204A4B4C00350B35204D4E4F007B
:10029000360B3620505152002B0A2B000000000074
:1002A000370B372053545500380B38205657580019
:1002B000390B3920595A2F002D0A2D00000000005B
:1002C000430C430000000000300B3020202E2C0097
:1002D0002C0A2C00000000003D0A435200000000E0
:1002E00000004A01460032002100004B004A01464E
:1002F0000032004D000096004A01460032005400D2
:1003000000E1004A01460032003D0000F00000001C
:10031000320050002D0000F0005000320050004725
:100320000000F000A000320050004B0000F000F090
:1003300000320050002B00005800B40004003800C8
:100340003800213803006A6100008700C80064009B
:1003500032003D4603006E65696E00000800C8006B
:1003600064003200215603004B004A01460032006F
:100370004D00000001000100E60063004D00000098
:100380000000A0001B00007105D700A0001A0200A9
:10039000710569000000180400730569001E011949
:1003A0000600730550726F64756B74200000537003
:1003B00061727465202000005F4944005F5273320F
:1003C0003332494400005F526F74617465005F54BA
:1003D000617374656E5800005F54617374656E5983
:1003E00000005F44656661756C744B6579002A4353
:1003F0006F64653000002A436F64653100002A4352
:100400006F64653200002A4D61784D6F64756C0031
:100410005F4572774D6F64756C002A546973636829
:1004200045005F4D795465726D4E72005F4D61738A
:100430007465725465726D7300005F454D6F64653D
:1004400000005F4543726564577472005F527330F9
:100450004D6F646500005F5634756E6435005F5003
:10046000756C736554696D6500005F41736B437211
:100470006564697400005F53656E64446562697405
:1004800000005F4372656469744D6F6465005F438B
:1004900072656469744D6173746572002A54616297
:1004A0006C655374617274002A5461626C65456EA8
:1004B00064002A4669727374426F6E5000002A4AC3
:1004C0006F6231002A4A6F6232002A4A6F6233003B
:1004D0002A4A6F6234002A4A6F6235002A4A6F62E4
:1004E00036002A4A6F6237005F4572726F723100C0
:1004F0005F4572726F7232005F4572726F723300C5
:100500005F4572726F7234005F4572726F723500B0
:100510005F4672656967616265005F4B6F6D6D6113
:10052000000054617374657200004C69745A0000D5
:100530004C656974540050756C7300005461737499
:100540002030000073657269656C6C0073657269B8
:10055000656C2032000054617374203200005461D5
:100560007374207061720000466F6C676554000000
:100570005377697463680000706F7274696F6E6995
:100580006572656E00002E666F6C67650000506FC7
:100590007274696F6E656E207369636865726E0050
:1005A000436865662D4D656E75004B206C697374EC
:1005B000656E00004B206C6F65736368656E0000AC
:1005C0004B20647275636B656E0054206C697374A4
:1005D000656E000054206C6F65736368656E000083
:1005E0005420647275636B656E0053797374656D26
:1005F0000000506F7274696F6E004B7265646974AD
:1006000065004B7265642E436C7200006D616E2E46
:10061000506F7274696F6E0054657374000050619E
:1006200072616D657465720050726F64756B74658C
:1006300000004B656C6C6E65720056656E74696C7B
:100640006500436F6C6F7273000030A00531AA051E
:1006500032B40533C00534CA0535D40536E0054645
:10066000EA0541F20543FA054402064A0C06000079
:10067000000030EA05371806391E063828064232CF
:1006800006453A066342060000004572726F72002A
:100690004F70742E0000496D70756C7300005469C2
:1006A0006D656F7574008A062F0C000500009006BA
:1006B000320C000300009606300C000500009E0678
:1006C000310C001400002E202C30414243314445AF
:1006D0004632474849334A4B4C344D4E4F355051C2
:1006E00052365354553756575838595A2F390500F2
:1006F000C11100000300D90B00000300C111030069
:10070000170E0300D90B00000500E00800000A00E6
:10071000C1110A00170E0A00D90B0A00C1110A0004
:10072000170E2800D90B0000000000000000000098
:1007300000000000000000000000000000000000B9
:10074000070C182022204D994D4011404891472018
:10075000222018C007000000070C1F3FEE3F7277F1
:10076000727FFF7F777F783FEE3F1FC0070000005A
:10077000000000000C183DEE3F3FEE3F1FC80F0782
:100780000002000000000000000000000002070856
:100790000F1FCE3F1FC80F0700020000000000001F
:1007A00000000007080F0F880F376F7F7FFF7F3231
:1007B00060070F8000000000000000020002070830
:1007C0000F1FCE3F3FEE3F1AC0070F800000000012
:1007D00000000000000000000006000F0F000600EF
:1007E0000000000000000000FFFFFFFFFFFFFFFF11
:1007F000FFF9FFF0F0FFF9FFFFFFFFFFFFFFFFFF33
:100800000000000000000600091088101088100980
:100810000006000000000000FFFFFFFFFFFFF9FFE0
:10082000F6EF77EFEF77EFF6FFF9FFFFFFFFFFFF40
:10083000000000000E01006A1E33286161886133E8
:10084000001E000000000000000000078C0C18666D
:1008500018186C0C078003030C0F03000300000042
:10086000020003038C0302CC0202800202000E1E6F
:10087000001E0C00000000000C000E0B08090CC448
:100880000E0B4C0938C478784C3103CC030180003E
:100890000000020202271FCC18306770306C181F4E
:1008A000C2270200020000000000001000181C0017
:1008B0001E1F081F1F001E1C001810000000000053
:1008C0000000000088010388070F881F0F880703B6
:1008D000880100800000000000000207080F1FC010
:1008E000020200020200021FC80F070002000000FF
:1008F00000081919881919881919881919881919D6
:100900008000198819000000000E1F36CC6666CCE6
:100910006636CC1E06CC0606CC0606CC06000000C9
:1009200000081F30C03030081F30CC301F8C000052
:10093000CC301F800000000000000000000000001C
:1009400000000000000000000E1F1FEE1F0000004E
:100950000200070F8C1F0200020200020200021FA9
:10096000C80F0700021FC00000000207080F1FC0C9
:100970000202000202000202000202000200000065
:100980000000020200020200020200020200021F36
:10099000C80F07000200000000000000000001086E
:1009A0000101CE3F01C8010100000000000000006D
:1009B00000000000000004000C1C0E3F1C000C0492
:1009C0000000000000000000000000000000000027
:1009D00000000000400040400040400E7F0000004A
:1009E000000000000000088C1838EF7F38EC180871
:1009F0008000000000000000000000000000000077
:100A00000207080F1FCE3F7FF0000000000000002B
:100A1000000000000000000F7F3FEC1F0F80070266
:100A200000000000000000000000000000000000C6
:100A300000000000000000000000000000000000B6
:100A40000600060F000F0F000F0F0006060006003D
:100A5000000006000600000000000019881919882F
:100A6000190000000000000000000000000000006D
:100A70000006060666063FFC0C0CC819198C7F336D
:100A800000333300000000000600061F8C3F3600D4
:100A9000363F8C1F06CC063FC81F0600060000002C
:100AA000000000001338387E3801C80307000E1C10
:100AB0000E3870EE600000000000070D88191980E4
:100AC0001B0E001E3E063333C8313BC61E0000001D
:100AD0000E000E0E000606000C00000000000000D4
:100AE00000000000000000000380060E000C1C0047
:100AF0001C1C001C1C001C0C000E0608030000003F
:100B00001C0006070003038803038803038803030C
:100B1000000706001C000000000000000C3636C86C
:100B20001F0F0C3F0F081F36CC36000000000000DE
:100B3000000000000000060006060C3F3FC006064D
:100B4000000600000000000000000000000000009F
:100B50000000000000000000000E0E000E06000C59
:100B6000000000000000000000000C3F3FC000003B
:100B70000000000000000000000000000000000075
:100B80000000000000000000000E0E000E0000003B
:100B900000010000370000EC010380070E001C3844
:100BA00000706000000000000F8E3F30676060FB47
:100BB000616333666C33787036303FE80F000000B5
:100BC0000300071F001F03000303000303000303C8
:100BD00000031FEE1F0000001FCE3F707360607E99
:100BE0000001C80307000E1C00387FFF7F000000D3
:100BF0001FCE3F7073600037000FEC0F0063006082
:100C000037703FEC1F00000001CC0307CC0E1CCC5A
:100C10003870CC607FFF7F00CC0000CC000000006B
:100C20007FFF7F600060600C7F3FE7000033006063
:100C300037703FEC1F00000003CC070E001C38008B
:100C4000307FCE7F7073606037703FEC1F00000014
:100C50007FFF7F00660000CC0001880103000306CF
:100C600000060C000C0000000F8C1F38E630306EC0
:100C7000381FCE3F7073606037703FEC1F0000007C
:100C80001FCE3F7073606037703FFF1F006E000122
:100C9000C8031F001E0000000000000000000E003E
:100CA0000E0E00000000000E000E0E0000000000FE
:100CB0000000000000000E000E0E00000000000EFC
:100CC000000E0E000606000C00CC010380070E008B
:100CD0001C3800381C000E07080301CC000000007F
:100CE000000000000000000E3F3FE000000E3F3F0C
:100CF000E0000000000000003000381C000E070873
:100D00000301CC010380070E001C380030000000F6
:100D10001F8C3F70E66060EC01038007060006064A
:100D200000000600060000001FCE3F306B676FBB5F
:100D30006D6DBB6D6DBE6F67C0703FCC0F00000066
:100D40000600060F000F0F081919881930CC3F3F15
:100D5000C6606066600000007F087F61CC6060CC88
:100D6000617F8C7F60E660606E607FC87F000000FE
:100D70000F8C1F38E63060006060006060006030FB
:100D80006E381FC80F0000007F087F61CC6060666E
:100D90006060666060666060CC617F807F0000009C
:100DA0007FEE7F6000606000607F887F6000606031
:100DB00000607FEE7F0000007FEE7F6000606000DB
:100DC000607F887F600060600060600060000000FD
:100DD0000FCE1F38603060006063EE636066603085
:100DE00066381FEE0F000000606660606660606637
:100DF000607FEE7F60666060666060666000000035
:100E00001F881F06000606000606000606000606E6
:100E100000061F881F0000000066000066000066D4
:100E200000006600006660606C703FC81F00000034
:100E3000606E6061C86367006E7C007C6E006763F3
:100E40008C6160E66000000060006060006060002F
:100E5000606000606000606000607FEE7F00000006
:100E6000606E7070EE7979E66F6F666666666060D8
:100E700066606066600000006066707066786C6630
:100E80006C66666663666361EE6060E66000000043
:100E90000F081F39CC306066606066606066603045
:100EA000CC391F800F0000007F8C7F60E660606699
:100EB0006060EC7F7F806060006060006000000028
:100EC0000F081F39CC30606660606660606663330F
:100ED000CC391FE60F0000007F8C7F60E660606603
:100EE0006060EC7F7F8067638C6160E6600000007B
:100EF0001F8C3F70E6606000703F8C1F00E6006052
:100F00006E703FC81F0000003FCC3F060006060081
:100F1000060600060600060600060600060000009B
:100F200060666060666060666060666060666060A3
:100F30006C303FC81F000000606660606C3030CCD1
:100F40003019881919800F0F000F060006000000E5
:100F500060666060666060666060666666666F793F
:100F6000EE7070E66000000060666030CC30198082
:100F70000F0600060F081930CC30606660000000D4
:100F800060666030CC301988190F000F0600060625
:100F900000060600060000007FEE7F00CC00018006
:100FA000030600060C00183000307FEE7F000000C2
:100FB0001F881F1800181800181800181800181893
:100FC00000181F881F0000000000406000703800FB
:100FD0001C0E0007038C0100E70000300000000039
:100FE0001F881F0188010188010188010188010112
:100FF00088011F881F0000000200070F8C1D38E7C2
:1010000070603000000000000000000000000000E0
:1010100000000000000000000000000000000000D0
:1010200000000000007FFF7F0000070700070600A8
:1010300006030000000000000000000000000000A7
:10104000000000000000000C1F3FE6001FEE3F60A4
:1010500066607FEE3F000000600060600060600836
:101060006F7FCE70606660606E607FC87F0000003A
:1010700000000000000000081F3FC67060006060B4
:1010800006703FC81F000000006600006600006692
:101090001F3FEE716066606066703FEE1F000000EB
:1010A00000000000000000081F3FC6707FEC7F605A
:1010B00000703FC81F00000007880F1C00181800B0
:1010C000187F007F1800181800181800180000007A
:1010D000000000000000000E1F3FE670606E703FD1
:1010E000E61F006E003FC83F600060600060600067
:1010F0006F7F8C7160CC6060CC6060CC6000000061
:1011000000000006000600000E0E0006060006069F
:1011100000061F881F000000000000018801000871
:10112000030388010188010188010188191F800FCC
:101130003000303000303008313380373E003E37E9
:10114000083331CC300000000E000E060006060009
:10115000060600060600060600061F881F0000009F
:101160000000000000000008597FCE7F66666666BA
:101170006666666666000000000000000000000869
:101180003F3FCE3030663030663030663000000091
:1011900000000000000000081F3FCE706066606025
:1011A0006E703FC81F000000000000000000000833
:1011B0007F7FCE6060666070EC7F6F8060600060F3
:1011C000000000000000000E1F3FE67060666070C7
:1011D000EE3F1F6600006600000000000000000CEB
:1011E000373FE6383000303000303000300000004B
:1011F00000000000000000003F7F80607F083F018A
:1012000088017F803F0000000000181800181800B7
:101210007F7F00181800181800181F880F000000A2
:1012200000000000000000066060666060666060AC
:101230006E703FE61F000000000000000000000686
:1012400060606C3030C81919800F0F000600000074
:101250000000000000000006666666666666666F4F
:101260006C3F39C810000000000000000000000CB6
:101270006071C83B1F000E1F083B71CC600000006E
:10128000000000000000000C3030C81919800F0F5A
:10129000000606000C0C0018000000000000000C06
:1012A0007F7F800306000C1800307FCC7F00000099
:1012B00003CC070E000C0C000C1C00381C000C0C9E
:1012C000000C0E0C0703C000060006060006060010
:1012D00006000006060006060006060006000000DE
:1012E0003C003E070003030003038C01038003035B
:1012F000000307003E3C00000000001C6C366380C9
:1013000000000000000000000000000000000000DD
:1013100000000000000006000F198C306066607F3E
:10132000EE7F00000000000000001E0060077E0746
:1013300000F01EF060F77EF7FBDE1F00E007FF07FE
:1013400000F81FF8E0FFFFFF00000F00E002EF02CF
:1013500000780F78E07AEF7AF7BD1F00E007FF070B
:1013600000F81FF8E0FFFFFF23000002000010005C
:1013700000050000FE0500182800FE0400182400E7
:10138000F90F00F80F0070001F71802372802A731C
:10139000111574111C75151B76151A77181C781504
:1013A00021050100FF000000013F2B020010072172
:1013B00000000100072300100000FD30000733008B
:1013C000113068FF0000E50080000100010001020B
:1013D00000040330100400000802020900000A00A3
:1013E000000C00000D00000F0000100000110700AD
:1013F000120000130000FD500010B01B110700FD8B
:101400005000121E01FD500013001F291F00FD5047
:1014100000200000210000FE01002B0C00FE000057
:101420002B20003000003106033200023507013660
:1014300004043706063805013907073C00063D0756
:101440000850000051EF00520000533F01FE010020
:101450006000A7FE00006000276101006A000080B4
:1014600000008100008200008300008400008500ED
:1014700000901000920007930700953F039700002B
:10148000980000070100FD5000072100072300FD20
:101490005000077301FD000000000000007C000008
:1014A000000001C000C000000000000000000000BB
:1014B000038380000000063007387FFFFC3FFFE019
:1014C00007FFFFC00400F0000000080E0808FFFF3F
:1014D000F8FFFFFC0FFFFFF008000E00FC1F1001DB
:1014E000F018FFFFF9FFFFFE0FFFFFF01000018172
:1014F0000330D0000019FFFFF3FFFFFE1FFFFFF8CE
:10150000100000C100C0D0000039FFFFE7FFFFFE60
:101510001FFFFFF8100000620000C80000300FFC41
:1015200007FE0FFE1FF81FF8200000320000C80061
:1015300000601FFC07FE0FFC3FF83FF8200000345E
:101540000000C80000601FFC0FFC1FFC3FF03FF8CC
:10155000200000340001880000C01FF80FFC1FFCB1
:101560003FF03FF0300000640001880000C03FF809
:101570000FFFFFF87FFFFFF0100003E40001880079
:1015800001803FF81FFFFFF87FFFFFE01C000F8482
:101590000003080001803FF01FFFFFF87FFFFFC03E
:1015A00004003C040003100001807FF01FFFFFF0E7
:1015B0007FFFFF00020070040006100003007FF0B0
:1015C0003FFFFFF0FFFFFC00020060040006200068
:1015D00003007FE03FF07FF0FFE0000002006004C6
:1015E000000C20000300FFE03FE07FE0FFC00000B0
:1015F0000200C004000C40000300FFE07FE0FFE1B8
:10160000FFC000000200C004001880000100FFC0FD
:101610007FE0FFE1FFC00000010180020030800098
:101620000181FFC07FC0FFC1FF8000000101800277
:10163000007100000181FFC0FFC1FFC3FF800000F7
:1016400001030002006300000181FF80FFC1FFC3AE
:10165000FF8000000103000300C2001E0183FF8021
:10166000FF81FF83FF000000018600010381807F6E
:101670000303FF81FF83FF87FF00000000CE00010E
:10168000C70080E18703FF01FF83FF87FF000000A1
:10169000007C00007E00F780EE07FF01FF03FF07DC
:1016A000FE0000000030000038003F007C07FF0310
:1016B000FF07FF0FFE00000007FE03FE07FF0FFEFF
:1016C000000FFE000007FE0000000FFE00000FFEEE
:1016D0000000000FFE00000FFE0000001FFF0000D2
:1016E0000FFC0000001FFFFFFFFFFFFFFFFF1FFFBA
:1016F000FFFFFFFFFFFFFF3FFFFFFFFFFFFFFFFFBA
:101700003FFFFFFFFFFFFFFFFF3FFFFFFFFFFFFF69
:10171000FFFE7FFFFFFFFFFFFFFFFE7FFFFFFFFFDB
:10172000FFFFFFFE7FFFFFFFFFFFFFFFFCFFFFFF4D
:10173000FFFFFFFFFFFCFFFFFFFFFFFFFFFFFCFFBF
:10174000FFFFFFFFFFFFFFF87FFFFFFFFFFFFFFF30
:10175000F87FFFFFFFFFFFFFFFF82564002B003E2F
:101760003E006B65696E204B726564697400436F5F
:101770006C6F72546F75636820567320312E35304C
:101780000049443D00202047433D002020353132B0
:101790006B004B653A00496E3A0043616C696272B6
:1017A0006174696F6E004F4B00546F74616C200060
:1017B0002D2D2D2D0054696E79200054696E7920ED
:1017C000626164006B65696E20454570726F6D00E3
:1017D0004D4F44554C2053544F5000446174612088
:1017E00000696E697400533F000066616C73636842
:1017F00065722054697363682000546973636820BC
:10180000766F6E204B20004665686C65722000562E
:10181000656E74696C20616B7469760054696D65DE
:101820006F757400435349204E722000436F646506
:1018300020006B65696E204B726564697400666197
:101840006C736368657220546973636800546973CC
:10185000636820766F6E204B005831393931303053
:1018600000504C5520203A00436F6465203A0054E4
:1018700069736368203A004D42005053004B656C19
:101880006C6E657220004D31004F310053500043A3
:10189000500044590062757379004D50002067650F
:1018A00073706572727400256400416272656368CA
:1018B0006E756E67004B656C6C6E65722000546FC0
:1018C00074616C004D6F64756C2000202000433FF4
:1018D0000073656300496D7000504C553A20005309
:1018E00070617274653A20005072313A2000507273
:1018F000323A200046756E6374203A2000547970A5
:101900003A20003A20563A2020302B2030003A006E
:101910003A20544F3A20003A2050733A2000537036
:101920003A004B204D6F6465204A6F62204A6F6217
:10193000466C616773004B20004D6F646520004A60
:101940006F62202000562020204572722050676C64
:1019500020496D7020544F0056200050617573650A
:10196000004B656C6C6E65723A004D49004D42004B
:101970004D43004D50004D4C0074657374202E2E65
:10198000004F4E002530325800253034580025369F
:1019900064002533642E253032640025356400252B
:1019A00064002532640025336400444400004B2366
:1019B00000425300422100424600542300544F008D
:1019C0004952004D5A0042510042520043530056C2
:1019D0005300564300494C00426600004B2300541C
:1019E0002300424500434500424100445300434226
:1019F0000023502241534349492D492F4F222C2285
:101A0000312E3030222C323030382D30312D3031E3
:101A10003B0023482245636F222C22312E30302296
:101A20002C323030382D30312D30313B00235322D1
:101A300045636F222C22312E3030222C3230303848
:101A40002D30312D30313B00504F00504632333B6A
:101A50005055002564002B302B303B0025640025B9
:101A6000303258002E3030004F4E000001002D4E15
:101A7000414E00000100DE0E6C1A0000F894EE27C3
:101A8000ECBBF1E0F5BFE5BFE0936C00F8E1F1BD20
:101A9000E1BD8DE0A2E0BB27ED938A95E9F780E0F8
:101AA00090E1A0E0B1E0ED930197E9F7E4E7FAE116
:101AB00085919591009761F0A591B591059015904C
:101AC000BF01F00105900D920197E1F7FB01F0CF06
:101AD000EFEFEDBFE0E1EEBFC0E0D3E00C94F9160C
:101AE0000A9902C0E1E00895E0E008951A931FEF1B
:101AF000E2E00E94166CE3EFE1BB85E38A95F1F723
:101B0000E0EFE1BBE4E4E09374000E941F6C0E94EC
:101B1000B266E03091F4E981EE0FE0520E94246C4D
:101B200041F4EDB7FEB7FA93EA931F930E94296C34
:101B30001F910E94C3660E942D6CE0E0E09371004B
:101B40000E942D6CE12F72C30E94326C10E01430A1
:101B5000F0F400E00430C8F4A12FECE30E94366CEE
:101B60000E943A6C0E943F6CE15BFF4FFA93EA934C
:101B70000E94446C0E94446CE02FEE0FEE0FE10FC8
:101B8000EA930E942F4C0F5FE5CF1F5FE0CFECE0A0
:101B9000E0930F04E0E0E09310040E94496C0E947F
:101BA000C8490E944F6C0E947B43E030D9F40E94E8
:101BB000566C0E94566CE6E9F0E00E945B6C0E9455
:101BC000566C0E94566C0E9419470E94656C0E94D8
:101BD000D2410E946C6C0E94D241EEE1F0E00E9482
:101BE000736CE1CF0E947E4341C4E881E03011F084
:101BF0001C9A01C01C9832C00E94566C0E94566C00
:101C00000E94776CEFE3F0E00E947C6C08951A93D9
:101C1000A0910403A43081F4E0910F04E093100438
:101C200010E0183048F4ABE01A9FF001E052FD4F8D
:101C30000E94826C1F5FF5CF42C0A0910403A430C4
:101C400039F4E881E0931004E0E0E0930F0406C06B
:101C5000E881E0930F04E0E0E093100421960895FA
:101C60001A93A0910403A43031F110E0143018F558
:101C70000E94866C3196E491EA93DFDFE0E0E09326
:101C800010040E948F6C3896FA93EA93EBE0F1E02F
:101C90000E94926C0E94926CFA93EA930E94866C66
:101CA000E491EA930E94866C32960E94976C0E949F
:101CB0003C441F5FDBCF0E949A6C0E949F6C19917D
:101CC00008952A970E94A27D30E010E000E047EDE1
:101CD00050E028E0E091190CE03019F020E149E6ED
:101CE00050E03217F0F50E94A36CE13098F10E94A9
:101CF000A36CE03870F0EEE00E94A96CEAE5F7E131
:101D0000FA93EA930E94A36CEF70EF5F0E94B16CAC
:101D100007C0ECE0EA9391DFE8E5EE83E0E0EF83D3
:101D20000E948F6C38960E943A6CE7E3F0E00E94C4
:101D30001C7BE40FF51F0E94926CFA93EA93EDE28C
:101D4000F0E0FA93EA930E94A36CEA930E94566C27
:101D50000E94BB6C1F5F143011F410E00F5F3F5FF7
:101D6000C0CF0E949A6C0E94C8490E94A97D6196CA
:101D700008950E94C16CECE0EA935FDF0E94496C19
:101D8000EBE0EA935ADF0E94C56C0E94CA6CEAEA53
:101D9000F0E00E94CF6CE0913A0CF0913B0CE491A2
:101DA000EA93E0913A0CF0913B0C31960E94D66C8C
:101DB0000E943C4401E00E94D96C0E94DC6C11F04E
:101DC0000F5FF9CF0E94EA6C031718F4E0E0E0938C
:101DD000C0050E94EA6C11E00E94F16C0E94DC6C6C
:101DE00011F0153008F021C00E94C56C0E94F46CFF
:101DF000E0E4F0E00E941C7B3496FA93EA93E2EE72
:101E0000F0E00E94CF6C0E94F16C0E94F76CE491AC
:101E1000EA930E94F16C0E94F76C31960E94D66C96
:101E20000E943C443F5F1F5FD7CF0E949F6C0E947F
:101E3000AB7D36C427970E94A27D22E354E0A09197
:101E40000403A43011F426E453E010E0143010F041
:101E50000C94750F00E0051710F00C94730FE12F30
:101E6000EE0FEE0FE00F3E2F0E94F16C0E94036D0B
:101E70003196E4910E94A96C0E94F16C0E94036D5E
:101E80003296FA93EA930E941569ED85E03039F4B1
:101E9000AF81A13210F4E0E0EF83E0E0E887A02F0B
:101EA000BB27E22FE85FF0E00E941C7B3896FA9394
:101EB000EA930E94F46CEAE3F0E00E941C7BE55B8D
:101EC000FF4F0E94086D0E94926CFA93EA930E9461
:101ED000F16C0E94036DE491EA930E94566C0E949B
:101EE000BB6C0F5FB8CF1F5FB1CF0E949F6C0E9489
:101EF000A97D2E96089522970E940D6DA13059F468
:101F00000E94126DABE2B1E00E94477B2E2F57E199
:101F1000E2ECF0E008C00E94126D0E94166D2E2FB8
:101F200053E0E7EEF0E0EE83FF830E941B6DA0918B
:101F30001908A13081F4E9ECF0E00E94326D0E94B2
:101F4000396D0E943E6DEBE2EA93EDE5F7E10E9408
:101F5000976C0E943C44E3E0F0E00E94326DEA8519
:101F6000FB850E94446D0E94476D0E944B6D3F5F50
:101F7000E091C10BAFEE0E94267BF0E0EE83FF8381
:101F800011E0E091C20B1E17B0F500E0E091C10B2B
:101F90000E1778F50E94516D49F10E94586DE0933B
:101FA00010040E94D96CAE81BF810E941C7B3396C5
:101FB0000E94086D0E94F46C0E941C7BDF010E944D
:101FC000626D0E94656DEA85FB8534970E94446DC1
:101FD0000E94476D0E944B6D3A930E946521EF3F2E
:101FE00029F0ADE05A9FF0010E946A6D3F5F0F5FDC
:101FF000CDCF1F5FC6CF0E949A6C0E949F6CC8C055
:1020000022970E94A27DE2E5F7E0EE83FF8340E0A5
:10201000443190F4AE81BF8111960E94726D139687
:10202000EFEFEC93AE81BF81EC93EE81FF813496AC
:10203000EE83FF834F5FECCFE091C10BA0EF0E94D6
:10204000267B2E2F0E94126DA0E4B1E00E94477BF8
:102050005E2F0E941B6D21FE23C00E94776D0E949F
:10206000776DEFEAF0E0FA93EA930E947C6D0E94AC
:10207000476D0E944B6D0E944F6CE6EBF0E0FA93C7
:10208000EA930E94776D0E94396D0E947C6DEFE7A4
:10209000EA93EFE5F7E1FA93EA93E0E0F0E011C0AC
:1020A0000E94776D0E94776DE8EEF0E0FA93EA9374
:1020B000E52F0E94826DFA93EA930E94476DEAE849
:1020C000FBE0FA93EA930E943C443F5F11E0E09109
:1020D000C20B1E1710F00C94C21000E0E091C10B6F
:1020E0000E1710F00C94C0100E94516D11F40C9456
:1020F000BD10A0919A0BE0E8EA23E03821F0A0910E
:10210000E20BA23019F40E94586D0AC00E94856D3E
:10211000E03011F4E0E001C0E8E0E0930F04E7E014
:10212000E0931004A02FBB27E22FF0E00E941C7B5D
:102130003396FA93EA930E94626D0E94F46C0E94B7
:102140001C7B33960E94446D0E947C6D0E94476DFB
:102150000E944B6D4E2FA0911E08E32F0E948A6DA6
:10216000EA0FFB1F43833A930E946521EF3F29F05A
:10217000ADE04A9FF0010E946A6D3F5F0F5FAECFF6
:102180001F5FA5CF0E949A6C0E949F6C0E945C36D4
:102190000E94A97D28960895E1E0E0930D04E2E015
:1021A000E0930E04E0E0E0931004ECE0E0930F0411
:1021B000ECE5F3E00E94826CEAE0E0930F04EAE4CD
:1021C000F3E00E94826C0E94C84908951A93A98185
:1021D000A43029F4A0E021FCA1E0A03009F426C03D
:1021E000E9810E94916D0490E9810E94976DE491CC
:1021F000A02DAE1BA2501A2F0E944F6CE4EBF0E012
:10220000FA93EA93EB810E94976D0E94CF7B3296FE
:10221000FA93EA93EAE3F0E00E949F6DEFE7EA9316
:10222000EFE5F7E10E94976C0E943C4418812296EA
:1022300008950E94326CE0E0EA930E945C190E94CB
:10224000856D0E2FE4E3F2E00E94CF7B33971E2FC3
:102250000E94566C0E94566C0E94776C0E94A66D7C
:102260000A930E942F4C0E94446C0E94AB6D0E9406
:102270003447E2E0E0930E04E091980BEF70E093B6
:1022800010040E94B06DEFE0E0931004AA81A13029
:1022900051F40E94B86D0E94CA6C0E941947E2E690
:1022A000F7E10E94BD6D21FE0DC0E4E0EA938EDFF0
:1022B000ECE3F2E00E94C16DEEE3F2E00E94C16D3A
:1022C0000E94E349A4DC80C0E8810E94976D0E94CF
:1022D000C16DEA810E94916D0E94C16D0E9471479B
:1022E000E881EA9373DFCAC11A930A93EC81EA93F7
:1022F000EBDF1AEEEC810E94916D0490EC810E945C
:10230000976DE491A02DAE1BA2500A2FAC81A43092
:1023100029F4A0E021FCA1E0A03009F409C01EEAE4
:10232000AA81BB811B96E0E0EC93EC81EA934EDF3F
:102330000E94586DE0931004EC810E94C66DFF93DB
:10234000EF930E94776DEE810E94976D0E94CF7B84
:1023500031960E949F6D0E94D96CFA93EA93EC85A6
:10236000E058EA930E94566C0E94CC6D0E943C4457
:10237000AF91BF91EC93EC810E94976D0E94C16D6B
:10238000EE810E94916D0E94C16D0E94E349198106
:102390000881259608950E94D16D0E94166D8F01C7
:1023A0000E94566C0E94566C0E94776C0E94D46DFD
:1023B0000E94B86D0E941947EA81EA930E945C1955
:1023C0000E94B06D0E94DB6D1981088123960895EB
:1023D0000E94D16D0E94166D8F010E94566C0E9462
:1023E000566C0E94776C0E94D46D0E94B86D0E945A
:1023F0001947EC81FD810E94BD6DAA81BB810E94BD
:10240000987D24F4A030E0E1BE070CF006C0EA811C
:10241000FB81FA93EA930E94DB41AA81BB81A13040
:10242000E0E1BE0724F0A030E1E1BE070CF00AC0F5
:10243000A6EEBBE0EA81FB81E150F0410E94E56D30
:102440000E94ED6D0E94DB6D19810881269608952A
:102450000E94D16D0E94166D8F010E94566C1A93D6
:102460000A930E94E349E0E0E0933C0C0991199142
:102470000895E881EA930E945C190E944120E030AF
:1024800051F10E94F36D0E94566C0E94F76D0E94FC
:10249000B06D0E94FB6DE881EA930E94AC21E88355
:1024A0000E94FF6D3B9734F00E94FF6D0E940A6E00
:1024B000E9E40BC0A6E0B7E00E940E6E0E94116E28
:1024C0000E94166E0E941B6EE3E7EA930E94B746D5
:1024D000E2E0E0930E04D2C00E94B268E0E0E09334
:1024E0000F04A0910403A43019F4E8E6F3E002C05D
:1024F000E4E7F3E0FA93EA930E941C4408950E94F3
:1025000040470E94B2680E94D968E1E0E0930D0460
:102510000E94F36DE6E0F0E00E941F6EEEE6F7E148
:102520000E94BD6D0E94566CE7E0F0E00E941F6EB5
:10253000E1E8F7E10E94BD6D0E94236EEA930E94DC
:10254000E841E5E8F7E10E94BD6DE0910403EA93FC
:102550000E94E841EBE8F7E10E94BD6D08952A97DB
:102560001A930A930E94566C0E94566C0E94776CD4
:10257000E4E6F0E00E947C6C00E010E01530B0F47E
:10258000053020F40E94286EE03009F40DC00E944E
:10259000566C0E94D96C0E941F6E0E942F6E0E9482
:1025A000286E0E94346E0F5F1F5FE8CF0E94366E68
:1025B0000E941947E2E9F7E10E94BD6DE091310800
:1025C000EA930E94E8410E94C56C0E94B86D0E9487
:1025D0001947E6E9F7E10E94BD6DE0912306EA9311
:1025E000E5E0EA930E949E41E091190CE03079F118
:1025F0000E94C56C0E94AB6D0E941947E0912806AD
:102600000E94396E0E94776D0E941947E09128065A
:10261000E295EF70E695E695AE2FE0912906EE0F74
:10262000EE0FEA0F0E94396E0E94CA6C0E94194791
:10263000E0912906E295EF70AE2FE0912A06E2952F
:10264000E07FEA0FEA93E6E0EA930E949E410E944F
:10265000C56C0E94AB6D0E941947E0913F0CEA9354
:102660000E94EE41198108817DC1E881E064E7B9EB
:10267000369A349BFECF349AE4B1F5B12196089591
:10268000E881F981AA81BB81AE17BF071CF4EA1B60
:10269000FB0B06C0A881B981EA81FB81EA1BFB0B19
:1026A0002496089528970E94A47DEFE0E0936100AE
:1026B000E1E0E09362000E941F6CE5E0E0936100BE
:1026C0000E941F6C0E943F6EE0936F05F0937005AF
:1026D000E0917B05F0917C05E0936D05F0936E052C
:1026E000E1E0EA93C2DFE0937B05F0937C05EFE045
:1026F000E0936100E8E0E09362000E941F6CEAE072
:10270000E09361000E941F6C0E94446EE0936B0591
:10271000F0936C05E0917905F0917A05E0936905F5
:10272000F0936A05E0E0EA93A0DFE0937905F09387
:102730007A050E94446EA0916B05B0916C05EA0F7A
:10274000FB1FA0917905B0917A050E94496E8F0117
:102750000E943F6EA0916F05B0917005EA0FFB1FBC
:10276000A0917B05B0917C050E94496E9F01E0918C
:102770006B05F0916C050E94506EFF93EF930E94E1
:10278000446E0E94506EAF91BF91EA0FFB1FFF9302
:10279000EF93E0917905F0917A050E94506EAF9128
:1027A000BF91EA0FFB1FE0937505F0937605E0916A
:1027B0006F05F09170050E94566EFF93EF930E9493
:1027C0003F6E0E94566EAF91BF91EA0FFB1FFF93C1
:1027D000EF93E0917B05F0917C050E94566EAF91DE
:1027E000BF91EA0FFB1FE0937705F0937805A09166
:1027F0007505B0917605E4E1F0E00E94EE7A0E2EC8
:10280000A0917705B0917805E4E1F0E00E94EE7ABE
:10281000E02919F00E94EC45A3C0009371051093C4
:1028200072052093730530937405A0916405A63456
:1028300028F4E0916405EF5FE09364050E945C6E0C
:10284000989724F40E94616E98970CF00EC0A091A6
:102850006405AA3019F4E1E0E0936105A0916405F4
:10286000A83219F4E2E0E09361050E945C6E99974A
:1028700024F00E94616E99970CF472C0E091670594
:10288000EF5FE09367050E94666E0E945C6E0E9497
:102890006B6E0E94726E0E94776E0E94217B7F9306
:1028A0006F93FF93EF93A2E0B0E00E94EA7B0F01E9
:1028B0000E94666EDF01F001EA1BFB0BAF91BF9136
:1028C0008F919F910E94806E0E94726E0E94856E11
:1028D0000E94616E0E946B6E0E948A6EAC81BD8107
:1028E0008E819F81EFE3F1E060E070E00E94217B48
:1028F0007F936F93FF93EF93A6E0B0E00E94EA7B93
:102900000F010E94856EDF01F001EA1BFB0BAF9106
:10291000BF918F919F910E94806E0E948A6EE0917C
:102920001204E03049F4E885F985E0935905F09305
:102930005A05EC81FD810AC0EC81FD81E0935905C7
:10294000F0935A050E94776E0E94B67AE0935B0579
:10295000F0935C050E94656C0E946C6C0E9474454B
:102960000E94AB7D2C9608951A930E944047E2E0A6
:10297000E0930E04E2E3F0E00E94926C0E948F6EFE
:10298000EAE9F7E10E94BD6DE4E1EA930E94474164
:10299000E0E9F1E00E94936EE4E1EA930E9447418E
:1029A000A0916705A13010F0A895FACF10E014307F
:1029B00010F00C943315E2E0E0930D040E94976E42
:1029C000DF010E94C16DFD0132960E94C16D0E941F
:1029D00034470E94976E3496E491EA930E94B7467A
:1029E000E1E0E0930D04A0916705AF3110F4A895E4
:1029F000FACFEAE0EA930E9447410E94976EDF0116
:102A000035960E94CF7BBF01FD010E949D6EDB01C8
:102A10000E94FA7BE2E3F0E0FA93EA930E94F46CFE
:102A2000E8E2F0E00E941C7BE65AFF4F0E948F6EA6
:102A30000E94976E0E949D6E0E940A6EA09167058B
:102A4000AE3110F0A895FACF0E94976EDF010E9478
:102A5000C16DFD0132960E94C16DE8E1F0E00E9477
:102A60005B6C1F5FA4CFE2E3F0E0FA93EA93EAEF36
:102A7000F0E00E948F6EE6EAF7E10E94BD6DE0EDA6
:102A8000F7E00E94936E0E9440474DC10E94A46EE1
:102A90000A93E4E6E2BF78940E94364503DEE6B38B
:102AA000AFEFEA27E0933108A2E6BBE00E94B36EE5
:102AB000E091620BE77031F4A0910A04E0E4EA27A8
:102AC000E0930A04E091620BEF7131F4A0910A04E3
:102AD000E3E8EA27E0930A040E9480660E944D2200
:102AE000E2B3EF700E2EA0911408B0911508EFE03C
:102AF000F0E0AE27BF27EA23FB230E94CF7AE0292C
:102B0000E2BBE0911408E07111F41D9A01C01D9818
:102B10000991199115C00E94A46EE6E0E4BDE0B1F0
:102B2000E295EF70AE2FE0916300E071E15FEA2380
:102B30001E2F0E94A66D0E9424220E945A6619919F
:102B4000E991EFBFF991E991B991A9919991899191
:102B500079916991F9901990099018950E9484656E
:102B60000E940A660E9475510E947D1F08951A9363
:102B7000A8950E944D43E13011F00C941816E09195
:102B8000C605E1501E2FA091C505A13021F40E9479
:102B9000B96EE03009F40CC0ADE01A9FF001E15FBE
:102BA000FC4FBF01E081E260DB01EC930E94C06E4C
:102BB000A091C505A23011F0A43089F40E94B96E2D
:102BC000E093DB050E94C56E31F0FD01E15FFC4F33
:102BD000E081E27009F403C01A930E94CE6EA091C6
:102BE000C505A33019F41A930E94FD27A091C505CD
:102BF000A53029F4E091C605EA930E943428A091FB
:102C0000C505A830A9F4E0E0EA93E091C605EF77A6
:102C1000EA930E942F191E2F1F3F51F0E0E0EA9324
:102C20000E944741E12FE058E093DB05E0932D0639
:102C3000E0910A04E078D1F0E0910A04EF77E093A4
:102C40000A040E940C4AE0910A04E07131F0E0911C
:102C50000A04E270EA930E941E46A0913208A13352
:102C600028F0E2E0EA930E94760D1E2FA0913C0C22
:102C7000A13039F4E0913D0CF0913E0C0E94D26EEF
:102C800009F401C0E5DB6ADF4EC01A930E94404799
:102C9000E1E0F0E00E94976C0E94194710E00E946A
:102CA000DC6E0E94566C0E94A66D0E941947E0914E
:102CB0002108E03049F4E9EAF7E10E94BD6D0E9485
:102CC000E26E0E941B6E1E5FA0912108A130F0F001
:102CD000E0912108E150EA930E948B19A091B30B77
:102CE000AD3229F40E94EB6E0E94947D79F0E3EB03
:102CF000FBE00E94ED6DE6E0F0E0FA93EA930E94BB
:102D0000F86E0E94EB6E0E941B6E1E5FE091210820
:102D1000EF5FE09321081C3020F4A0912108AB3034
:102D200008F001C0BECF199108951A930E94404740
:102D3000E981E03019F4E0E0E0931E08A981A230B7
:102D4000A9F410E0A0911E08A13010F01C3008F08A
:102D50000DC0E0911E08E150E0931E080E94FC6E39
:102D600019F40E940A6F09F01F5FECCF0E94DC6E1D
:102D700010E00E94566C0E94A66D0E941947A09117
:102D80001E08A33608F50E94FC6E19F40E940A6F13
:102D9000D1F0E0911E08EA930E945C190E94B06D88
:102DA0000E94566C0E94F86E0E94156F0E940A6E77
:102DB000E8E7EA930E94B7460E94FB6D0E941A6FF3
:102DC0000E941B6E1E5F05C0E0EBF7E10E94BD6D27
:102DD0001E5FE0911E08EF5FE0931E081C3020F498
:102DE000A0911E08A43608F001C0C3CF1881229616
:102DF0000895E0E0E5BFE0936D00E0936C00EBBB6D
:102E0000EFEFEABBE0E0E8BBE7BBE5BBEFEFE4BB1D
:102E1000E0EFE2BBE1BBE0E2E3B9ECEBE2B9E0E01A
:102E2000E0936200E0936100EFE0E0936500E093DF
:102E30006400E0E0E0BFE7E0E3BFE4E6E2BFE0E03B
:102E4000E1BFEFBDEEBDEDBDECBDE7BDE6BDEBBD49
:102E5000EABDE9BDE8BDE0937900E0937800E3E0E6
:102E6000E5BDE6E0E4BDE0E0E3BDE0938B00EAE031
:102E7000E0938A00E0E0E0938900E0938800E0932B
:102E80008100E0938000E2E1E0938700E4E3E093D7
:102E90008600E0E0E0938500E0938400E093830007
:102EA000E0938200E0936A00E0E3EABFE0E4E9BF78
:102EB000E8BFE1E4E7BFE0E0E0937D00EBB9E8EDD7
:102EC000EAB9E6E0E0939500E0E0E0939000E7E601
:102ED000E9B9E0E0E0939B00E8EDE0939A00E6E0DA
:102EE000E0939D00E0E0E0939800E3E3E093990035
:102EF000E0E8E8B9E0E0E0BDE0E4E7B9E7E8E6B93A
:102F0000E0B5EF7EE0BDE0E2E0937000E0E0E0934A
:102F10007200E4E4E0937400EFE1E1BDEFE0E1BDB5
:102F20000E942D5E0E94CB4B0E940F4678940E9417
:102F3000CB4B0E940F46E1E0EA930E94F50D0E9400
:102F4000236EE53128F0A9E0B0E0E0E00E94027CC9
:102F5000D6DA21E030E0E0E0EA930E94760DE093DB
:102F60003208EAE0F0E00E94936E3F5FA0913208E1
:102F7000A43511F03A3008F001C0EDCF0E94B86DD1
:102F80000E94C56C0E941947A0913208A43581F4B3
:102F9000E1E0EA930E94760DE0933208E5EBF7E179
:102FA0000E94BD6DE0913208EA930E94B74607C0C7
:102FB000E0E0E0933208EBEBF7E10E94BD6D94D0C6
:102FC000E03059F40E94B86DE9E0F0E00E941F6E15
:102FD000E4ECF7E10E94BD6D20E00E94666E0F01F7
:102FE000A2E0B0E00E94EA7B0E161F0654F40E9495
:102FF000856E0F01A6E0B0E00E94EA7B0E161F0668
:103000000CF0B2DC203071F40E94B86DEAE0F0E020
:103010000E941F6EE0EDF7E10E94BD6DA8950E9431
:10302000236FFCCF0E9443370E94B86DE9E0F0E0C7
:103030000E941F6EEBEDF7E10E94BD6D0E94071C20
:10304000E03019F0E1EEF7E102C0E6EAF7E1FA93C9
:10305000EA930E94CE460E949266E1E0EA930E94C3
:10306000474100E010E00436E0E01E0724F40E942F
:103070000A66E03009F007C0EAE0F0E00E94936ED3
:103080000F5F1F4FF0CF0436E0E01E072CF0A09139
:103090006705AF3108F068DC6ADD0E94A0320E944B
:1030A000391EFACFFFCF0E94266F17FD02C01030E5
:1030B00011F4E0E067C3E12F65C30E94266F17FD9E
:1030C00010E01A3008F41F5F0E94336F5BC30E9448
:1030D000266F17FD02C0103011F4E0E053C3115009
:1030E0000E94336FE1E04EC31A930A9310E0E4E6C6
:1030F000F0E00E94936EA8950E94B266E03021F441
:10310000E0EA0E943E6F09F002C001E001C000E069
:103110000E94C3661F5F003011F4153008F001C033
:10312000E6CFE02F0991199108950E94436F47C49B
:103130000E94436F0E94506F0895A881B9810E9438
:10314000987D24F4A83EE3E0BE070CF005C00E9481
:10315000566F0E94256717C3E0E015C3A881B981A7
:103160000E94987D24F4A83EE3E0BE070CF005C061
:10317000EA81E03011F4EFEFEA830E94566FED81AF
:10318000EA930E94516760C10E94A47D20E030E074
:10319000283EE3E03E077CF4A8953A932A93CDDFDE
:1031A0001E2F1F3F29F0EFEFEA933A932A93D6DFC1
:1031B0002F5F3F4FEDCF0E94AB7D4FC01A930A9314
:1031C000E0E0F0E0E093400CF093410CAA81A336DC
:1031D00068F40E945F6FE55FFD4E8F010E94666F8D
:1031E0001A930A93E0E4FCE00E94696FE091400CBE
:1031F000F091410C27C11A931FEF1F5F1A93DEDF76
:10320000A981BA81EA17FB0711F0143608F001C052
:10321000F4CFE12F188118C11A930A93A091C10B22
:10322000E091C20BEA9FF001A0911E08EA0F0E2F59
:10323000043608F002E610911E08101758F41A938D
:10324000BDDFAA81BB81EA17FB0711F4E12F03C0A0
:103250001F5FF3CFEFEF19810881249608950E9434
:10326000A27D10E0133618F50E94F46CE8E2F0E05D
:103270000E941C7BE050FE4EAF01E0EAEA93FA01A7
:1032800070960E946D6FEC713E2FE0EAEA93FA01AE
:103290003F960E946D6F0E2FEF81E31719F4EE81B8
:1032A000E01709F002C0E12F03C01F5FDBCFEFEF93
:1032B0000E94A97D289608951A930A93E091890B9C
:1032C000AA81EA17C1F0A33668F40E945F6FE0504C
:1032D000FE4E8F010E94716F0E94696FEA81E09338
:1032E000890B09C0EFEFE093890B0E947C6F0E946D
:1032F000816FE093940BA6C01A930A930E945F6FAC
:10330000E050FE4E8F01AA81A33620F40E94716F17
:103310000E94506F97C01A930A93E091B20BAA8152
:10332000EA17A1F00E948B6F40F40E94976F0E94F1
:10333000696FEA81E093B20B09C0EFEFE093B20B43
:103340000E94A26F0E94816FE093BD0B7BC01A9315
:103350000A930E948B6F20F40E94976F0E94506F17
:1033600071C01A930A93E091330CAA81EA1761F1B4
:103370000E94A76F18F50E94666F1A930A93E4E300
:10338000FCE00E94696FEA81E093330CE0E0E09397
:103390002B06A091350CA13020F0A091350CA8305F
:1033A00008F00BC0A8EDBBE0E091350C0E94B16FB6
:1033B000AE0FBF1FEC91E0932B0606C0EFEFE0933A
:1033C000330CE0E0E093340C3DC01A930A930E9462
:1033D000A76F40F40E94666F1A930A93E4E3FCE03F
:1033E0000E94506F2FC01A930A93E0912E0CAA816D
:1033F000EA17C1F00E94B46F70F4E0EAEA930E9409
:10340000CA6C1A930A93EFE2FCE00E94696FEA81AA
:10341000E0932E0C07C0EFEFE0932E0C0E94BE6FDE
:103420000E94EA680FC01A930A930E94B46F50F486
:10343000E0EAEA930E94CA6C1A930A93EFE2FCE076
:103440000E94506F19810881239608950E94BE6FD3
:103450000E94EA68E881EF5FE093300CD6C12497C0
:103460000E94A27D0E94C56F0E94EA68AA85A336C9
:1034700098F5AB85A13010F0A13208F009C0EB85BA
:103480000E94B16FA3E6B0E00E94CC6F0E94DD6F96
:10349000EB85E03009F5E0E0EE83EF83E887E9872C
:1034A00040E050E020E030E02032E0E03E0794F4DD
:1034B000D901E3E6F0E00E94CC6F0E94DD6F0E942C
:1034C000156F4E0F5F1F0E941A6F0E94E26F2F5FF1
:1034D0003F4FEACF0E94ED6F3FC11A930A93AB8131
:1034E000A13010F0A13208F01CC0EB810E94B16F36
:1034F000A3E6B0E00E941C7BDF01EA810E94FE6F20
:10350000E8E0F0E00E941C7BE050F04D8F01E0EA23
:10351000EA930E94C56C1A930A93ECE1FCE00E94C6
:10352000506F198108810C947B1F0E94A47DEC814F
:103530000E940270E83109F459C00E940770309768
:1035400029F00E9407700E940C70EC830E943520C5
:103550000E2F10E0101710F00C94F61A0E94107045
:103560007EDFAEE1BCE00E94B36EA091200CB09172
:10357000210C8091220C9091230C0E9415700E94C6
:10358000B17AE093200CF093210C6093220C70939D
:10359000230C0E941070A1DFE0EAEA93EE810E9402
:1035A000B16FEE0FFF1FE050F04F0E946D6FE270A1
:1035B000D9F4ED81E093240C0E940770309751F408
:1035C0000E94236E0E941C70EF5EF84DDF010E9486
:1035D000227002C00E940770E093250CF093260C25
:1035E0000E9427700E942C701F5FB4CF0E94AB7D99
:1035F000269608951A930A930E943270ECE2F0E046
:103600000E9439700E943D700E94427010E0133693
:10361000D8F41A9351DEE0912208EA931A931FDF3F
:103620000E944B70EA0FFB1F0F010E944B700E941B
:103630005370DF01CB010E941A6F0E94B17AD00152
:103640000E94CA7B1F5FE3CFA0911908A330B9F590
:1036500000E00031A0F50E94D96C0E94587069F515
:1036600010E01A3050F5E02FE05DEA93E6EEF7E166
:103670000E945D70E12FE05D0E946470E1F40E94A1
:1036800069700E947070EA0FFB1FFF93EF930E9416
:1036900070700E9453707F936F93FF93EF930E941B
:1036A0007662AF91BF918F919F910E94B17AAF9155
:1036B000BF910E94CA7B1F5FD4CF0F5FCACF10E0BB
:1036C0001A3090F40E9470700E945370A0912908E3
:1036D000B0912A0880912B0890912C080E94B17A11
:1036E0000E9442701F5FECCF0C94C31F24970E946E
:1036F000A27DEA85EA9362DD9F01022E032A39F159
:103700003A932A9378DD1E2F40E050E0E0E0EE830C
:10371000EF83E887E987AA851A17B1F4012F0336EA
:1037200098F40A934BDD2E173F0761F4EB85EA937B
:103730000A9395DE0E94156F4E0F5F1F0E941A6F4D
:103740000E94E26F0F5FEBCF0E94ED6F05C0EB852B
:10375000EA93EB85EA9383DE0E94A97D2C96089577
:103760001A93A895A981A13268F40E94C56F0E949E
:10377000EA6810E0133630F4E981EA931A93ADDE7B
:103780001F5FF8CF1881229608951A9311E0113225
:1037900020F41A93E5DF1F5FFACF67C3E1E0E093FF
:1037A000340CE093350C31C0A8950E94A26FEEEA6C
:1037B000F3E0FA93EA930E94C56C0E947770E0935D
:1037C000BB0B0E948070E093BC0BE0E0E093BD0B6C
:1037D0001CC0A895E9E8FBE00E948770E9E2F0E0F0
:1037E0000E9439700E947C6FE4EAF3E0FA93EA9356
:1037F0000E94C56C0E947770E093920B0E948070CB
:10380000E093930BE0EBE093980B219608950E94D0
:10381000A27D0E948C70E03228F0AAE0B0E0E0E0E7
:103820000E94027C00E081DCA091BE0BB091BF0B36
:10383000A633E2E1BE0741F110E01A3030F41A93EA
:10384000B3DF1A9384DD1F5FF8CF10E0133630F436
:103850001A93BFDF1A9350DD1F5FF8CF10E01038C6
:1038600030F41A939BDF1A93B0DD1F5FF8CF8DDF22
:10387000A9E0B0E0E0E00E94027CE6E3F2E1E09340
:10388000BE0BF093BF0B01E010E0183210F00C9467
:103890009A1C0E9491709F010E949170AF010E943A
:1038A0009B703496E491E03011F0E13069F4D90175
:1038B000AC910E949B703596E491EA1720F40E9427
:1038C0009B700E94A27034C0E23091F4DA010E9431
:1038D000C07BE031A7E2FA0714F4FF2342F40E9410
:1038E0009B7036960E94CF7BDA01ED93FC9320C04B
:1038F000E33049F4D901AC91AF3F21F40E949B70B1
:103900000E94A27015C0E43099F4D901AC91AF3F88
:1039100079F400E00E949B703596E4910E1740F414
:103920000E949B700E94A2702F5F3F4F0F5FF2CFEB
:103930001F5FABCFFDDB10E0153060F41A9353DD51
:10394000A0912F0CA63020F01A9380DD1A936BDD26
:103950001F5FF2CFE02F0C944B21E881EF5FE883EB
:10396000A881A43610F0E0E0E883E8810C94C4213B
:103970000E940E6EA5E0B0E00E941C7B30960C9475
:10398000C421A091370CBB27E091360CA6C0F9DF0B
:10399000329774F00E94A770E091360C0E94AE70CE
:1039A0000E94506FE091360CEA93D7DFE093360C1B
:1039B00008950E94A770E091370C0E94AE70FA93B0
:1039C000EA930E9472670895E4E2FCE00E94B670F8
:1039D0000E94A770E091370C0E94AE700E94506F59
:1039E000E091370CEA93B9DFE093370C08950E9419
:1039F000A47DE0E0E093360CE093370C10E030E07B
:103A0000343680F5A8950E94A7703A93B1DFFA93F7
:103A1000EA93E4E2FCE00E94696F00E0A091240CCC
:103A2000A13010F0A03808F001C001E0E12FE03033
:103A300041F4013029F43093370C3093360C11E007
:103A40000FC0E13031F4003019F43093360C12E03D
:103A500007C0E23029F4013019F43093370C13E039
:103A60003F5FCECF46C21A93A091CF0BA870B9F09A
:103A700010E0E981FA810E94F46CAE17BF077CF474
:103A8000ED81E093240CEB81FC81E851FC4F0E9416
:103A9000BD70E0E0F0E00E942C701F5FEACF18815B
:103AA0000C944D21E881EF5FE883A881A43610F0E3
:103AB000E0E0E883E8810C94C421E881E150E883E8
:103AC000A881A43610F0E3E6E883E8810C94C421D1
:103AD000A091390CBB27E091380CF0E031960E94A0
:103AE000C270EC59FF4FDF01E4E6F0E00E94797B01
:103AF00008950E940E6EA5E0B0E00E941C7BE0508D
:103B0000FE4F0C94C421E9E2FCE00E94B670E8810B
:103B1000EA93BBD10C94C4211A9336DBE1E0E09325
:103B2000860BA3C1A89510E0143680F41A93A6D191
:103B3000A091290CAF3F31F40E94C770AF3FEFEF67
:103B4000BE0711F01A93DFDF1F5FEECF0E94CC702B
:103B5000689420F88AC10E94A47D1091390CAD812F
:103B6000AA23CAF5E091380CE11719F0AD81AA2318
:103B70000AF030C01A9382D10E94C770EE81FF8193
:103B8000EA17FB0729F4E885A091290CEA1709F048
:103B90001EC00E94D270EC81FD810E94BB7AEA17A0
:103BA000FB0744F40E94D7700E94E070E0E0EC83D1
:103BB000ED830BC00E94D770EC83FD83E0E0F0E062
:103BC0000E94E070E0E0E093290C1A935ED10E941D
:103BD000E570C8CF46C0E091380CE11729F0AC8100
:103BE000BD810E94987D0CF01BC01A9347D10E94A2
:103BF000C770EE81FF81EA17FB0729F4E885A091E1
:103C0000290CEA1709F009C00E94D7700E94E070E1
:103C10001A933BD1E0E0EC83ED830E94E570DBCFAB
:103C2000AC81BD810E94987D1CF452DF33970CF467
:103C300018C0E885E093290CEE81FF810E94EA70AC
:103C4000EC81FD810E94E070E091380CEA931DD177
:103C5000E091380CEA9326DFE093380CE0E0EC8347
:103C6000ED83689420F8EC81FD810E94AB7D29965C
:103C700008951A93A091420CA03059F4E091450C9C
:103C8000F091460CFA93EA93E8EBFBE00E94EF70A8
:103C900009F40BC0E1E0E093420CE091380CE093B2
:103CA000440CE091380CE093430CA091420CA130FD
:103CB00011F00C94B71EE091390CA091440CEA1756
:103CC00011F40C94A81EE091440CEA93F6DEE09304
:103CD000440CEA93D3D0A091290CA13010F0A03865
:103CE00008F035C0E091430CEA93E7DEE093430C23
:103CF000A091440CEA1759F1EA93C7D0E091E20B86
:103D0000E030E9F410E01530D0F4ABE01A9FF00198
:103D1000DF01E352FA4FE081E03049F0FD01E45267
:103D2000FA4FE081AE2FE091440CEA1709F005C08C
:103D30000E94F570A091430CA0831F5FE4CFE9E2DD
:103D4000FCE00E94B670E091440CEA939ED00FC054
:103D5000E091430CE093390CE0E0E093420C68946E
:103D600020F80E948C68E093450CF093460C7DC0CF
:103D70001A93A8951091390CE091380CE117C1F015
:103D80000E94FB700E94987D64F4EB81A091290C45
:103D9000EA1739F40E94C770E981FA81EA17FB0734
:103DA00009F003C0E12F1881A6C00E94E570E4CF9E
:103DB000EFEF1881A0C00E94D2700E94987D84F419
:103DC000E0912B06E87031F4E0912F08A091290CC6
:103DD000EA1731F40E94FF700E940C70E33608F07D
:103DE00001C05CC10C942222A895E091380CA881F6
:103DF000EA1761F0E8810E94047119F0E8810C94DF
:103E0000C421E881EA934EDEE883EFCFEFEF0C9414
:103E1000C4211A93A8951091390CE091380CE11740
:103E2000E1F00E94FB700E94987D8CF4E0912B06DB
:103E3000E87031F4E0912F08A091290CEA1739F4C9
:103E40000E94C770E981FA81EA17FB0709F002C0F6
:103E50000C9409220E94E570E0CFEFEF0C940A2247
:103E60001A931091390C1A93BFDF19910895E881C4
:103E7000EA9318DEE883EA93B7DF86C20E94A77050
:103E80000E940B710E94696F7FC20E94A7700E94FE
:103E90000B710E94506F78C20E94A47D0E94CC706A
:103EA00010E030E0343628F5A8953A93E7DF00E0DB
:103EB000A091290CA03808F401E0E12FE03041F492
:103EC000013029F43093390C3093380C11E00FC0D5
:103ED000E13031F4003019F43093380C12E007C0AF
:103EE000E23029F4013019F43093390C13E03F5FCC
:103EF000D9CF0E94AB7D249608951A930A93A0917E
:103F00001908A43009F43FC010912F080091510CFA
:103F1000E0913108E03059F0E0932F08689424F8DC
:103F20000E941471E0E0E0933008E0E520C0E091E9
:103F30003008E03021F0E0932F08E2E518C0E0E01F
:103F4000E0932F08E093510CE091C40BE03031F086
:103F5000E091C40BE150EA930E94B119A091340C96
:103F6000A17039F0E091C40BE0932F08E4E4E093F2
:103F7000510CA0912F081A1721F4A091510C0A1787
:103F800011F0689423F80991199108950E941A710B
:103F9000EBE0EC93EC81D8011696EC93EB81D80121
:103FA0001796EC93D8011896E0E0F0E0ED93FC93BF
:103FB000D80112960E942771D80114960E94277189
:103FC0000E942C71F2C00E941A71ECE0EC930E94E6
:103FD0002C7121C21A9318E0113108F5E0911408F0
:103FE000F0911508A981BA81EA27FB27BF010E9439
:103FF0003871E623F723309781F00E943871A98148
:10400000BA81EA23FB23309731F01A93E0E0EA9378
:104010001A93BCDF02C01A93D6DF1F5FDDCFFAC14F
:10402000A0911A0CA93030F0E091590CA091580CD5
:10403000EA1709F414C0E091590CE03021F4E3E6EA
:10404000EA93C1DF08C0E0911A0CEA93E0E0EA933A
:10405000E3E6EA939BDFE091590CE093580C089556
:10406000A0919A0BECE1EA230895A0919A0BA07419
:1040700011F0E2E00895A0919A0BA07809F0E2C156
:104080000DC0A091890BAF3F09F4DCC1E9DFE4303A
:1040900009F4D8C1E5DFE03109F4D4C1E1E00895C5
:1040A0000895A881AF3F11F4E0E06EC1D9DFE4309C
:1040B00011F4E1E069C1E0E067C1A881A23019F420
:1040C000CFDFE83011F0E1E05FC1E0E05DC1E88101
:1040D000A3E2EA9FF001ED55F94FE081E13010F0E5
:1040E000E43108F002C0E1E04FC1E0E04DC1A88139
:1040F000A13118F0E881E051E883E8810E94437122
:104100000E944D71A091D00BA13018F0A881A4306D
:1041100009F006C0E6E9F0E00E94CF7B0E944D71F5
:1041200033C1A881A13010F0A63008F006C0E881A4
:104130000E945871E15CF94F26C1E0E025C1A881D9
:10414000A13010F0A63008F006C0E8810E94587136
:10415000EC5BF94F18C1E0E017C10E94A47DEC812F
:10416000EA93EDDFEF731E2F1030E1F0EC81EA935C
:10417000E6DFE0743E2FE12FE150A1E00E94C77A14
:10418000A0912306EA230E2F303011F4003009F0FD
:1041900002C0E1E008C0303011F0003009F402C084
:1041A000E1E001C0E0E00E94AB7D259608950E9409
:1041B000A27D00E00530A0F50A930E94F3190E9449
:1041C0005D71A7E10A9FF001EE5CF94F0E948770D4
:1041D000E4E1F0E00E943970E091300CDA01509691
:1041E000EC93A0912F0CEFE3EA23AE2FE091320C79
:1041F000E295E07FEE0FEE0FEA0FDA015596EC93B1
:10420000E091300CE1503E2F3F3F41F0E091310C06
:104210000E941C70DA015196ED93FC930F5FCACF98
:1042200010E01336C0F51A930E945C191A9339DF17
:10423000E13079F5E0919D0BEA9373DFE1500E2FA9
:104240000F3F39F10E945D71E12FDA011396EC9373
:10425000E0919D0BDA011496EC93E091A30BF091A1
:10426000A40BDA011696ED93FC930E941570A4E658
:10427000B0E080E090E00E94217BDF01CB01E09183
:10428000A30BF091A40B0E94806EDA011A96ED93B5
:10429000FC931F5FC6CF0E94A97D26960895A0912A
:1042A0001908A23031F0A83021F0A73011F0A53064
:1042B00009F40AC00E943270EFEFF0E00E943970FA
:1042C00076DFE0E0E093A20608951A93E981E058D2
:1042D000E98310E01530C0F4A3E21A9FF001EB551A
:1042E000F94FE081AE2FE981EA1749F4F001EC556E
:1042F000F94FE081AE2FE0912F08EA1709F002C0D4
:10430000E12F03C01F5FE6CFEFEF188122960895DB
:104310000E94A47DED81EA93D8DF1E2F1F3FC1F0DC
:104320000E9464719F01D9011296EC91EF77EC9392
:10433000EC81D9010E946A71EF5EFC4FBF01E08100
:10434000EF77DB010E946A71E15FFC4FA1E0A0837F
:10435000E12F0E94AB7DE2C40E940E6EED55F94F35
:10436000E081E03061F4E0914B0CEF5FE0934B0CA7
:104370000E940E6EED55F94FA0914B0CA0830E9448
:104380000E6EED55F94FE081219608951A931FEFB7
:10439000E091D40BF091D50BA981BA81AE17BF077C
:1043A0003CF0E091D60BF091D70BEA17FB070CF429
:1043B00012C00E9471710E949D181E2F103031F0A2
:1043C0001F3F21F0E0912F08E11729F4E1E0E0938D
:1043D000590CE0E01FC0E0E0E093590C1AC01A93BA
:1043E0000E947171D3DF1E2F103099F01F3F39F4F6
:1043F000EAEEF7E1FA93EA93EB81FC8106C0EAEF7B
:10440000F7E1FA93EA930E947671FA93EA930E9495
:10441000E811E12F188123960895E0916505E030B9
:1044200009F00895E0912C06E03009F008950AC0E3
:10443000E0916605E03009F00895E0912D06E03046
:1044400009F00895E0E008950E94A47DE091260619
:10445000F0912706AC81BD81EA27FB279F0110E080
:10446000153090F4F901E17049F0A7E11A9FF001CD
:10447000EF5CF94FDF01EC91EF5FEC93D9010E9403
:1044800079719F011F5FECCFEC81FD81E0932606DF
:10449000F09327060E94AB7D41C428970E94A27D1D
:1044A0003091260610E01530B8F5A7E11A9FF0010B
:1044B000EB5BF94F0081E12FA1E00E94C77A2E2F1C
:1044C000E22FE32391F0003810F0003C08F001C027
:1044D0000F5F003C31F4E22FA0912306EA2BE0931A
:1044E0002306003808F400E80FC0003408F40F5F1A
:1044F000003439F4EFEFE227A0912306EA23E0939A
:104500002306003808F000E0A7E11A9FF001EB5BFA
:10451000F94F00831F5FC7CFE0E0E0932C06E0E097
:10452000F0E0E0931608F0931708E091590CE030A2
:1045300021F0E0911A0CEA93DADDE0911D08EF5FBB
:10454000E0931D08E091E30BA0911D08EA1751F4D8
:10455000E091E30BF0E0A0E0B1E00E94E37BEA1B16
:10456000E0931D08A0911908A13019F0A93009F0B5
:1045700096C0A091620BB091630BE4E1F0E00E9461
:10458000797B309719F4E1E0E0931F0846DFE030D3
:1045900019F04EDFE07809F462C04ADFEF775E2F52
:1045A0005A930E945C190E94626DED55F94F50813B
:1045B000503011F40C942F2364DDE13031F4E0919C
:1045C0001A08EA937ADDE03009F449C00E947E714E
:1045D0000E94FE6FEC91EC71EC3021F4E0911D082B
:1045E000E07851F40E948371EC91EA9380DD0E949F
:1045F0008871EC91EA937BDD0E948371AC91A630C7
:1046000070F5A6E0B7E00E94626D0E94116E0E94F4
:10461000B36E0E948371EC91EA9383DD1E2F1130FB
:10462000F0F00E948D710E949071CF010E948D71F7
:104630000E94116E6D917C91E12F0E945871EF5C88
:10464000F94F0E949571E60FF71FDC01ED93FC9383
:10465000E12F0E945871EF5CF94FA0E0A08310E0B9
:104660001530E8F40E94987113965C915F3FA9F0B1
:104670005A9372DE5E2F0E94A2710E948D710E9479
:104680009071BF010E948D710E94116E0E94A871ED
:10469000AE81BF811296E0E0EC931F5FE1CFA09165
:1046A0001908A23039F0A83029F0A53019F0A73048
:1046B00009F0E4C1E0E0E093200800E0053010F0EC
:1046C0000C943E25A3E20A9FF001ED55F94FEA87CD
:1046D000FB87AA85BB85AC91A03019F0A281A07898
:1046E00009F0CAC1E0912008EF5FE0932008AA8595
:1046F000BB8513960E94C07B309771F0AA85BB855D
:1047000013960E94B5710E94BB7129F4AA85BB85DE
:1047100013960E942771B0C180DEE03021F00E9424
:10472000BB7109F4A9C120E030E0333010F00C94E3
:10473000EB240E94C371DF010E94F16C0E94E56DC1
:10474000E887F987A181A27021F4A481B58110972F
:1047500009F40CC1E885F985A181A47011F40C94C9
:104760001124A181A87021F40E942034E03009F4C2
:1047700057C00E94C971EBE0EC93A885B9850E94EF
:10478000D671A885B9851396EC91AC85BD85179631
:10479000EC93EC85FD8538960F01E885F985A181BC
:1047A000E1E0EA230E94DD71ED93FC93A885B985D1
:1047B00014960E94C07BAC85BD851296ED93FC9348
:1047C0000E94E071AC85BD851496ED93FC93A02FFB
:1047D000EAE0EA9FF001E30FEF5F0E94E671E885EF
:1047E000F985A085B185E2E0F0E00E941C7BA885F8
:1047F000B9851896ED93FC930E94E071309739F4D7
:10480000A885B9851896E8EEF3E0ED93FC93E8856A
:10481000F985A181E8E0EA2BA885B9851196EC938A
:104820006CC0E885F985A181A17031F4A885B985AE
:1048300014960E94B57141C00E94EF7172DCE15084
:104840001E2F0E9498711296EC91E030F1F4AE8127
:10485000BF8153960E94B36EEE81FF81A189B28918
:10486000109751F003881488AE81BF8151960E9441
:10487000C07BE015F1050CF007C00E94F47111F047
:104880000E94F9710E9401720EC0E885F985349684
:104890000E9409720E94DD710E94C2700E94117212
:1048A00053960E942771E885F985A581AA232AF4E9
:1048B000A885B98514960E942771A885B985EC91C1
:1048C000EC71EC3021F4E0911D08E078B1F4E8855A
:1048D000F985A481B5815E971CF4A181A07209F4C9
:1048E00004C0E885F985A28106C00E94EF71FFDB54
:1048F000E885F985A381AA93FADB0E94E0713097DD
:1049000081F0A885B98518960E94B5710E94E07162
:10491000309739F40E94F47111F00E94F9710E94ED
:1049200001720E94EF7119DCE03001F10E94F47114
:1049300059F00E94F971AA85BB85EC91E150ADE078
:10494000EA9FF0010E946A6DAA85BB851296EC91E0
:10495000E058AA85BB851296EC93E3E0E093240629
:104960000E94EF71ECDBEF73E0932506A885B98513
:1049700014960E94C07B309761F52F5F323048F566
:10498000A885B98516960E94C07B309789F0E88586
:10499000F985A681B7810E941872AA85BB851396F6
:1049A000ED93FC93A885B98516960E94277111C0D6
:1049B0000E94C371DF01E32FEF5FF0E00E94E56D1D
:1049C000E887F987A181EDEFEA23A885B9851196DB
:1049D000EC933F5FAACE233011F00C943C250E944B
:1049E000F47111F00E94F9710E942034E03069F0F6
:1049F0000E94C971E8E0EC93AA85BB850E94D6713C
:104A0000AA85BB85EC910E94E671AA85BB85E0E092
:104A1000EC93EA85FB85A581ECE1EA23E83061F5BA
:104A20000E94236EAE2FEA85FB85E38DEA1741F4E1
:104A3000EA85FB85E48DE150EA930E945D181CC075
:104A40000E942034E030C1F00E94C971E3E0EC9391
:104A5000AC85BD85EFEFEC931896EA85FB85E38D79
:104A60000E941D72AC85BD851296EA85FB85E48D9A
:104A70000E941D720E9421720F5F20CE0E94277239
:104A800049F4A0911908A23021F0A83011F0A53006
:104A900009F401C050C010E0153010F00C949B25B3
:104AA0000E94987113965C915F3F11F40C949925C4
:104AB0000E94A271AE81BF81BD010E94A871EE81EA
:104AC000FF8138960E9409720E942D720E94117215
:104AD0000E94C07BDF010E94987DB4F4EE81FF81CB
:104AE000A681B7810E94987D7CF4AE81BF810D9034
:104AF0001C90AE81BF8116960E94C07BD001AE1B78
:104B0000BF0B0E94987D0CF014C0AE81BF81BD0127
:104B10000D901C90EE81FF81A681B781F001EA1B08
:104B2000FB0BDB01ED93FC935A93E5E0EA930E94C3
:104B30006B431F5FB1CFE0911C08E03041F4E0917E
:104B40001608F0911708E0931408F09315080E94D6
:104B5000A97D2E9608950E94A47DA091C10BE0919D
:104B6000C20BE150EA9FF001EF5F1E2F2FE330E010
:104B700000911E08A091180CA13080F0E091180C53
:104B8000E150A0911E08AE1728F0E091180CE150FA
:104B90003E2F04C0E091180CE2502E2FEC81E03043
:104BA00049F1EF3F51F4A0911E08A11BA31720F07B
:104BB000E0911E08E11B0E2F1DC0EE3F59F4E12FBE
:104BC000A0911E08AE0FA21720F4A0911E08EA0FB4
:104BD0000E2F10C0EC3F49F4A091180CA13020F02A
:104BE000E091180CE1500E2F05C0AC81A1501A9F26
:104BF000F0010E2FE0911E08E01751F00A930E9479
:104C00005C19A0918A0BAD3209F4032F00931E08A2
:104C10000E944047A0911908A83019F40E94001082
:104C200002C00E947B0F0E94AB7D259608950E94D2
:104C3000A27D16DAE03111F40C948B2620E030E0EE
:104C400040E050E010E0133060F50E9431720E94A5
:104C5000116E0E94C07B309711F10E9434720E9445
:104C600043712E2B3F2B0E943472EA9376DAE030A8
:104C700029F0E3E0E0932406E0E04EC00E943B729E
:104C80000E9443712E2B3F2B0E943B72EA9365DA00
:104C9000E03029F0E3E0E0932406E0E03DC01F5F50
:104CA000D2CF00E0053068F5A3E20A9FF001ED5590
:104CB000F94FE081E03019F110E0133000F50E9467
:104CC000C371DF010E9476710E944272AE0FBF1F56
:104CD0001296EC910E9443714E2B5F2B0E94C37180
:104CE000DF010E9476710E944272AE0FBF1F1396C1
:104CF000EC910E9443714E2B5F2B1F5FDECF0F5F45
:104D0000D1CFF901E423F523309729F0E1E0E093D6
:104D10002406E0E001C0E1E00E94A97D2696089506
:104D20001A93E0914F0CE03011F40C94D726E091E7
:104D3000E40BE13059F4A0914F0CA13311F4EFE0F2
:104D400001C0E0E0EA930E94C55E31C0E23059F450
:104D5000A0914F0CA13311F4E6E001C0E5E1EA9324
:104D60000E94C55E24C0E330B1F410E0173040F477
:104D70000E947671E05CF64F0E9449721F5FF6CF89
:104D8000A0914F0CA13311F4E1E301C0E0E3EA93F9
:104D90000E94C55E0CC00E944D72E9E4EA930E9435
:104DA0001A63E0914F0C0E9454720E94597285C49C
:104DB00022970E94A27D30E0A0911908A23029F02C
:104DC000A83019F0A53009F014C1A985A33610F058
:104DD0000C94F827E0912F08E03009F40AC1E98526
:104DE0000E940270E03131F4E1E3E0934F0C98DF70
:104DF000E1E0FFC046D9E03009F4FBC010E0153017
:104E000058F40E946471E081AE2FE885EA1711F42E
:104E1000E0E0EFC01F5FF3CF0ADFE03011F40C9445
:104E2000F82710E00E946471EE83FF83AE81BF819A
:104E3000EC91E03011F00C94F12713960E94277149
:104E400000E0033010F00C94C127A3E21A9FF00198
:104E5000E855F94FDF010E94D96C0E94E56DAF0162
:104E6000DA0116960E9427710E945E72DA0112968C
:104E7000EC930E946572DA011396EC93A0919A0B61
:104E8000EEEFEA23DA01EC930E946C72DA011196DC
:104E9000EC93E6D8E43139F0FA01A181E2E0EA2BA3
:104EA000DA011196EC930A9308D9E03011F40C94CE
:104EB000A327FA01A281AA9334D9E1502E2F2F3FC4
:104EC00081F0A7E12A9FF001EF5CF94FA0E0A083F9
:104ED000A7E12A9FF001EE5BF94FA0E0B0E0A083CC
:104EE000B1830E9474720E94116E0E94C07BDA012D
:104EF0001496ED93FC93013040F00E9474720E946E
:104F0000116E0E94C07B309709F00EC0AE81BF8148
:104F10001596E02F0E94B16F0E944272AE0FBF1F24
:104F20001196EC91E062EC93AE81BF815A96EC91C0
:104F3000E062EC93023030F40E947772DA01169648
:104F40000E941D7204C0DA0114960E94277188D84D
:104F5000EC3019F4E0E0E0931D080E947E720E949C
:104F60001C70DA011896ED93FC93FA01A281A63029
:104F700030F0A181E4E0EA2BDA011196EC930F5FA7
:104F800060CFA0911908A23011F0A53019F4A885BE
:104F9000AF3F08F007C0E0912F08EA93EA85EA9353
:104FA0000E94951AE885AE81BF81EC93E0912F08AD
:104FB000AE81BF811196EC93E985AE81BF811296D7
:104FC000EC93A885A43130F4E885E1500E94857205
:104FD000A1E0A083AE81BF811696EC91ED7FEC93AA
:104FE00031E01F5F303011F4153008F001C01ACFE6
:104FF000E32F0E94A97D2A9608951A930A93A091FF
:105000001908A23011F0A53049F4EA810E94857296
:10501000A0E0A083EA81EA930E94CE6EA0911908D5
:10502000A830F1F4EA810E948572A0E0A083EA81B1
:10503000EA93E1E0EA930E94A247E091E20BE030BC
:1050400069F4EA810E948B72E081EF771E2FABE05A
:105050001A9FF001EA51FA4FA0E0A083689420F86B
:10506000198108812396089564970E940D6DA230DE
:1050700039F4E0912F08EA93EB8DEA930E94951A98
:10508000A0911908A83011F00C94AA280FEF20E085
:10509000253050F4A7E12A9FF001EE5CF94FE08142
:1050A000AE2FEA8DEA1709F402C02F5FF1CFA7E116
:1050B0002A9FF001E15DF94FAF01DA0115960C91DD
:1050C0000F3F11F40C94AA280E94917210810E9443
:1050D000FB700E94987DECF4ACE2BCE00E94B571DC
:1050E0000E9497720E94D270A083B1831A930E948B
:1050F000451FABE00A9FF001E252FA4F30810A935C
:10510000FE0137960E949D723A93FE0137960E94E7
:10511000A1720E94A772F1F40E949172AFEFA08376
:10512000DA011396EFEFEC93DA011596EC930E94F7
:1051300097720E94AD72E0E0F0E00E94E070E0E063
:10514000E093290C1A930E94451F0A930E94641150
:10515000689420F80E94A97D6B9608951A9310E038
:105160001031B0F4A7E11A9FF001EC5BF94FE08138
:10517000EF73AE2FE981EA1729F41A930E94AD204C
:10518000E03009F403C0E1E01881E0C01F5FE8CF20
:10519000E0E01881DBC01A93E091520CF091530CBF
:1051A000FA93EA93E4EFF1E00E94EF70F9F00E94C5
:1051B000B27210E01530D0F4A091560CAF5FE5E06C
:1051C0000E94767BE093560CEF5FEA93C7DFE030F6
:1051D00059F0E3E0E0932406E091560CF0E0EF5F35
:1051E000FF4EE093250669C21F5FE4CF66C21A93A3
:1051F000E0912306E0934E0CE8E7F0E0FA93EA939F
:10520000ECEDF0E0FA93EA930E94714710E015305C
:10521000D8F4E12FEF5FEA93A1DFE03099F00E942C
:10522000566CE12FEA5FF0E00E941F6EE7E0F8E1C4
:105230000E94BD6DA6EEBBE00E9476710E94E56DF6
:105240000E94ED6D1F5FE3CF38C2A5DFE091240619
:10525000E13029F4EFE0F8E10E94B9723CC0E2309D
:1052600029F4ECE1F8E10E94B97235C0E33051F461
:10527000E7E0F8E1FA93EA93E0912506F0E0E050E8
:10528000F04F29C0E43019F4E4E2F8E11FC0E53042
:1052900031F4E0912506EA930E94CB1120C0E6305C
:1052A00019F4ECE2F8E112C0E73029F4E2E3F8E1A6
:1052B0000E94B97210C0E83029F4EEE3F8E10E94D0
:1052C000B97209C0E93059F4EDE4F8E1FA93EA93D0
:1052D000E0912506F0E0FA93EA930E94E811E0E0FD
:1052E000E09324060895A881B9811196E1E0EC933A
:1052F0000E94FF70A881B9811296ED93FC930E94E1
:105300003520A881B9811796EC930E94236EA8815D
:10531000B98118960E941D72E091C605A881B981D5
:10532000EC93E091290CA881B9811696EC93E09159
:10533000890BA881B9811A96EC93E091AC0BF0919E
:10534000AD0BA881B9811496ED93FC932296089534
:1053500064970E94A47DA091E20BA230E1F4EB8D52
:10536000EA930E945C190E943520ACE2BCE00E94E6
:105370001D72AAE2BCE0EB8D0E941D72E0912F0825
:10538000E093290C0E940770309721F00E9407706B
:105390000E94EA7014C0AA8DAF3F09F4CAC0EA8D1A
:1053A000EA930E943E1FAB8DAF3F29F40E94FF702D
:1053B0000E940C70EB8FEB8DEA930E945C190E94A7
:1053C00035200E2FA98DAF3F21F00E944120E03003
:1053D00009F001C0AEC00E94D2700E94D96CAE1715
:1053E000BF071CF024DCE13009F0A3C0A091D10B71
:1053F000A03021F4A091E20BA23011F50E94236E9F
:10540000E13041F00E942034E03021F00E94363437
:10541000E03009F002C00E94BE720E94236EE130AB
:1054200021F40E942634E03009F409C00E94CA72B7
:10543000EE55F84FFA93EA9356DF0E94D07277C088
:10544000EB8DEA93EA8DEA93B3DC1E2F113011F055
:105450000C94972AA091D30BA13059F4E0912F0816
:10546000EA930E94FF70FA93EA93EFEFFFEF0E9436
:10547000D6720E94D2700E94D96C0E94C2700E94A3
:10548000E070689420F8A091E20BA03019F4A88D88
:10549000AF3F09F437C00E94DA72EE51FA4F0E9412
:1054A000D270A083B183E88D0E94C66D3081E88DF3
:1054B000EA93FE0135960E949D72E88D0E94C66DAA
:1054C000E081EA93FE0135960E94A1720E9430208D
:1054D000E03131F00E94DA72EA51FA4FA1E005C0E2
:1054E0000E94DA72EA51FA4FA2E0A0830E94DA72B7
:1054F000EC51FA4FFF93EF930E948C68AF91BF91EC
:10550000ED93FC930E94A77219F4E0E0E093290C5C
:10551000EA8DEA930E94451FE0912F08EA930E94CA
:1055200007700E94DF72FA93EA930E94331DE1E054
:1055300001C0E0E00E94AB7D6C96089578DBE1301D
:1055400041F40E942034E03021F00E943634E030F3
:1055500009F007C00E9407700E94EA700E94BE72A4
:1055600026C32EC30E94A47D0E94E2721F3F11F445
:105570000C94092BE0914F0CE03011F00C94082BA7
:105580001A930E945C19E5E0E09324061093250627
:10559000A0911908A23031F40E94EB720E94EF2111
:1055A000E03009F010C0A091500CA13331F4E0912B
:1055B0002F08EA931A930E94951AE1E3E0934F0CA7
:1055C0000E94AB7DE2C2A0911908A830A1F40E940C
:1055D00007700E94EF720E2F0A930E9496343E2F9E
:1055E0001A930A93EFEFEA933A93B2DEE03019F0A0
:1055F0000E94AB7DCAC2A0911908A53031F49EDF8C
:10560000E03019F00E94AB7DC0C2E0E3E0934F0CA4
:1056100006C0E0E3E0934F0CE4E0E09324060E9430
:10562000AB7DB3C2E09140090E94F37208951A93D2
:10563000E6E0EA930E94C55E0E944D72A091400987
:10564000A83539F4E9E5F8E10E94FF72E0E00E9434
:105650005972A0914009A33509F510E0A0911908ED
:10566000A83021F0A23011F0A53009F411E3E3E5F0
:10567000EA930E941A631A930E941A63E0E8EA937D
:105680000E941A63E0E8EA930E941A63E0E80E942D
:105690005472E0934F0CE0E00E945972A0914009CF
:1056A000A93459F40E940373E09325060E940D73F8
:1056B000EC91E093500C56DF33DB199108950E9472
:1056C000A47DA0913F09A53411F00C94A62B0E9453
:1056D0001273E2E3F0E0E093490CF0934A0CA091DE
:1056E0004009A73741F4E4E4F9E00E9419730E94ED
:1056F0001E730E94F372A0914009A03310F0AA33E8
:1057000008F023C02091270830912808E0E4F9E050
:105710000E941973E2E0EA930E94C0620E2F0E9479
:105720001E73E09325060E941E730E9422730E943E
:10573000E2720A931A930E94951A209327083093D5
:105740002808E2E5EA930E94C55E1CC0E091470C80
:10575000F091480CFA93EA93E091490CF0914A0CCD
:105760000E94EF7079F0E0E0E0933A09E5E4EA9313
:105770000E94C55E0E941273E8ECF0E0E093490CD1
:10578000F0934A0C0E94AB7D00C20E9427730E94D6
:105790002D730E94566C0E94566C0E941947A0916E
:1057A0001B08A23021F4E1E6F8E10E94BD6DA09152
:1057B0001B08A13021F4E8E6F8E10E94BD6DE091FC
:1057C0001B08E03021F4EFE6F8E10E94BD6D0E9475
:1057D00037730E94976C0E9419470E943A730E9487
:1057E0003F73FA93EA93E0915F05F09160050E94A0
:1057F00045730895E1E003C0E0E001C0E2E0E0931A
:105800001B08C3DF08950E943020EC3109F0D8C195
:10581000E091990BE33631F4A0911908A23009F414
:10582000EBDF17C0E23631F4A0911908A23009F479
:10583000E5DF0FC0A091C505A23011F0A63021F41C
:10584000E091990BEA9387D9A091C505A43009F49A
:10585000D1DFADC10E94F36D0E94566C0E94F76DBE
:105860000E94566C0E94566C0E941947E8E7F5E0CA
:105870000E94BD6DE0911A080E944973E6E8F5E0C8
:105880000E94BD6DE2E0E0930E0408950E94327024
:10589000E3EEF0E00E943970E881E03009F406C0E0
:1058A000A0911A08AF5FE3E00E94767BE0931A08AC
:1058B000E1E0E0934B0C0E94D72072C20E94A47DCD
:1058C00010E0133610F00C94AB2C0E947671ED555D
:1058D000F94F30813F3FE9F11A930E945C1900E0D3
:1058E0000E944D730E94116E0E94C07B3B9794F002
:1058F0000E9450730F010E944D730E94116E0E940E
:1059000056730E945C730E94FE6FEC91EE7FD00193
:10591000EC9301E00E9461730E94116E0E94C07BB3
:10592000759794F00E9450730F010E9461730E945A
:10593000116E0E9456730E945C730E94FE6FEC9180
:10594000E160D001EC9301E0013019F41A930E9458
:105950007C191F5FB6CF0E94AB7D17C11A930A93C3
:1059600023FE03C00E9464733FD70E947B43E03054
:10597000C1F1E0E00E946B73103820F5113219F488
:105980000E94647331D71D3439F40E9472730E94EF
:105990003064E3E0E09318081B3271F40E947773DF
:1059A000EAE2EA93EAE7F8E1FA93EA93E0911A0867
:1059B000E05DEA930E9430641F3219F4E1E0EA935B
:1059C000CAD848DF103868F00E947D731A930E948D
:1059D000AC2119DFE03011F4103208F002C0E8ED1C
:1059E000F6E20E9418220E2F0038C8F10F77033616
:1059F000A8F5E0911F08E03031F00A930E943912B7
:105A0000E0E0E0931F08E091570CE01739F10A93AA
:105A10000E945C190E948371AC91A83028F40E9406
:105A20008871AC91A830A8F0E02FEF5FE093A20658
:105A30000A930E94AC210E948371EC91EA930E9428
:105A40008871EC91EA93E091A206EA930E94C61F46
:105A500003C0E0E0E093A2060093570C0EC0A091B3
:105A6000570CAF3F51F0E091A206E03019F0EA93F5
:105A70000E94E31FEFEFE093570C099119910895ED
:105A8000A881A03310F0AA3308F01DC00E948173D2
:105A90000E948673AAE0B0E00E941C7BDF01E881CF
:105AA0000E948B73EA0FFB1FE0932508F0932608F2
:105AB000E2E0E0930E040E9437730E94976C0E940C
:105AC000F76D0E943A73A881A33451F40E942D739C
:105AD0000E9437730E94976C0E94F76D0E943A7380
:105AE0005FC11A930A93A0E023FCA1E0A03019F053
:105AF000AA81A03009F016C0E89423F8E7E0E0930B
:105B000018080E946046A0913108A03019F40E9444
:105B10008E7309F407C0E7E0EA930E94937364D69A
:105B2000E89424F824FE24C00E949673EAE5F0E08D
:105B30000E949D7319F0AA81A130C9F481D6E0308A
:105B4000B1F00E94A3730FEF1FEF0E94EB720E944F
:105B5000C621E03021F40091270810912808EB813C
:105B6000EA93E0912F08EA931A930A933DD60BC06B
:105B70000E949673ECE2F1E00E949D7321F40E9472
:105B8000AA73E09330081981088124960895E09162
:105B9000C70BF091C80B0E94AE7311F4E2E00895B8
:105BA000E091C50BF091C60B0E94AE7311F4E1E0D9
:105BB0000895E091CB0BF091CC0B0E94AE7311F4E1
:105BC000E0E00895EFEF0895A0911908A23021F4C4
:105BD0000E9440470E947B0FA0911908A83009F449
:105BE00062D6A0911908A53009F449D1D9C0E2E0E4
:105BF000EA930E944741E2E0E0930E04E881EA93D1
:105C00003FDFA881AF3721F4E0912B06E37009F460
:105C100003C0E2E0E0931808A881A13239F0A33470
:105C200021F40E948173109709F004C0A091190813
:105C3000A23009F011C0A0911B08A33009F4DEDDE9
:105C4000A0911B08A23019F4E1E0EA93BDDFE091D6
:105C50001B08E03009F4D0DDA881AD3311F00C94BD
:105C60008C2E0E946046E0911B08E030B1F4E09178
:105C70002508F0912608FA93EA930E94EF21E0307C
:105C800051F4E0912508F09126080E942273E0E08B
:105C9000EA939ADF01C0B0DD3FC0E13079F477DFED
:105CA000EF3F41F0E3E00E94B2730E9472730E94E2
:105CB000B87303C0E1E0EA9387DF2EC0E230F1F46D
:105CC0000E948173A336E0E0BE07B4F4E09125089A
:105CD000EA930E94BF73E2E0E0930E040E94566CC8
:105CE0000E94566C0E9419470E94B06D0E94CC1011
:105CF000E3E0E0931B0801C081DD0EC0E33061F4F6
:105D0000E0912508EA930E945C19E0912508EA9346
:105D1000EEEFEA934DD872DDA881AD3409F46ADD67
:105D2000A881A43521F4A0911908A23009F001C07E
:105D300063DDA881AB3221F4EEEFEA930E94AB253C
:105D4000A881AD3221F4EFEFEA930E94AB25A88140
:105D5000A73421F4E1E0EA930E94AB25A881AB349B
:105D600021F4ECEFEA930E94AB251AC00E944F2168
:105D70000E944047E0E0E0931B08A881A13039F47D
:105D80000E948E7321F0A091CA0BA03009F402C0CA
:105D900033DD06C00E947B0F0E94EB720E94C62179
:105DA000219608951A930A930E94C3730E941020AB
:105DB0000E947B43E03091F10E94CC7378F10E9405
:105DC0007D7321DDE03051F50E94D4730E9488215B
:105DD000EF3F09F006C50E94EB720E94EF21E03010
:105DE00021F40E944120E13009F018C00E943020C7
:105DF000E83119F40E94D97309F001C0F2C40E947D
:105E0000D4730E94D8260E2F013021F4A091990B53
:105E1000A03009F403C01A930E94CB11A0912E0662
:105E2000AF3F61F110912E06EFEFE0932E061A932B
:105E30000E945C190E94EB720E94EF21E03021F475
:105E40000E944120E13009F019C00E943020E83161
:105E500019F40E94D97309F001C0C3C41A93EEEF7C
:105E6000EA930E94D8260E2F013021F4A091990BBD
:105E7000A03009F403C01A930E94CB11B2C40E944F
:105E80004F210E94D720E89421F8E0E0E0931E081B
:105E90000E94E0730E9440470E94566C0E94566C1C
:105EA0000E941947E09132060E94346EE091330659
:105EB0000E94346E0E94566C0E94B86D0E94194771
:105EC000E0913F060E94346EE0913906F0913A0667
:105ED0000E940A6E08950E94A47D0E94C3730E94CE
:105EE0007B43E03049F00E94CC7330F00E947D7318
:105EF0008ADCE03009F422DBE091540CF091550C7F
:105F00000E94D26E11F40C94E52F0E94E0730E945F
:105F1000566C0E94AB6D0E94F76DE0913706F091D0
:105F200038060E940A6EE0913B06F0913C060E9402
:105F30000A6E00E0053010F00C94E52FA7E10A9FEF
:105F4000F001E15DF94F9F01F901A381AF3FD9F164
:105F5000D9011A960E94166E7F936F93FF93EF9369
:105F60000E94E773AF91BF918F919F910E94DE7A5B
:105F70000E94217BDF01CB010E94EC73D9011C96AA
:105F8000ED93FC93F90104841584D9011E960E94B7
:105F9000C07BE015F105B9F0F90104841584A685EC
:105FA000B785F001EA1BFB0BE093AC0BF093AD0B54
:105FB000C5DAE13041F4D9011C960E94C07BD901B9
:105FC0001E96ED93FC930F5FB5CF0E94AB7D2AC464
:105FD0000E94A47D0E94C3730E9410200E947B43F4
:105FE000E03011F40C947E300E947E430E2F0A9311
:105FF000FEDD003820F0A091C605A03808F429C0C5
:106000000F770A930E94F3730E94EF721E2FA091E4
:10601000E20BA03011F41F3F09F416C030E0353018
:1060200098F4ABE03A9FF001E452FA4FE081E117B7
:1060300049F43A9FF001E252FA4FE081EF5FE093BA
:10604000C605232F3F5FEBCF0A930E94D4732A9398
:1060500054C0A091E20BA03021F4003810F00538B4
:1060600008F00AC00F770E9491721081EFEFEA9357
:106070000E94D4730A936CD9A091E20BA03011F066
:10608000003808F43BC00F770A930E945C19BBDB11
:10609000E030A1F50E94F6730E948821EF3F19F0CD
:1060A0000E94AB7DBFC30E944120E13039F50E94C0
:1060B0003520E03049F40E94F6730E94D826E03083
:1060C00011F00E94FB731AC00E943020E83141F4A5
:1060D0000E94D97321F00E94F6730E94D8260EC048
:1060E000A0911E08E02F0E948A6DAE0FBF1F1C9169
:1060F0000A930E94D473EFEFEA932AD9A0912E0657
:10610000AF3FF9F000912E06EFEFE0932E060A93D1
:106110000E94F3730E94EF721E2F0A931A93EEEF00
:10612000EA93EFEFEA9314D91F3F41F4A0919D0B3E
:10613000A03021F4A091A00BA03009F002C00E9471
:10614000FB7320FE0AC0E89420F8E091E20BE030F7
:1061500019F4FFD350D501C0AFD530E0353080F50C
:10616000ABE03A9FF001DF01EA51FA4FE081E03005
:1061700049F0AC51BA4F0E940174E8EEF3E00E947E
:10618000EF7099F4ABE03A9FF001EA51FA4FE081E9
:10619000E23051F43A9FF001EC51FA4FDF010E94D6
:1061A000C07B0E94D26E09F409C0ABE03A9FF001B7
:1061B000EA51FA4FA0E0A083689420F83F5FCECF69
:1061C0000E94AB7D2FC30E940D6DA33011F40C947F
:1061D0009C32E0913A08ED3411F00C94C531E09115
:1061E0003B08EA3511F00C947A3124FC83C0E0912D
:1061F0003C08E0532E2FE0913D08E0533E2FEEE3A4
:10620000F8E00E9419730E940D73AC91AB3429F42D
:106210000E9406740E944C620E2F0E940D73AC9176
:10622000A43529F40E9406740E944C62AF01E091EB
:10623000CD0BE31731F5E0E0E0934D0C0E94A37322
:106240004093270850932808A09130080A1759F066
:10625000E7E0E09318080093300820934C0CE0E04E
:10626000E0932F080DC0A0914C0C2A1721F0A091AB
:106270002E08A03009F004C02093180820934C0C7D
:1062800035C0A0913008A03049F4A091CE0B0E94F7
:10629000F16CE255FF4FE491EA2309F40CC0E7E00A
:1062A000E093180820934C0CE0E0E0932F08E09175
:1062B0003908E0934D0CE0913908A0914D0CEA1794
:1062C000A9F44093270850932808009330080E94AF
:1062D000A373A0914C0C2A1721F0A0912E08A03096
:1062E00009F004C02093180820934C0C273011F4B7
:1062F0000E941471E0913B08E93439F4E7E00E9410
:10630000B2730E94AA73E0932F08E0913B08E23435
:1063100039F4E4E00E94B2730E94AA73E0932F085C
:10632000E0913B08E03519F4E1E0E0931808E091D2
:106330003B08EC3449F4E4E0E0931808E0913C08B1
:10634000E053EA930E949516E0913B08E334E9F4A8
:10635000A0913C08A13320F0A0913C08A93308F09B
:1063600014C00E940974E0912208EA930E94B01BB5
:10637000E0913908EA93E6E8F8E1FA93EA930E949B
:106380003D700E94D37B0E942364E0913A08E0357F
:1063900021F4A0911908A13009F003C00E9477737D
:1063A00059DAE0913A08EF3459F4E0913B08EE34C1
:1063B00039F4E0913908EA93E9E8F8E10E940F74B2
:1063C000E0913A08E33569F5E0913B08EF3349F590
:1063D000A0913C08A03320F0A0913D08A03308F420
:1063E00020C00E940974E0913D08E0531E2FA09147
:1063F0002208A13210F41A3008F013C0103011F442
:106400000E94FA1AE0913908EA93ECE8F8E1FA936D
:10641000EA930E9470700E9453700E94D37B0E9486
:106420002364E0913A08E33411F00C946432E09173
:106430003B08EF3311F00C946432E0913D08E033F7
:1064400019F4EFEFE0932308A0913C08A033F8F093
:106450000E940974A0912208A132C8F4E091230897
:10646000EF5FE0932308E0912208EA93E09123088C
:10647000EA930E94761BA0911E0CB0911F0C1097FE
:1064800021F4A0912308A33608F001C0E7CFE091E2
:106490002308EA930E945C190E941574EFE8F8E162
:1064A0000E94FF720E94156F0E941A740E941F744E
:1064B0000E941A6F0E94D37B0E941F740E947C6FFF
:1064C0000E94A4630E94F363E0913A08E434A1F5CA
:1064D000E0913B08E43481F514E0E1E0E093390910
:1064E000103538F40E947671E85CF74FE081E032B5
:1064F00008F41AC00E947671E85CF74FE081E3323D
:1065000059F40E947671E75CF74FE081E053EA931B
:106510000E94C55E1F5F06C00E947671E85CF74F5F
:106520000E9449721F5FDCCF0E941574E2E9F8E116
:106530000E94FF720E94F3630E94A97D269608952F
:106540001A930A930E94277211F40C941C33E0E012
:10655000E093590CE0911808EF770E2F009318087C
:106560000E9440470E94B86DE4E0F0E0FA93EA939D
:106570000E941947013021F0A0911908A13009F0BB
:106580000BC0EEE8F5E00E94BD6D98D9E4EFF1E0B4
:106590000E94736C0E944047073049F40E944F21CB
:1065A000E0E0E0931B080E946C120E94F728043080
:1065B00031F4E5E9F8E10E94BD6D0E94300E08302B
:1065C00019F40E9425746FD1053019F40E942574C6
:1065D00056DC013051F4E89423F8E0E0EA9356D910
:1065E0000093190837D90E947B0F093071F4E0E05D
:1065F000EA934CD9E0E0E0931E08E89423F80E9467
:106600007B0F0E942F74E093590C023069F4E0E094
:10661000E0931E08E0E0F0E00E942273E89423F883
:106620000E942F74EA93A2DB033011F40E94F94018
:10663000009319080E941020A0911908A73011F0AA
:106640000C94CA33E091520CF091530C0E94D26E1C
:1066500021F0A0911B08A03009F00AC00E94B2727C
:10666000E0914E0CA0912306EA1711F00E94F72842
:106670000E947B43E030E9F0E2E00E946B731A93E2
:10668000FFD91D3409F4B6D81D3399F40E94604631
:106690007EDAEF3F41F0E3E0E09318080E94727366
:1066A0000E94B87306C0E7E8E0931808E0E0E093C2
:1066B0001B08A0912F08A03031F0E0912F08A09185
:1066C0002E08EA1709F457C0E0912F08E150EA9329
:1066D0000E94B119A091340CE1E0EA23E13021F4E9
:1066E000E0912B06EF7C09F429C0E0E0E0932E084E
:1066F000E0914C0CE03019F0E09318081EC012E055
:10670000E0912B06EC7009F018E0E091C40BA09129
:106710002F08EA1781F0E0912B06E07439F011E0C0
:10672000EAE2EA93EAE9F8E10E940F74E0912B06AD
:10673000E07809F019E0109318081DC00E94404746
:106740000E946C120E94B86DE4E0F0E0FA93EA93C4
:106750000E941947EBE4EA930E94B746E0912F08A4
:10676000EA930E94E841EDE9F8E10E94BD6DE091F5
:106770002F08E0932E08A0912F08A03021F4A091BB
:106780002E08A03009F406C0E0E0E0932E08E7E808
:10679000E0931808A0911908A33011F40E94F63E66
:1067A000A0911908A13009F4D9D8A0911908A230F4
:1067B00009F4F8DAA0911908A83009F409DCA091CD
:1067C0001908A53009F487DBA0911908A93049F40C
:1067D000E0E0E0932008E0911908EA93E0E0EA9312
:1067E00080D90991199108950E943674E652F84FA4
:1067F000A6E0A0830E943674E752F84FAB81A083D5
:106800000E943674E152F84FAA81A0830E94367428
:10681000E552F84FA881B981A083B1830E9421720B
:106820000E947551249608950E943C74A881B981F4
:10683000AC91A53020F0A881B981E0E0EC9387C04D
:10684000A0911308BB27E091120805C0A091110880
:10685000BB27E0911008F0E031960E94C270359697
:10686000DF01E5E0F0E00E94797B08951A93109132
:106870001308E0911208E117A1F0ABE01A9FF001B4
:10688000E652F84FE081E13011F0E23011F4E1E03E
:106890004BC0EDB7FEB7FA93EA931F93C5DF1F9184
:1068A000E8CFE0E041C01A930E944F21ECEDF5E003
:1068B0000E9487700E94396D0E94EA6810E01530CE
:1068C00068F40E94F570AFEFA083ABE01A9FF0016F
:1068D000EE51FA4F0E94AD721F5FF1CF10E01530FC
:1068E00048F4A7E11A9FF001EC5CF94FAFEFA083E9
:1068F0001F5FF5CFE0912B06E37019F00E948E73B5
:1069000009F402C0689401C0E89421F8EFEFE09325
:106910002D08E091E20BE03029F41BD06CD1E89413
:1069200020F802C00E940010199108951A9310E0F7
:10693000153058F40E94F570E081AE2FE981EA1716
:1069400011F4E12F03C01F5FF3CFEFEF1881229600
:10695000089522970E94A27D00E0053058F40E941D
:106960004274A0E00E944874E152FA4FA0E0A08374
:106970000F5FF3CF00E00530C0F50E949172E08117
:10698000EF3F89F10E949172E0810E940471B9F099
:106990000E949772DF010E94C07B0E94D270EA17AA
:1069A000FB0751F00E9497720E94D270A083B183BE
:1069B0000E944D74A1E0A0830E94427412C0ABE01B
:1069C0000A9FF001EA51FA4FE081E03061F40E9441
:1069D0009172AFEFA0830E9497720E94AD720E94E5
:1069E0004D74A1E0A0830F5FC6CF0E94301F1E2F01
:1069F0001F3F11F0E1E001C0E0E0E093590C1F3FC0
:106A000011F40C94553550E000E0053048F40E9434
:106A10009172E0811E1711F451E002C00F5FF5CFB3
:106A20005030E1F500E00530C8F50E949172E08138
:106A3000EF3F91F50E94917210830E9497720E941D
:106A4000D270A083B183ABE00A9FF001E052FA4F0D
:106A5000A091290C0E944874EF51FA4FFF93EF93D5
:106A60000E94FF700E940C70AF91BF91EC930E9446
:106A70004D74A1E0A0830E944274A1E00E9448747A
:106A8000EC51FA4FFF93EF930E948C68AF91BF9146
:106A9000ED93FC9351E002C00F5FC5CF503029F059
:106AA0001A930E94371F1E2FAACF30E0353010F006
:106AB0000C949B35A7E13A9FF001E15DF94FEE831D
:106AC000FF8350E000E0053048F5503029F5ABE099
:106AD0000A9FF001EF51FA4F20812A930E945C191E
:106AE0000E944274E081E13059F42A930E945120BF
:106AF000E13031F4A32FAF5FE0919D0BEA1709F06D
:106B00000BC0E22FAE81BF811396EC93E02FAE81D4
:106B1000BF811596EC9351E00F5FD5CF503049F40B
:106B2000AE81BF811396EFEFEC93AE81BF811596D6
:106B3000EC933F5FBBCF0E94A97D0C9443380E9429
:106B4000A47DAC81BD81EBE4EC93EC81FD813196B9
:106B5000FA93EA930E945374E052FA4FE0810E9444
:106B6000B16C00E00E945C74EC91E03011F00F5FBA
:106B7000F9CF0E945C74E0E2EC930F5F0E946274B4
:106B80000E94656D0E945374EE51FA4FDF010E941E
:106B9000166E0E946774EE81ABE0EA9FF001EF5140
:106BA000FA4F10811A930E945C1900E00E945C74F5
:106BB000EC91E03011F00F5FF9CF0E945C74E8E7D0
:106BC000EC930F5F0E945C74E0E2EC930F5F30E0A7
:106BD0003A3060F40E946274EA0FFB1F0F01AAE8CA
:106BE000BBE00E946E740F5F3F5FF2CF0E945C7447
:106BF000EC930C94883864970E94A47D00E010E028
:106C0000153040F40E94F570E081EF3F09F40F5F0A
:106C10001F5FF6CF053021F0A0912D08A03009F4B8
:106C200006C0E0E0E0932D08EA930E94191110E0FD
:106C3000153088F5ABE01A9FF001E152FA4FE08180
:106C4000E03039F11A9FF001E352FA4FE081E03071
:106C5000B1F01A93FE0135960E949D72ABE01A9F27
:106C6000F001EF51FA4F30813A930E945C191A9368
:106C7000FE013596FA93EA930E9474110AC01A93A2
:106C80000E946411ABE01A9FF001E152FA4FA0E0BC
:106C9000A0831F5FCDCF053021F4A0912D08A13036
:106CA00009F406C0E1E0E0932D08EA930E9419116F
:106CB0000E94AB7D689608950E94A27DA091E20B90
:106CC000A23011F40C94223A30E0343168F40E947E
:106CD00075740E947874DA011296E0E0EC93DA01A0
:106CE000EFEFEC933F5FF1CF0E94301F0E2F0F3F6D
:106CF00011F0E1E001C0E0E0E093590C0F3FA1F199
:106D00000E94FF70FA93EA930E940C191E2F1F3FF6
:106D100031F1A0911E08E12FEA1B3E2F3431F8F427
:106D20000E9475740E947874FA0132960F01E08116
:106D3000AE2F0E947E74B0E0EA0FFB1FD001EC93EF
:106D4000FA01A281A43620F0DA011296E3E6EC9370
:106D5000DA01AC91AF3F19F4E02FDA01EC930A931A
:106D60000E94371F0E2FCACF0E94AE1530E034317B
:106D700010F00C9441370E9475740E947874FA01E7
:106D8000A381AF3F11F40C943F370E9483740E949B
:106D90000270E83139F40E948374EA930E94531818
:106DA000E03009F408C00E948374EA930E945318EB
:106DB000DA011296EC93A0919A0BA07839F4FA01BB
:106DC0000280DA011196EC91E01509F458C0DA015D
:106DD00013962C91ADE02A9FF001EF5EFC4F0F015E
:106DE000DA011296EC91D001EC930E948374EA933D
:106DF0000E946521EF3F29F0ADE02A9FF0010E943B
:106E00006A6DDA011296EC91E03089F00E94887484
:106E1000DF010E94856DEC93ADE02A9FF001E25FF7
:106E2000FC4FDF01E091980BEF70EC9313C00E94D0
:106E3000856DE03021F40E948874A0E003C00E94B8
:106E40008874A8E0A083ADE02A9FF001E25FFC4FC8
:106E5000A7E0A0830E948374EA930E946521EF3F1C
:106E600019F0ECE0E0930F04DA011296EC91DA01EC
:106E70001196EC932A93E1E0EA930E94A2473F5FC8
:106E800076CF0C94223AE7E0E09318080E94951818
:106E9000A8950E94F71CA8950E944C1FA895EFEF9B
:106EA000E093B20BE093890BE093330CE0932E0C4C
:106EB000E0932E060E948E74EC7F29F0A8E0B0E0EB
:106EC000E0E00E94027C089524970E94A47D0E9425
:106ED0009642EAEAF8E10E9487700E9422430E94EB
:106EE000BE42E0912208E03061F0E5EBF8E10E945B
:106EF00087700E942243E09122080E9493740E94AE
:106F000097740E94BE420E94FA1A00E00A30A0F470
:106F10000A930E948B190E94A26FEFE0EA930E94ED
:106F2000FC42E02FA3EAB6E00E949B740E945370DB
:106F30000E949F740F5FEACF0E94D042EEEBF8E10F
:106F4000FA93EA93EFE0EA930E9422430E94E26EF2
:106F50000E949F740E94D2420E94BE4210E01031F3
:106F600010F00C943F380E94236EE117E1F5E4EC39
:106F7000F8E10E9487700E9422430E94A66D0E9441
:106F80009774E0E0E0931E08A0911E08A33648F530
:106F9000E0912208EA93E0911E08EA930E94761B92
:106FA0000E94156F3097B9F0E0911E08EA930E9495
:106FB0005C190E94156FFA93EA930E94A5740E94CF
:106FC00022430E947C6FEAE0EA930E94FC420E9406
:106FD0001A6F0E949F74E0911E08EF5FE0931E08F5
:106FE000D3CF0E94AA740E9476710E94587011F04B
:106FF0000C943D38E4ECF8E10E9487700E94224333
:107000000E94A66D0E9497740E94AE74E0E30E94F5
:10701000647029F40E9469700E944C629F010024F0
:107020000216030644F50E9406740E9476620E94CE
:107030008A6E0E9406740E94B6743A932A930E9444
:10704000A5740E9422430E94BA74EAE0EA930E9467
:10705000FC42EC81FD816E817F810E949F740E94C1
:10706000AE74E1E30E94647029F40E9469700E948A
:107070004C629F01D4CF0E94AA741F5F70CF0E9400
:1070800097420E94AB7D289608950E94A47DAD8111
:10709000BE812C910E94BF740E94A66D0E94D96C83
:1070A0000E941F6EECE3EA930E94B746EC81EA93DC
:1070B0000E940B472A93ED81EA930E948841EEE3F8
:1070C000EA930E94B7460E943F730E94DF720E94BB
:1070D00045730E94C474333409F431E2313320F033
:1070E000EC81E05DE31708F407C0E32F0E948B7387
:1070F000E255FF4FE4912E273D3311F0313209F470
:1071000001C0CACF3D3319F4AD81BE812C93E32F6A
:107110000E94AB7D279608950E94A27D20E0AF815A
:10712000B8855C910E94BF740E94A66D0E94D96CC4
:107130000E941F6EE2E0EA930E940B475A930E945E
:10714000E8410E943F730E94DF720E9445730E94D3
:10715000C474303310F03A3308F00EC0203009F414
:1071600050E021E0A52FEAE00E94767BAAE0EA9FAA
:10717000F001E30FE0535E2F3B3211F4533608F079
:1071800001C05F5F3D3211F4513008F401C051502D
:10719000333429F4203009F431E250E020E03D336B
:1071A00019F4EE81E51708F005C0AF81B8855C9150
:1071B00030E020E03D3311F0313209F401C0B4CFAA
:1071C0003D3319F4AF81B8855C93D0C00E94A27D95
:1071D00020E0AF81B8854D915C910E94BF740E9400
:1071E000A66D0E94D96C0E941F6EAE81A23051F430
:1071F000E6E0EA930E940B47FA010E941A740E948B
:10720000C74108C0E5E0EA930E940B475A934A93AE
:107210000E94D2410E943F730E94DF720E94457318
:107220000E94C474303310F03A3308F01EC020308E
:1072300011F440E050E021E04031E7E25E0734F035
:10724000DA01E0E1F7E20E94797BAF01493BEBE034
:107250005E0724F0DA010E948673AF01DA010E9412
:10726000C9740E94CE74D097AD013B3221F44033F3
:10727000E5E75E070CF002C04F5F5F4F3D3221F43F
:107280000024041605060CF002C04150504033346F
:1072900031F4203009F431E240E050E020E03D33A9
:1072A00011F0313209F401C09ACF3D3321F4AF819E
:1072B000B8854D935C935AC00E94A27D0E94BF7412
:1072C00020E050E04FEF0E94A66D0E94D96C0E9412
:1072D000D3740E94D674E885EA930E94E346E52FB2
:1072E000E10FF0E00E94DF720E9445730E94C474B7
:1072F000303310F03A3308F021C03053431729F0EF
:107300004F3F09F05F5F20E005C0A22FAF5FEA2F7B
:10731000E3702E2FE52FAF81B8850E94DB740F013B
:10732000E32FA6ECB6E00E949B74AE0FBF1FE22FC6
:107330000E94DB74E491D001EC93432F3B3219F4AB
:10734000EE815E1708F002C05F5F4FEF3D3211F42F
:10735000513008F402C051504FEFEE815E1720F417
:10736000313211F03D3309F401C0ADCFE32F0E945B
:10737000A97D299608951A930A93A0919A0BECED92
:10738000EA231E2F00E00D3040F40E94DF740E94BB
:10739000E374E11711F00F5FF6CF0E94DF74EA0F7C
:1073A000FB1F0E94CF7B0E94BD6DE02F3DC4AAE968
:1073B000BBE00E940E6EAE0FBF1FEC91E17011F4A6
:1073C000E3E701C0E9E4EA930E94B74621960895F5
:1073D0000E94A27D0E94BF740E94A66D0E94D96C7B
:1073E0000E94D374C8DF5E2F0E943F730E94DF7239
:1073F0000E9445730E94C4743D3211F0363311F47B
:10740000503009F401C051503B3211F0333311F4C4
:107410005C3008F001C05F5FA0919A0BE1E0EA23C5
:107420002E2FE52FA0E0B2E00E949B740E94E3742F
:10743000E20FE0939A0B3D3311F0313209F401C0B1
:10744000CBCFE32F0E94A97D269608950E94A47DAC
:107450000E94BF740E94A66D0E94D96C0E94D374D2
:10746000AAE9BBE0EC810E94FE6FEC91E17019F497
:10747000E1EDF8E102C0E5EDF8E1FA93EA930E944C
:10748000CE460E943F730E94DF720E9445730E94A5
:10749000C474303310F03A3308F00FC0AAE9BBE0EF
:1074A0000E9422700F01AAE9BBE0EC810E94FE6FEE
:1074B000AC91E1E0EA27D001EC933D3311F0313299
:1074C00009F401C0C7CFE32F0E94AB7D2596089534
:1074D0000E94C16CE1E0EA930E941A0F0E94566C70
:1074E0000E94566C0E9419470E947C6FEAE0EA9362
:1074F000E3DEE13209F45FC40E94566C0E94566CD0
:107500000E94F76DE9EDF8E10E94BD6DE5E9FBE051
:107510000E9487705BDEE13209F44DC40E94566C14
:107520000E94566C0E94F76DEFEDF8E10E94BD6D70
:10753000E091970BEF5F0E2FEDB7FEB7FA93EA934A
:107540000F93EAE0EA93E8DD0F91E13209F433C4E6
:1075500000240216030624F4E02FE150E093970B79
:107560000E94566C0E94566C0E94F76DE8EEF8E19E
:107570000E94BD6DECEAFBE00E94E87409F41BC4B4
:107580000E94566C0E94566C0E94F76DEEEEF8E178
:107590000E94BD6DEEEAFBE00E94E87409F40BC4A2
:1075A0000E94566C0E94566C0E94F76DE4EFF8E161
:1075B0000E94BD6DE9E9FBE0FA93EA93E3E60E94DD
:1075C000F17409F4F8C30E94566C0E94566C0E9434
:1075D000F76DEDEFF8E10E94BD6DFADEE13209F4DE
:1075E000EAC310E0133010F00C94AD3B0E94566CCF
:1075F0000E94566C0E94F76DE12F0E944973E3E0F0
:10760000F9E10E94BD6D0E94F6740E941947ADE930
:10761000BBE00E9476710E94656DE0E10E94F1740A
:1076200009F4C9C3E9E0F0E00E94976C0E94194791
:10763000A0EABBE00E9476710E94656DE0E10E94C5
:10764000F17409F4B8C30E94566C0E94566C0E94F3
:10765000F76DE12F0E944973EEE0F9E10E94BD6DE4
:107660001A93F4DEE13209F4A6C30E94F6740E9474
:10767000FA7451F40E9431720E940475E2E00E9493
:10768000077509F498C309C00E9431720E940475FD
:10769000E0E00E94077509F48EC30E94566C0E94B8
:1076A000566C0E94F76DE12F0E944973E0E1F9E109
:1076B0000E94BD6D0E94F6740E941947A9EABBE0C2
:1076C000EE27A10FBE1F2C913327EDB7FEB73197E0
:1076D000FA93EA933F932F93E0E0EA9377DD2F91BB
:1076E0003F91E13209F467C3A9EABBE00E947671D9
:1076F000EA0FFB1F2083123070F50E94566C0E9427
:10770000566C0E94F76DE12F0E944973E7E1F9E1A1
:107710000E94BD6D0E94F6740E941947A0EBBBE069
:10772000EE27A10FBE1F2C913327EDB7FEB731977F
:10773000FA93EA933F932F93E0E0EA9347DD2F918A
:107740003F91E13209F437C3A0EBBBE00E947671B0
:10775000EA0FFB1F20831F5F45CF2DC30E94A47D2E
:1077600010E01A930E94BF730E940C750E94566C21
:107770000E9419470E942F6E0E9410750E94B06DE2
:107780000E9407700E940A6E0E94566C0E94B86D9B
:107790000E9419470E9415700E941B6EE7E0F0E0FE
:1077A000FA93EA930E94B86D0E941947E091AE0BDC
:1077B000F091AF0B0E94DE7A0E941B6E0E94566C05
:1077C0000E94AB6D0E941947EEE1F9E10E94BD6D88
:1077D000E091970BEF5FEA930E94E841E7E0F0E069
:1077E000FA93EA930E94AB6D0E941947C4DD0E9490
:1077F000FB6DE091990BE03029F0E091990BEA9351
:107800000E94E84100E00330D8F50E94566CE02F5A
:10781000ED5FF0E00E941F6E0E945E72EA930E948C
:10782000E841EBE2EA930E94B7460E946572EA9350
:107830000E94E8410E94FB6D0E946C7251F40E940C
:1078400074720E94116E0E94166E0E941475E3E716
:1078500009C00E9474720E94116E0E94C07B0E9437
:107860000A6EE9E4EA930E94B7460E94FB6D0E940B
:107870007E72EA930E94EE410E9418750F5FC3CF9B
:107880000E947E433E2F3B3211F4133608F001C0B4
:107890001F5F3D3211F4113008F401C011503D3426
:1078A00039F41A930E945C1913DE1A930E947C1912
:1078B000313209F056CF7FC20E94A47D10E00E94B1
:1078C0004047012F0E94566C0E94566C0E94194737
:1078D000E2E2F9E10E94BD6D31E03C3018F510386C
:1078E000F8F40E94566C0E94F16C0E941F6E1A936D
:1078F0000E94B1190E942F6E0E94FB6DA091340C62
:10790000E3E00E941C75A091350CE7E00E941C7515
:10791000E0912B06EA93E8E0EA930E9488411395F0
:107920003F5FDBCF0E94300E0E947E433E2F3D34EE
:10793000E9F50E942773102F1038C0F51A930E94A2
:10794000B1190E94566C0E94566C0E94F76DE6E3D6
:10795000F9E10E94BD6D0E942F6E0E9410750E9479
:10796000366E0E941947E9E3F9E10E94BD6DE4E338
:10797000FCE0FA93EA93E3E00E94F17409F41BC27D
:107980000E94366E0E94F76DEFE3F9E10E94BD6D33
:10799000E5E3FCE0FA93EA93E7E00E94F17409F46E
:1079A0000AC21A930E94E5191F5FC6CF313211F047
:1079B000103808F001C083CFFEC10E94C16C0E9444
:1079C0000C750E94566C0E941947E5E4F9E10E948B
:1079D000BD6D10E01530F0F41A930E94F3190E9467
:1079E000566C0E94F86E0E942F6E0E941075E091F6
:1079F0002F0C0E942175E091320C0E942175E091BC
:107A0000300C0E942175E091310CEA930E94EE4106
:107A10001F5FE0CF0E947E430E2F0D34E9F50E94D8
:107A2000277310E01530C0F51A930E94F3190E94D5
:107A3000566C0E94566C0E94F76DE8E5F9E10E94D1
:107A4000BD6D0E942F6E0E94107530E03430F8F446
:107A50000E94366E0E94F76D0E94F16C0E94D17AEE
:107A6000EA55F94F0E94CF7B0E94BD6D0E94F16CD8
:107A70000E94D17AEA55F94F0E942575FD0135968D
:107A8000E4910E94F17409F496C13F5FDFCF1A932D
:107A90000E94131A1F5FC6CF8EC10E94326CE1E0B4
:107AA000EA930E941A0F00E0083210F00C94143E82
:107AB0000E94FC0D0E94566C0E94566C0E94194751
:107AC0000E94D96C0E9428750E94CF7B31960E943B
:107AD000BD6D0E94FB6D0E94D96C0E942875349682
:107AE000E491E038A9F40E94236E1E2FEDB7FEB793
:107AF000FA93EA931F93E0E1EA930EDB1F91E132E0
:107B000009F492C0E12FA9E0B0E00E94027C88C095
:107B1000E238A9F40E948C701E2FEDB7FEB7FA93DD
:107B2000EA931F93E0E1EA93F7DA1F91E13209F457
:107B30007BC0E12FAAE0B0E00E94027C71C0E13876
:107B4000E1F40E948E741E2FEDB7FEB7FA93EA930C
:107B50001F93E3E0EA93E0DA1F91E13209F464C095
:107B60000E94FC0D0E948E74E11731F0E12FA8E015
:107B7000B0E00E94027CFFCF53C0E03069F40E9465
:107B8000D96C0E94287532960E94C16DE1E00E9476
:107B9000F17409F449C044C0E13069F40E94D96C21
:107BA0000E9428750E942575FD013596E4910E947A
:107BB000F174D1F135C0E23061F40E94D96C0E94B9
:107BC000287532960E94C16DEFE00E94077561F141
:107BD00027C0E33071F40E94D96C0E9428750E947E
:107BE0002575FD013596E491EA934FDAE132E1F033
:107BF00017C0E430A9F40E94D96C0E94287532960F
:107C00000E94CF7BE0935A0CF0935B0C0E94DF72D2
:107C10000E9428753596E491EA934EDBE13221F01B
:107C20000E9498180F5F40CF099119910895E8813B
:107C30000E944973ECEDF8E10E94BD6D0C949442F2
:107C40001A930E94277310E0133010F00C94793EC1
:107C50000E94566C0E94566C0E94F76D1A93E7DFE3
:107C6000ECE0F0E00E94976C0E9419471A939FDBAA
:107C70000E94F6740E94FA7451F40E9431720E94BC
:107C80000475E2E00E94077509F4FFC209C00E9472
:107C900031720E940475E0E00E94077509F4F5C294
:107CA000123028F50E94566C0E94566C0E94F76DA7
:107CB0001A93BDDFEBE5F9E10E94BD6DECE0F0E069
:107CC0000E94976C0E9419470E941875EAE0F0E044
:107CD0000E94976C0E941947A0EBBBE00E9476714E
:107CE0000E94656DE3E60E94F17409F4CEC21F5F45
:107CF000ABCFCBC20E94A47D10E01A930E94BF7349
:107D00000E940C750E94566C0E9419470E942F6EAB
:107D10000E9410750E94B06D21E000E0033080F5F4
:107D2000E3E0F0E00E94086D0E941F6E0A937FDF7F
:107D30000E946C7249F40E9474720E94116E0E943B
:107D4000166E0E94147508C00E9474720E94116E13
:107D50000E94C07B0E940A6E0A9329DB2F5F0230CB
:107D600068F4E7E0F0E00E94086D0E941F6E0E9438
:107D700077720E94346E0E9418752F5F0F5FCECF0E
:107D80000E947E433E2F3B3211F4133608F001C0AF
:107D90001F5F3D3211F4113008F401C011503D3421
:107DA00039F41A930E945C194BDF1A930E947C19D4
:107DB000313209F0A2CF0E94AB7D249608950E9433
:107DC00027730E94566C0E94566C0E941947E1E688
:107DD000F9E10E94BD6DE1E0E0932208E2E2F8E003
:107DE000FA93EA93E0E2EA9397D9089522970E94E2
:107DF000A27D0E947E430E2FE0911B08E03011F01F
:107E00000C94A7400132D1F4EAE4F6E0A0913A0CD8
:107E1000B0913B0CEA17FB0761F4E7E0E093180828
:107E2000EAE2EA93EAE6F9E10E9487700E94306490
:107E3000A8C0E0E0E093C0050E942D750D3331F439
:107E4000E091C005F0E00E94F76C04910D3441F41C
:107E5000EAE2EA93EDE6F9E10E9487700E9430645D
:107E6000063449F4E2E7F6E0E0933A0CF0933B0C79
:107E7000E0E0E093C005003311F00B3229F4E0910B
:107E8000C005EF5FE093C0050D3229F4E091C00515
:107E9000E150E093C005013329F491DFED3311F493
:107EA0000E943475033321F48ADFED3309F40CD8D2
:107EB000063329F4E0E0E09322080E94643704339B
:107EC00029F4E0E0E09322080E943475A091240890
:107ED000A13010F40C943D40023301F570DFED3316
:107EE000E9F40E944175D1F4E0912208EA930E94DE
:107EF000B01B30E0303190F40E94F16C0E94587059
:107F000059F4E32FE05DEA93E0E7F9E10E945D7048
:107F1000E0E3EA930E9452643F5FECCF053331F512
:107F2000E0E0E09322080E94417501F511E0113272
:107F3000E8F41A930E94B01B30E03031A8F40E949C
:107F4000F16C0E94587071F4E32FE05DEA93E0E772
:107F5000F9E1FA93EA93E12FE05DEA93E0E3EA9333
:107F60000E9452643F5FE9CF1F5FE1CF013469F4A3
:107F7000EAE2EA93E3E7F9E10E940F74E1E0E093BB
:107F800018080E94A97D289608950A3409F4B2DEE3
:107F9000073311F00C943D400E944047E0E0EA9323
:107FA0000E94610EE1E0E0931C08E0E0F0E0E09365
:107FB0001408F0931508EFE2F6E00E948770E3E7FB
:107FC000F0E00E9439700E948C68EE83FF830E946B
:107FD0004A75E8E2F0E00E94EF70B9F00E94AF123B
:107FE0000E948C68EE83FF83A091190CA03021F0D1
:107FF0000E942034E03009F408C00E943674E65232
:10800000F84FAEE0A0830E942172E5E0F0E00E940C
:10801000736C40E050E00E941822E03868F00E9443
:108020001822EF573E2F313010F0313108F004C0E4
:10803000E32F0E944371AF015A934A930E94EA1FB3
:1080400040931408509315080091DB05E0E0E0939D
:10805000DB05013211F00B3209F401C0B8CF0B324D
:1080600021F4E1E0EA930E94610E013209F0A3CF0E
:10807000E0E0E0931C08E093DB05A0912408A23027
:1080800011F00C94A040093309F407DD053409F41C
:1080900094DC033611F40E94A40D083309F45EDB6E
:1080A000023409F409DC0334B1F51091390C0E9453
:1080B000404700E0E091380CE11711F00C3008F077
:1080C0001DC00E94566C0E94D96C0E941F6E1A93AC
:1080D0000E943E1F1A937CD10E94FB6DE091290CF7
:1080E0000E942175E0912C0C0E9421750E94FF7066
:1080F0000E940A6E0E94E5700395DCCF0E94300E4C
:108100000E947E430E2F013221F0E091380CE117DE
:1081100009F401C0CCCF043499F40E94417581F474
:10812000A091D30BA03021F4A091D10BA03031F05D
:108130000E9493730E94566C0E94A5530E948C1D4E
:10814000E0911B08E03011F40E94B90E49C0E13003
:10815000D1F4A0912108AB3010F4013209F405C02C
:108160000E9445160E94300E0DC0E0E0E0931E080C
:108170000E944F750E940F74E0E00E945475E2E087
:10818000E0931B082DC0E23059F5013269F4E0E0BC
:10819000E0931B080E944047EAE2EA93EDE6F9E12A
:1081A0000E940F740E94B90E0B3211F00D3359F476
:1081B0000E944F75FA93EA93E1E3EA930E943064D8
:1081C000E1E00E9454750D3259F40E944F75FA9304
:1081D000EA93E2E3EA930E943064E2E00E9454757D
:1081E000A0911808A33009F404CE0E94A97D0C9434
:1081F000EA451A93E3E0E09319080E9440470E9481
:10820000566C0E94566C0E941947E9E7F9E10E94FA
:10821000BD6D0E94566C0E94B86D0E941947E3E143
:10822000F6E00E948770E0E1F0E00E94397010E013
:10823000E091C90B1E1700F50E94236EE117D1F0E3
:10824000E12FE05DEA93E1E8F9E1FA93EA93E0E3F4
:10825000EA93E0E00E94647049F40E947671ED5E5A
:10826000F94FA1E0A083E12FE05D01C0EEE2EA93C7
:108270000E94B7461F5FDCCF0E942D75E0E0E093BF
:10828000C005E0931B080E94B90E19910895E8817A
:10829000E03021F4E4EFF6E00E945975A881A130A6
:1082A00021F4EEEEF6E00E945975A881A23021F487
:1082B000EAEFF6E00E945975A881A33021F4E8E0C6
:1082C000F7E00E945975A881A43021F4EEE0F7E0B0
:1082D0000E94597529C11A930A93E0E0E0937D0545
:1082E000E0937E0510E0143190F400E0033068F470
:1082F000A3E01A9FF001EC57FA4FDF01EE27A00F21
:10830000BE1FE0E2EC930F5FF1CF1F5FECCFE9C33C
:108310001A9311E0E981E11780F00E947671E2552D
:10832000FF4FE491AA81EA2319F0E12FE05D01C03B
:10833000E0E2EA931CD51F5FEDCF2DC51A9311E043
:10834000E981E11778F00E947671E255FF4FE491E0
:10835000AA81EA2311F0E1E301C0E0E3EA9307D543
:108360001F5FEECF18C52A97A0911B0CA13038F0E3
:10837000EA85FB856C857D850E94147507C00E9487
:108380005E750E9462750E945E75F9D426C12A97B7
:108390000E945E750E946B750E9474750E945E75E6
:1083A000EED41BC12A970E945E750E9487750E94B9
:1083B0008E75E5D41FC12A970E945E75EFE9F9E139
:1083C0000E9493750E941A740E948E75D8D412C1AF
:1083D0002A970E945E75E2EAF9E105C02A970E9499
:1083E0005E75E6EAF9E1FA93EA93EE850E94B16CD4
:1083F0000E945E75C4D42B9608950E94A47D10E05F
:10840000E1E3E0933809E89431F8EA930E94D863F5
:10841000EAEAF9E10E94FF7200E0E09182050E179E
:10842000E0F40E94D96CEC57FA4FE081E03258F446
:10843000E3E2EA930E941A630E94D96CEC57FA4F68
:10844000E081E05D05C00E94D96CEC57FA4FE081F5
:10845000EA930E941A630F5FE0CF0E9498759F0114
:108460000E94B7153A932A93E8ECF0E0FA93EA9366
:108470000E9498680E2FA0E031FCA1E0A03011F41A
:10848000003009F001C0ECCF31FE09C0E0E0E0931C
:108490008205E89431F8E1E00E94AB7DEFC41F5FF4
:1084A000123008F4ADCFE0E0E09382050E94AB7D8E
:1084B000E5C4E0918105E03021F4E881EA930E946F
:1084C000C55EA0918105A13069F4A0E09299A1E078
:1084D000A13021F4A8950E94236FF7CFE881EA9399
:1084E0000E946561A0918105A230F1F4E0918205BE
:1084F000F0E0EC57FA4FA881A083E0918205EF5F8E
:10850000E0938205E0918305EF5FE0938305A0325D
:1085100018F4EF5FE0938305A0918305A83320F062
:108520006CDFE0E0E09383052196089508950E94B2
:10853000AA740E94AA7422D0EBE1EA93BADFE9E6BA
:10854000EA93B7DFA0918105A13061F4E8ECF0E097
:108550000E94936EE0919A00E069E0939A00E9E14D
:10856000E0939900A0918105A23021F446DFE0E07C
:10857000E0938305E0E0E09381050895EDE0EA9360
:1085800098DFEAE0EA9395DF08951A9310E0E98115
:108590001E1728F4EA81EA938CDF1F5FF8CFFBC334
:1085A000EDE201C0EDE3EA93E8E2EA93EEDFE6DF15
:1085B00008952A97A0911B0CA13038F00E945E7597
:1085C0000E946B750E94747504C00E945E750E94C3
:1085D0006275FE010E9487700FD02E9608952A972B
:1085E0000E945E750E9487750E949C75FE010E9424
:1085F000877002D02C9608951A930A9310E0EA81AE
:10860000E03011F408E201C00A81AB81BC81EE27A1
:10861000A10FBE1FAC91A03011F0101708F007C0D9
:10862000AB81BC810E94A1750E94A675EECFEA8144
:10863000E03039F0EA811E1720F4E0E20E94A675CE
:10864000F9CF27C01A930A9310E0EA81E03011F4C1
:1086500008E201C00A81E12FAB81BC810E94DB747A
:10866000E491E03011F0101708F009C0E12FAB8160
:10867000BC810E94DB74E4910E94A675ECCFEA8174
:10868000E03039F0EA811E1720F4E0E20E94A6757E
:10869000F9CF1981088125960895E091C405A0912C
:1086A000C305EA17B1F00E94AB750E94116EEC9100
:1086B000E093C6050E94AB750E949071E181E09342
:1086C000C505A091C4050E94B175E093C405E1E021
:1086D0000895E0E008950E94B675A981A0830E94E4
:1086E000B6753196A881A083A091C3050E94B1758B
:1086F000E093C305BFC0E091DB0508951A93E091B4
:10870000DB05E03059F40E94B7150E94277221F46E
:10871000A091DB05A03009F001C0F5CF1091DB0579
:10872000E0E0E093DB050E94277209F011E2E12FFF
:10873000D6C30E94A47D0E948C688F010E94B71549
:10874000EC81FD81E00FF11FFF93EF930E948C6895
:10875000AF91BF91AE1BBF0B9D0100240216030613
:108760001CF40E94277209F001C0E8CFE0E00E94EB
:10877000AB7D269608951A93E9810E948B72A0E042
:10878000A0830E94BC75108117FF05C0E12F0E94D5
:10879000C375A0E0A08316FF05C0E12F0E94CA7533
:1087A000A0E0A0830E94BC75A0E0A083E9810E94A4
:1087B0008572A0E0A08318815DC00E94A47D30E096
:1087C000EE81ADE0EA9FF001E05FFC4F108116FF03
:1087D00017C0E12FEF730E2F0E94D17511F03A30C0
:1087E00008F009C00E94D975DF010E94F16C0E9457
:1087F000DF753F5FF1CF0E94D9750E94CE74EC9374
:1088000017FF17C0E12FEF730E2F0E94D17511F0E3
:10881000343108F009C00E94E575DF010E94F16C57
:108820000E94DF753F5FF1CF0E94E5750E94CE7414
:10883000EC930E94AB7D42C2E881F9810E94C16D38
:10884000EA81FB8132960E94C16DEC81FD813496F4
:108850000E94C16DEE81FF8136960E94C16DE88550
:10886000F9853896E491EA93E985FA8539960E946C
:10887000D66C02D022960895A0970E94A27DEDA505
:10888000FEA5A9A9BAA9EA0FFB1FAF01E5E0F3E035
:10889000EE83FF8310E01431C0F5AE81BF81AC914F
:1088A000A03049F1EE81FF81A381B481EFA5F8A941
:1088B000EA17FB0701F5EE81FF81A181B281E9A9E9
:1088C000FAA9AE17BF07BCF0EE81FF81A181B2818A
:1088D0004A175B0784F00E94EB75AE0FBF1FE9A932
:1088E000FAA9AE17BF073CF00E94EB75AE0FBF1F91
:1088F0004A175B070CF402C01A933DDFEE81FF813B
:108900003D96EE83FF831F5FC6CFE5E0F3E0EE8385
:10891000FF8310E0143110F00C943145AE81BF811B
:10892000EC91E03011F00C942A45EAA5EC93E9A90A
:10893000FAA9AE81BF811196ED93FC93EFA5F8A93A
:10894000AE81BF811396ED93FC93EDA5FEA5AE819C
:10895000BF811596ED93FC93EBA5AE81BF81179671
:10896000EC93E0910904A0910F04EA27AE81BF8146
:108970001896EC93E0911004AE81BF811996EC93A8
:10898000E0911104AE81BF811A96EC93AE81BF8154
:108990001B960E94726D1C96E0E0EC93E887E8A5B8
:1089A000F9A5309741F00E94F6750E94FB75E4E14D
:1089B000EA930E944969EEA1FFA1309751F00E940D
:1089C000F675E8A5F9A5FA93EA93E4E1EA930E9423
:1089D0003569E0E0EC8F0E94F6750E9420693E2F19
:1089E0003B30C8F000E00E94E575E081E03011F016
:1089F000053008F002C00F5FF6CF0E94E575E081F8
:108A0000E03049F40E94E5750E940076E058AE819E
:108A1000BF811B96EC93E0E0EA8B3130C8F000E0B8
:108A20000E94D975E081E03011F0043108F002C0F5
:108A30000F5FF6CF0E94D975E081E03049F40E94C3
:108A4000D9750E940076E05CAE81BF811B96EC93E5
:108A5000E12F08C0EE81FF813D96EE83FF831F5F0B
:108A600059CFEFEF0E94A97DE39608951A930A93D8
:108A70000E940B763097A9F1E0916205E03061F534
:108A80000E940B76049000926205E0916205E0304E
:108A900031F4E0E0F0E00E945975E0E01AC00E9475
:108AA00010760E940B760E94CF7BF595E7958F019B
:108AB000D801E0E0F1E00E94477BE0938700D80115
:108AC000E0E0F1E00E94797BE09386000E9410765E
:108AD000E0E4E0938B0005C0E0916205E150E09393
:108AE00062050991199108950E94A47D00E025E096
:108AF00033E010E01431B8F5D901EC91E03079F1B0
:108B000011960E94C07B0E94187624F5D901139615
:108B10000E94C07BAC81BD81EA17FB07DCF4F90140
:108B200001801280D90115960E94C07BE00DF11DD5
:108B3000AE81BF81AE17BF076CF4F90103801480CA
:108B4000D9011796EC910E942D72AC81BD81AE17B0
:108B5000BF070CF004C0E12FEF5F0E2F04C0235FAE
:108B60003F4F1F5FC7CF003049F0E0916305E0172A
:108B700021F0A0916305A03009F401C022C0A091AA
:108B80006405A53079F40A93E1E0EA93A4DD00934B
:108B9000630500936505D901EC91E0936605E3E078
:108BA000E0936105A0916405AE3119F4E4E0E0932F
:108BB0006105A0916105A33018F0E5E0E093680538
:108BC00007C0E0E0E0936405E09361050E941D7634
:108BD0000E94AB7D28960895E0916305E03091F006
:108BE000A0916405A93220F4EA93E2E0EA9373DDF0
:108BF000A0916405AD3330F0E0916305EA93E4E0C1
:108C0000EA9369DDE0E0E0936105E09364050E948A
:108C10001D76E0E0E0936305E0936705089530D1A9
:108C20005ADB0895EA81E0937F05E881E0938005AF
:108C3000E0910A04E061E0930A0420C10E94A27D51
:108C4000A0917F05A43120F4A0918005A33008F005
:108C500033C0E0917F05F0E0ACE0B0E00E941C7B07
:108C60008F01E0918005F0E0A4E1B0E00E941C7B60
:108C70009F010E942376ECE0F0E00E942876F0E06D
:108C80000E94CF7A0E947C6CEE81E030A9F0E091E6
:108C90007F05A3E0EA9FF001EC57FA4FDF01E09176
:108CA00080050E94FE6F4C9155270E9423764A93BF
:108CB000EFE0EA930E94D74D0E94A97D2796089580
:108CC000E0910A04E07141F0E2E0EA93B7DFE0915D
:108CD0000A04EF7EE0930A0408950E942D76AF3EC9
:108CE000E0E0BE0744F4A0910203B0910303AF3368
:108CF000E1E0BE070CF039C00E9432760E9410708D
:108D00000E94D74DA0915D05B0915E05549734F453
:108D1000A0915F05B091600513970CF012C0E0912F
:108D20005D05F0915E05A3E0B0E00E94F47AEC5797
:108D3000FA4FA0915F05B0916005EA0FFB1FA98172
:108D4000A083E0910D04ACE0EA9FF0010E942D7633
:108D50000E94DB740E943F76E0915D05F0915E0514
:108D60003196E0935D05F0935E050C941C4BE88111
:108D7000EA93E0911004EA93B0DF0C94EB4A1A9363
:108D800010E00E944476E03031F00E944476EA938D
:108D9000EEDF1F5FF6CF1881239608950E94477675
:108DA0000E944C76E03021F00832E0E01E070CF023
:108DB00007C00E944C76EA93DADF0F5F1F4FF0CFB7
:108DC000198108815BC00E944776F801AB81BC81A4
:108DD0000E94537621F0EA810E9458760CF009C077
:108DE000F801AB81BC810E945D76C1DF0F5F1F4F30
:108DF000ECCF198108810EC30E94A47D0E942D76BC
:108E00000E94627631978F010E9467760E942376D6
:108E10000E946F7633C00E94A47DAC810E9476765A
:108E20000E2F11270E9467760E9423760E946F768C
:108E3000F1C2EA81FB81E0935D05F0935E05E88174
:108E4000F981E0935F05F0936005AA81BB81ECE0B6
:108E5000F0E00E941C7B0E943F76A881B981E4E18A
:108E6000F0E00E941C7B06C0EA81FB810E943F76F5
:108E7000E881F981E0930203F093030324960895B7
:108E80000E947E76143120F41A9375DC1F5FFACFAE
:108E90000E94566C0E94566C0E94776CEFE3F1E0E2
:108EA0000E947C6C10E0153048F4A5E11A9FF00197
:108EB000E051FB4FA0E0A0831F5FF5CF10E014311D
:108EC00048F4ABE01A9FF001EC5EFB4FA0E0A083FA
:108ED0001F5FF5CFE0910A04EF7EE0930A04199139
:108EE00008950E947E76143100F5ADE01A9FF001DE
:108EF000BF01E85FFC4FDF010E94C07B0F01DF0173
:108F0000EB81FC81AE17BF075CF0E981FA81E015C7
:108F1000F10534F0FB01E05FFC4FE081E03009F443
:108F200002C01A9328DC1F5FDECF0E94566C0E949D
:108F300086760E94776CA985BA850E948B760E94FE
:108F40007C6C67C2A2970E94A27DE9A50E948B72E9
:108F50008F01D8011B96EC91E03009F415C2D801BD
:108F60001B96EC91E9A3E07859F0FE013696FA934E
:108F7000EA93EBA10E94C375FA93EA930E940A69EF
:108F8000E9A1E07459F0FE013696FA93EA93EBA159
:108F90000E94CA75FA93EA930E940A69FE01369606
:108FA000FA93EA930E942069E8A3E0910D04EB8F05
:108FB000E0910E04EA8F0E94DC6ED80111962D918B
:108FC0003C91D80113964D915C91D80115960E9461
:108FD000C07BEEA3FFA3D8011796EC91F0E0ECA3C1
:108FE000FDA3D8011896EC91EC8FE0910E04A0E15E
:108FF0000E94366CEAA3FBA30E9490760E94FB7548
:109000000E94FB75ECA1EA930E942F4CD80119969F
:10901000EC91EC8FE03011F4E8E0EC8F0E94907658
:109020000E9495765A934A930E949C760E94A0765D
:109030000E94A7760E94AA760E9490763A932A937D
:109040000E94AA76EEA1FFA10E94B1765A934A939C
:109050000E9495760E94AA76A8A5A130B1F43A9311
:109060002A93FA0131960E94A776FA013196FA9373
:10907000EA930E949C76F90131960E94B676F90136
:109080003196FA93EA930E94AA76A8A5A230F1F449
:109090000E94A07631970E94A776EAA5FBA5E40F6F
:1090A000F51F3197FA93EA930E949C76EEA1FFA1F7
:1090B000E20FF31F31970E94B676EAA5FBA5E20FF7
:1090C000F31F3197FA93EA930E94AA76E8A5E0305D
:1090D00011F40C949449D8011996EC91EC8FE0911D
:1090E0000D04ACE00E94BB760E94477BED8FA8A1E7
:1090F000EA1710F40C94C348E1E0E0930E04E0306A
:1091000021F0ECA1FDA1B5970CF402C00E94C1763C
:10911000AAA1BBA1ECA1FDA1EA1BFB0BDF010E94F0
:109120007971EAA3FBA3ABA1AA231AF4E0E0EAA3B6
:10913000EBA3A8A10E947676AEA1BFA1F0E00E94A9
:10914000C976EE8FA8A5A13021F40E94CC760E94AA
:10915000CF76A8A5A23031F40E94CC760E94B176D9
:109160000E94DB76E0E0E9A30E94E176AE0FBF1F2C
:10917000EC91E03039F00E94E1760E945D760E9429
:10918000E676F2CFD1C0E1E0E0930E04E03031F0BA
:10919000ECA1FDA1E734A0E0FA070CF402C00E94A4
:1091A000C176E8A1EF8FEAA1FBA1EE0FFF1FACA1F2
:1091B000BDA1AE1BBF0BE3E0F0E00E94477BEAA33A
:1091C000FBA3ABA1AA2322F4E1E0F0E0EAA3FBA316
:1091D000EF8DE150EF8FEF8DF0E0DE011696AE0FD0
:1091E000BF1FAC91A03219F0AF8DA13008F404C0BC
:1091F000EF8DE150EF8FEFCFAF8D0E947676AE2FDF
:10920000EEA1FFA1B0E0EA17FB0714F3EF8DE03009
:1092100011F4ED8DEF8FAF8DECE00E94BB760E94D4
:10922000C976EE8FA8A5A13021F40E94CC760E94C9
:10923000CF76A8A5A23031F40E94CC760E94B176F8
:109240000E94DB76E0E0E9A30E94E1760E9453767B
:1092500021F0EF8DA9A1AE1708F007C00E94E176BA
:109260000E945D760E94E676EFCFAF8DE8A1EA1B03
:10927000AE2FED8DEA1768F0AF8DE8A1EA1BACE0E8
:10928000EA9FF001A0910D040E94BB760E94C9766E
:1092900001C0E0E0EE8FA8A5A130A1F40E94CC7639
:1092A000E20FF31F31960E942876AFE00E94366CE1
:1092B000E40FF51FDF01ECA1FDA10E949071319632
:1092C0000E948F6EA8A5A23089F40E94CC76E20F8E
:1092D000F31F0E942876AFE00E94366CE40FF51F62
:1092E000DF01ECA1FDA10E940475BEDD0E94E176C4
:1092F000AE0FBF1FAC91A03219F4E9A1EF5FE9A353
:109300000E94E1760E94537639F0AF8DE9A1EA1B05
:10931000AE2FED8DEA1708F407C00E94E1760E9497
:109320005D760E94E676ECCFD8011C96EC91E03099
:1093300029F10E94DC6E0E94907696DDF801A485EA
:10934000A43698F4EFE0E0931004F801A485AA3065
:1093500028F0A485AA930E94E84106C0D8011C9673
:10936000EC91E05DEA9303DD09C0ECE0E0931004CA
:10937000E2E5EA93FCDCEDE4EA93F9DCEB8DE093C3
:109380000D04EA8DE0930E040E94A97DAA9608952B
:109390001A9310E0E89427F8143170F40E94B96E23
:1093A000E03011F00E94C06E1F5FA895E12FE370BE
:1093B00011F40E94AE15F0CFEFE0E09310040E948C
:1093C000AE150C94744E1A9310E01431F8F40E9408
:1093D000C56EB1F0A85FBC4F0E94C07BDF01EB817E
:1093E000FC81EA17FB0764F4F001E85FFC4FDF0142
:1093F0000E94C07BDF01E981FA81AE17BF070CF044
:1094000002C00E94C06E1F5FA895DFCFEFE0E0931F
:1094100010041881259608951A9310E0143190F4E1
:109420000E94C56E31F0FD01E15FFC4FE081E1700B
:1094300009F406C01A93E0910A04E170EA9382DD10
:109440001F5FECCF0C94744E2C970E94A27DAD89C7
:10945000BE890E9479710E94EE76EB8BFC8BED89C0
:10946000FE890E94F376EB89FC89E017F107FCF096
:109470000E9426772E2F33270E944A770E94517729
:109480000E9458770E945D770E944A77F801A98D63
:10949000BA8D0E94656D0E945877F8010E94677727
:1094A000EA8DEA930E94924C0F5F1F4FDCCF48C0B9
:1094B0002C970E94A27DAD89BE89E4E0F0E00E9475
:1094C000477B0E94EE76EB8BFC8BED89FE89EE0FDD
:1094D000FF1F0E94F376EB89FC89E017F10784F106
:1094E0000E942677AE2FED89FE89B0E0EA0FFB1FC0
:1094F0009F010E944A770E945177E98DFA8DEE0F05
:10950000FF1F0E9467770E945D77ED89FE89EE0F4D
:10951000FF1FA98DBA8DAE1BBF0BBA93AA93F8019A
:10952000A98DBA8D0E94656D0E945877F8010E943E
:109530006777EA8DEA930E94924C0F5F1F4FCBCF63
:109540000E94A97D6B960895EA81F0E0EBBBF5BB24
:10955000F7E1F09365001F98E6E1E0936500F09372
:1095600065001F9AE881F981EBBBF5BB1F98FFE10D
:10957000F0936500EEE1E0936500F09365001F9ABB
:109580000C94E74EE2E2EBBBE0E0E5BBE7E1E09301
:1095900065001F98E6E1E0936500E7E1E093650070
:1095A00008951F9A0895A0910403A23021F4E88140
:1095B000A8E4B3E10BC0A0910403A43021F4E88136
:1095C000A8E4B3E103C0E881A8E2B3E1F0E00E94BF
:1095D00090710E94CF7B21960895E0910403E230C0
:1095E00011F4EEE40AC0E43039F4E0E2EA93A98130
:1095F000BA810E94627604C0E0E2EA93E981FA81CE
:10960000FA93EA930E94A44A17C0E0910403E2305F
:1096100011F4EFE40AC0E43039F4E1E2EA93A981FD
:10962000BA810E946B7704C0E1E2EA93E981FA8192
:10963000FA93EA930E94A44A22960895E0910403C3
:10964000E230B9F4E4E4EA930E947077AE0FBF1FF2
:10965000FD01FE2FE0E0AF81B8850E94656D0E949C
:10966000A44AE5E4EA930E9486760E94A44AE6E4CE
:1096700053C0E33089F4E7E3EA93FF81E0E00F01B0
:109680000E947077EA0FFB1F0E9475770E94867612
:109690000E94A44AE6E340C0E43049F5E7E3EA93D8
:1096A000AF81B8850E946276DF01EB81FC81AE1B41
:1096B000BF0BFD01FE2FE0E00F01AF81B8850E94D6
:1096C00062760E947577AD81BE810E946B77DF0163
:1096D000E981FA81AE1BBF0BBA93AA930E94A44AF8
:1096E000E6E3EA93AD81BE810E946B771CC0E0E5A2
:1096F000EA930E94D6740E94A44AE1E5EA930E948C
:1097000070770E94656D0E94A44AE2E5EA930E9488
:1097100086760E94A44AE3E5EA93E981FA81AD8165
:10972000BE81EA0FFB1FFA93EA930E94A44A28968F
:109730000895E0910403E33029F4E3E0EA93E0E1E3
:10974000F1E00BC0E43029F4E3E0EA93E0E2F1E079
:1097500004C0E3E0EA93E0E3F0E1FA93EA930E94C5
:10976000A44A0895E0910403E33029F4E3E0EA9386
:10977000E1E2F1E00BC0E43029F4E3E0EA93E1E157
:10978000F1E004C0E3E0EA93E8E3F0E1FA93EA935E
:109790000E94A44A08951A930A93EFE10E947E77EB
:1097A000EBE10E947E77EFE10E947E77E8EFFFEF2A
:1097B000E0935C0CF0935D0CE491EF3F39F0E091A5
:1097C0005C0CF0915D0C049000920403E6ECF3E174
:1097D0008F01A0910403A23019F4E8EAF3E18F01AC
:1097E000A0910403A43019F4E8E6F3E18F01F80135
:1097F000E491ED3F39F4F80131960E94C16D0E9469
:10980000A17A19C0EE3F71F4F80131960E94CF7B26
:10981000DF01E0910403F0E0EA17FB0711F00D5FB0
:109820001F4F09C0F801E491EA93F80131960E94B4
:10983000C16D0E94A44A0D5F1F4FF801E491EF3FF4
:10984000B1F60E944F6CE1E0E0930E04E0930D044A
:10985000E4E1E09313046DDF0991199108950E94EA
:109860008277AE85AA2362F0AD85BE85A03FE0E099
:10987000BE0734F4AB85BC85AF33E1E0BE070CF026
:1098800050C00E948A77AE0FBF1FA03FE0E0BE0726
:1098900034F0AD85BE850E946276E987FA87EF8154
:1098A000F885AB85BC85AE0FBF1FA034E1E0BE07D5
:1098B00034F0AB85BC850E946B77EF83F8870E94FC
:1098C000CC6D0E94CC6D0E94CC6D0E94CC6DB6DE3A
:1098D0000E94CC6D0E948F77498554DE0BBB15BB6F
:1098E0002EE13FE100E010E0EF81F885E017F1079D
:1098F00064F050E0451730F0209365003093650028
:109900005F5FF8CF0F5F1F4FEFCF4BDE0E94566CAB
:109910000E94566C0E94776CEFE3F1E0FA93EA93B1
:109920008DDEC9C00E9482770E948A77EA17FB0702
:1099300041F0EF81F885AB85BC85EA17FB0709F09C
:109940003EC00E9497771CF00E949E7784F42D857C
:109950003E85ED85FE85E987FA872D873E872B8535
:109960003C85EB85FC85EF83F8872B873C870E943D
:10997000CC6D0E948F770E948A77EA17FB0749F423
:10998000F1DEEB85FC85ED87FE87EF81F885E987C1
:10999000FA87F8DD0BBB15BB2EE13FE10D851E8577
:1099A000E985FA85E017F1073CF0209365003093D4
:1099B00065000F5F1F4FF4CFF4DDBBDE7CC000936A
:1099C0000B0410930C040E94A5770E94AC77FF93C0
:1099D000EF930E94B0770E94AC77AF91BF91EA17E6
:1099E000FB0780F10E949E77B4F420E030E00E94F3
:1099F000B377E217F30774F00E94A5770E94BA7755
:109A00000E94B3770E94BF770E94C87758D02F5F1B
:109A10003F4FEDCF16C020E030E00E94B077E21754
:109A2000F3077CF00E94A5770E94BA770E94B07776
:109A30000E94BF77F9010E94CF7741D02F5F3F4F3F
:109A4000ECCF39C00E949777DCF420E030E00E9430
:109A5000D377E217F3079CF00E94B0770E94BA77A1
:109A60000E94D377D0010E94477BAF010E94C87744
:109A7000FA010E94CF7723D02F5F3F4FE8CF1BC062
:109A800020E030E00E94A577E217F307A4F00E94DF
:109A9000B0770E94BA770E94A577D0010E94477BD9
:109AA000AF01F9010E94CF77FA010E94CF7707D06A
:109AB0002F5F3F4FE7CF0E94A97D2F960895EA813F
:109AC000FB81FA93EA9389DD0E94DA779EDDE2E278
:109AD000EA93E0910B04F0910C04FA93EA930E944C
:109AE000A44A249608950E94A27D00910D0410E0DE
:109AF000E0910E041E1710F00C94D64DE885F98500
:109B0000FA93EA9382DD2C853D854A855B85022E9A
:109B1000032A11F40C94CE4D37FF36C05A934A9362
:109B20005CDDE2E2EBBBE0E0E5BBE7E1E093650092
:109B30001F98F6E1F0936500E0936500EE81EBBBC2
:109B4000EF81E5BBEFE1FEE1E0936500F093650096
:109B5000E093650001FF04C0F0936500E0936500A9
:109B600036FF11C0F0936500E093650001FF06C069
:109B7000F0936500E09365004F5F5F4F220F331F46
:109B80004F5F5F4FEDCF1F9A220F331F01FF02C0BF
:109B90004F5F5F4F4F5F5F4F0C94874DE885F985AE
:109BA0003196E887F9871F5F0C94784D38C022976B
:109BB0000E94A27DE885EA930E94D34AEE83FF8348
:109BC000E985A8E1EA9FF001E85DF84F8F0130E0F8
:109BD000383028F5F801E4915E2F0F5F1F4FF80130
:109BE000E4914E2F407F0E94DF770E94E477EA875E
:109BF000FB87F801E4914E2F440F440F440F440FAC
:109C00000F5F1F4FF801E4915E2F0F5F1F4F0E94FF
:109C1000DF770E94E477EA87FB873F5FD9CF0E9416
:109C2000A97D2E96089524970E94A27DEA85EA9345
:109C30000E94D34AEE83FF8300E010E0EB850E9490
:109C40005876D4F5EF85F889E887F98720E030E089
:109C5000EC850E94F1772CF5E989FA894491552722
:109C60003196E98BFA8B5A934A93EA85FB85FA93EE
:109C7000EA93E989FA89FA93EA93EC85FD85FA93E8
:109C8000EA930E94734DE0910D04EE0FEE0FEE0F7C
:109C9000A885B9850E94DB74E887F9872F5F3F4F5D
:109CA000D7CFE0910E04AD85BE850E94DB74ED87B1
:109CB000FE870F5F1F4FC2CF0E94A97D6396089554
:109CC0001A93EFEF0E945472E093390910E00E945A
:109CD0007671E05CF54FE081EF3F31F00E947671E4
:109CE0000E94F6771F5FF3CF199108951A930A9394
:109CF0000091CF0BAA81A53411F4E0E066C0AA81DF
:109D0000A23539F4A0913508A13019F40E94F977F1
:109D100009F405C00E94E41CE0E0E0933508AA8144
:109D2000AB3411F0A33599F4E02FE470E43011F472
:109D300014E001C013E0E02FE270E23009F41C5F90
:109D4000E02FE170E13009F41F5FE12F3EC0AA81EE
:109D5000A13511F0A13799F4E02FE470E43011F44B
:109D600017E001C016E0E02FE270E23009F41C5F5A
:109D7000E02FE170E13009F41F5FE12F26C0AA81D6
:109D8000A33421F0A13411F0A23441F413E0E02F08
:109D9000E170E13009F41F5FE12F17C0AA81A737F6
:109DA00041F417E0E02FE170E13009F41F5FE12F8B
:109DB0000CC0AA81A03441F415E0E02FE170E1303D
:109DC00009F41F5FE12F01C0EFEF1981088123968D
:109DD000089524970E94A27D2091CF0BA091400965
:109DE000A53411F00C94B34FE0E0E09335080E94E5
:109DF0004D72E0E0E0935D0BE091D30BE03089F52C
:109E0000E0911008A0911108EA1739F00E94FF773D
:109E1000ED55F84FE081E13009F023C0E7E7EA9320
:109E20000E941A630E94FF77E855F84F0E949571CF
:109E3000FA93EA930E940578EC55F84FDF010E94EF
:109E400001740E940578E755F84F0E940A78E2E015
:109E5000E09335080E94FF77ED55F84FA2E0A0830C
:109E60002FDFE0913508E03011F00C94B34F0E94E1
:109E7000F97711F40C948D4F0E94D91CE1E0E09326
:109E80003508E22FE870E83081F40E940F78E8EEA0
:109E9000F3E00E94477BDF010E94987D14F4E1E328
:109EA00001C0E0E3EA930E941A63E22FE074E03419
:109EB00011F413E001C012E0E091240C0E949374AD
:109EC0001A930E947763E22FE470E43049F40E9411
:109ED0000F78E0E1F7E20E94797BAF0114E006C061
:109EE0000E940F780E948673AF0113E0E22FE071A9
:109EF000E03111F4415050405A934A931A930E9412
:109F00007763E22FE072E03211F414E001C013E055
:109F1000E091270CF091280C17C018E0E22FE470B4
:109F2000E43009F41F5FE22FE870E83009F41F5FA6
:109F3000E22FE072E03209F41F5FE22FE074E034B8
:109F400009F41F5FE0E0F0E0FA93EA931A930E94AD
:109F50007763E22FE170E13029F4E0915D0BEA9341
:109F60000E941A63ADDEA0914009A73729F4E2E010
:109F7000E0933508E03009F473C00E944D720E94EE
:109F800014780E9403731E2F0E941E73AF01E1E03C
:109F9000EA930E94C0620E2FE0911008A091110870
:109FA000EA1739F00E94FF77ED55F84FE081E23073
:109FB00009F053C00E94FF77EC55F84FDF010E9473
:109FC000C07B4E175F0711F00C9429500E94FF7759
:109FD000E655F84F008011800E94236E0E94DD71CB
:109FE000EA17FB0769F10E94FF77E655F84FDF019A
:109FF0000E94C07B0E941A780E94FF77E655F84FB6
:10A00000DF010E94C07BEC59F44FE0810E9422786E
:10A010000E9429780E94A66D0E942C78E1EBF9E15C
:10A020000E94FF72003029F05A934A930E944D63B8
:10A0300002C00E9432780E9436780E94F36309C001
:10A04000003039F00E943A7820F40E94F6730E94A2
:10A05000D826E1E1F8E00E944178E0E0E09335089D
:10A06000A0914009A33421F40E942034E03009F487
:10A070000BC00E944D720E9414780E9493730E943C
:10A08000566C63D30E948C1DA0914009A13411F03D
:10A09000A23421F40E944D720E941478A0914009CC
:10A0A000A03421F40E942034E03009F420C00E9442
:10A0B0000373E887F987E2E0EA930E94C0621E2FEB
:10A0C0000E9445780E94AE180E9436740E944B7818
:10A0D000E152F84F10830E943674E652F84FA7E021
:10A0E000A0830E9421720E944D720E941478A09158
:10A0F0004009AB3439F0A33529F0A13519F0A13767
:10A1000009F076C00E942034E03011F40C94F25033
:10A110000E944D720E945278E1E4F9E00E941973A6
:10A12000E22FE270E23029F4E4E0EA930E94C06298
:10A1300002C0E1E0F0E0E887F987A0914009A1358D
:10A1400011F0A13721F40E941E731E2F02C010913E
:10A15000E50BE22FE470E43011F4E4E001C0E3E049
:10A16000EA930E94C062AF01A0914009A33511F0AB
:10A17000A13731F4E885F9850E94BB7AE887F98731
:10A180000E943A7820F0A091D30BA13011F51A93D8
:10A190005A934A93EB85FC85FA93EA930E94AB1D90
:10A1A0000E94AC77EE83FF83AE81BF810E94987DD1
:10A1B00084F40E944D72E6E6EA930E941A63EE81EF
:10A1C000FF813197EE83FF83AE81BF810E94987D2E
:10A1D00094F31A935A934A93EB85FC850E94D672A6
:10A1E0006FDD06C00E9493730E94566C0E94AB1DE7
:10A1F0000E94A97D2A9608950E945678E89422F834
:10A200000E941574E2E7EA930E941A63E0913B080A
:10A21000EA930E941A63EFE0EA930E941A63A09106
:10A220003808AA3219F41A9365D31AC0A0913B08D2
:10A230000E947671EC59F44FE081EA1721F4E09125
:10A240003B08E03349F40E94F46CAC59B44FE09100
:10A250003B08EC931A934ED322FC02C00E94F36396
:10A26000C0C20E945678E0913B08E053AE2F0E9496
:10A270007671EB58F44FE081EA1741F51A933AD31F
:10A28000A0913608A23019F40E945E7809F402C049
:10A290000E946478A0913608A33019F40E945E7879
:10A2A00009F402C00E946478E0E0E0933608E0938D
:10A2B000600C0E947671EB58F44FBF01E081EF5FB4
:10A2C000AE2FEAE00E94767BDB01EC938AC2E88144
:10A2D000E03019F40E94327806C0E881E8500E940C
:10A2E00093740E944D63219608950E94A27D25FCDF
:10A2F00028C20E945E7811F40C94F5520E9467788F
:10A30000E752F84F9F01D9011196EC91E43071F5B5
:10A310000E946D780E9470780E947778F901A6817A
:10A32000A03021F4A281B381109709F007C0E4EBBB
:10A33000F9E10E94FF720E94367815C00E942978C8
:10A340000E947B780E942C78E7EBF9E10E94FF7273
:10A350000E947F780E948578F901A085B185BA9323
:10A36000AA930E944D630E948B78EBC1E730C9F439
:10A370000E946D780E9470780E947778EAEBF9E18C
:10A380000E94FF720E947F780E942C78EDEBF9E129
:10A390000E94FF720E947B780E944D630E948B781E
:10A3A000D0C1E93089F40E946D780E9470780E94D3
:10A3B0007778E0ECF9E10E94FF720E9492780E94A7
:10A3C0002C780E948B78BDC1E63029F5EAE2EA9349
:10A3D0000E94D863E3ECF9E10E94FF72D901EC918D
:10A3E0000E949578E091CD0B0E949578EBE4EA937A
:10A3F0000E941A630E947B780E944D63E4E5EA9311
:10A400000E941A630E947F780E944D630E94F3634A
:10A410000E94647896C1E530C9F40E94E7730E94F7
:10A420001A78D901EC910E9422780E9429780E9422
:10A430007B780E942C78E1EBF9E10E94FF720E9488
:10A440007F780E944D630E948B787BC1E83039F59C
:10A450000E946D780E9470780E947778E6ECF9E1AE
:10A460000E94FF72F901A681AA930E94F3733097AC
:10A4700019F00E94077004C0D9011696EC91F0E023
:10A48000FA93EA930E944D630E9436780E94F36328
:10A49000D9011196E0E0EC930E94647852C1E1305A
:10A4A000C9F5A0911908A53029F4E091CD0BE65F1C
:10A4B0001E2F01C011E0E12F0E9499780E94767151
:10A4C0000E949E780E94A1780E9429780E947B7841
:10A4D0000E942C78E9ECF9E10E94FF720E947F78DB
:10A4E0000E948578D9011796EC910E9493740E947E
:10A4F0004D63A0911908A53041F40E94A578A4816C
:10A50000B581BA93AA930E94AF630E9498750E9486
:10A51000AB7817C1E330B1F40E94E773F0960E9464
:10A52000B6780E94E7730E949E780E94A178ECECB6
:10A53000F9E10E94FF720E947F780E94BA780E941F
:10A54000AB78FFC0EB3069F50E94BD780E94C078FF
:10A550000E94A178EFECF9E10E94FF72F901A68157
:10A56000AA93B5DE0E94A578A781AA93B0DE0E94C7
:10A57000A578A085B185BA93AA930E9485780E9498
:10A580007F780E948578F901A481B581BA93AA9356
:10A590000E9485780E9492780E94BA780E94AB78D7
:10A5A000D0C0EC3089F40E94BD780E94C0780E942F
:10A5B000A178E2EDF9E10E94FF720E9492780E9478
:10A5C000BA780E94AB78BDC0EE3079F40E94BD78B5
:10A5D0000E94C0780E94A178E5EDF9E10E94FF7227
:10A5E0000E9498750E94AB78ACC00E94F97761F028
:10A5F000A0913608A03041F4A091D20BA13021F4F3
:10A600000E94236EE13009F426C0A091850BA03092
:10A6100059F0E091870BF091880BFA93EA93E8EEFA
:10A62000F3E00E949D73B9F4E1E30E94B678E091F3
:10A63000760BE05D0E9422780E94236EEA930ED191
:10A64000E09336080E949875E0935E0CF0935F0CDF
:10A65000E0E0E093850BA0913608A03059F0E0913E
:10A660005E0CF0915F0CFA93EA93E4E6F0E00E944E
:10A670009D7309F025C0A0913608A23019F40E94FC
:10A680005E7809F402C00E946478A0913608A33075
:10A6900019F40E945E7809F410C0A091600CA330F8
:10A6A00030F00E946478E0E0E093600C06C00E9405
:10A6B0006778E652F84FA8E0A083E0E0E093360820
:10A6C000A091860BA130E9F5E091390CA091380CEE
:10A6D000EA1791F1EAE20E94B678E091740BE05D2E
:10A6E0000E942278E091390CEA930E943E1F0E945A
:10A6F0002978E091290C0E9493740E942C78E8ED4F
:10A70000F9E10E94FF720E94FF70FA93EA930E949F
:10A7100085780E947E740E94C4780E94F363E09161
:10A72000390CEA930E94831DE091390CEA930E9450
:10A73000521DE093390C05C0E0E0E093860B68946D
:10A7400020F80E94A97D269608951A930A930E94E4
:10A750002034E030D9F00E943674E752F84F8F0170
:10A76000EC81FD81D8011296ED93FC93EA81FB8187
:10A77000D8011896ED93FC93EE81D8011696EC93D0
:10A78000D8011196E4E0EC930E94217219810881AE
:10A7900027960895E091420BEA930E941A63E09194
:10A7A000430BEA930E941A630895F4DF0E94DA775C
:10A7B0000E94C7780E94C7780E942C7899C01A938B
:10A7C0000E944C621E2F103021F0E12FE150E093E7
:10A7D000400BE0DFE091400BEF5F0E9493740E941A
:10A7E0002C78199108950E94A47D31E00E94CE78C2
:10A7F00028F00E940D73AC91A43308F02AC030E019
:10A800000E940D73EC91E270E6951E2F0E940D736D
:10A81000EC91E1700E2FA0915A0B1A1729F4E1E088
:10A82000EA27E0935A0B31E0A0915B0B0A1729F05D
:10A83000E1E0EA27E0935B0B31E0E0915B0BEE0F88
:10A84000E05DA0915A0BEA0FEA930E941A630E94FE
:10A850000674E32F0E94AB7D249608951A9310E0AE
:10A860000E94F97711F40C9474540E94D91CECEDF9
:10A87000F9E10E94FF72E091240C0E9493740E94FF
:10A880002C78EFEDF9E10E94FF72E091270CF09136
:10A89000280C0E94C4780E940F78A031E7E2BE071E
:10A8A0004CF4E2EEF9E10E94FF72E091250CF09188
:10A8B000260C13C0E5EEF9E10E94FF72E9810E94C7
:10A8C0001C700E940F78EA0FFB1F0E94BD70E09180
:10A8D000250CF091260CE051F742FA93EA930E947E
:10A8E0004D630E94367811E00E94D278E12F1881E2
:10A8F0002296089524970E94A27D0E94D2780E94F9
:10A90000F561E13010F40C944E57E091420BEB34BA
:10A9100041F4E091430BE33219F40E944C621E2F84
:10A92000BAC2E435A9F4E091430BE33221F40E946A
:10A930004C62EE83FF83E091430BEF3441F40E94BD
:10A940004C621E2F1A930E94D6740E94AE18A3C2A6
:10A95000E23411F00C94ED55E091430BE13251F4E7
:10A96000AA85AF3F29F40E9493730E94566CEDDED6
:10A970000E948C1DE091430BE134E1F40E944C6293
:10A980001E2F113071F4A0913608A13019F40E94E5
:10A99000F97709F402C00E94E41CE0E0E093850B23
:10A9A00009C0E1E0E093850B0E948C68E093870B7F
:10A9B000F093880BE091430BE534A9F4E8EEF9E15C
:10A9C0000E94FF720E94C11CF3973CF00E944C62EF
:10A9D0000E94BD700E94D97801C0E0E3EA930E9412
:10A9E0001A630E943678E091430BE634D9F40E9452
:10A9F000E57819F40E944C62AF01E885F9850E9460
:10AA00000C700E2F033620F0A091D30BA13021F44F
:10AA10000E94F1780E94AB1DAA85AF3F19F40E94F5
:10AA2000F17893DEE091430BE23511F00C94AA55D6
:10AA30000E94E57819F40E944C62AF0130E0A091C9
:10AA4000D30BA03021F40E94236EE13009F027C01F
:10AA50000E942634E03011F10E94CA72EC55F84F82
:10AA6000A885B985A083B1830E94CA72E655F84FC4
:10AA7000DF01EA850E941D720E94CA72E855F84FF4
:10AA800010830E94CA72E755F84F40830E94CA7231
:10AA9000ED55F84FA1E0A0830E94D07259C00E94EA
:10AAA0002034E23010F40C94A8550E9445780E949E
:10AAB000B81E3E2F3F3F29F00E94D270A417B50761
:10AAC0000CF412C00E947E74E41BF50B0E94E0702F
:10AAD0000E94A77219F4E0E0E093290C3A930E94D7
:10AAE000451F689420F803C0E0E0E887E9870E94EA
:10AAF0003674E752F84FDF01EA85F0E0EC59F44F85
:10AB0000E081EC930E9436740E944B78EF51F84F2D
:10AB1000DF01EA850E941D720E943674E152F84FEF
:10AB200010830E943674E652F84FA5E0A0830E947D
:10AB30002172E885F985309759F00E944578FA012D
:10AB40000E94BB7A0E94D6720E94F1780E94331D47
:10AB5000689422F8E091430BE335F1F50E944C62D2
:10AB6000E887F9870E946778DF01E652F84FE081B5
:10AB7000E23081F4FD01EF51F84F008011800E9416
:10AB8000236E0E94DD71EA17FB0721F4A0913608BD
:10AB9000A23009F01FC00E946778E552F84FDF012C
:10ABA0000E94C07BDF01E885F985EA17FB0779F48D
:10ABB0000E946778DF01ED51F84FE081EA93FD01D3
:10ABC000E752F84FE081EA930E94D82603C0E7E0FD
:10ABD000E0932406689422F85EC1E43411F00C94EA
:10ABE0005656E091430BE33559F4EBEEF9E10E9440
:10ABF000FF720E94EA5E0E949578E1E0E0933909D5
:10AC0000E091430BE03511F00C9455560E94F57815
:10AC1000E03011F40C94555620E00E94F97840F091
:10AC20000E940D73AC91A23219F00E94FD7809F4D4
:10AC30003CC0E22FE03061F40E940D73AC91A3326E
:10AC400011F421E004C00E9401790E94C55E2AC06F
:10AC5000E13051F40E940D73AC91A43211F422E062
:10AC600001C020E010E01EC0E23011F0E330D1F46A
:10AC70000E9401790E946468EF3F99F0E12FE2950C
:10AC8000E07FEF930E9401790E946468AF91EA0F20
:10AC90001E2F2F5F243021F41A930E94C55E20E0FE
:10ACA00001C020E00E940674B8CFF5C0E33411F073
:10ACB0000C94BE56E091430BE534B9F4E8EEF9E1AB
:10ACC0000E94FF720E94C11CF3974CF00E944C62DC
:10ACD000E05FF84D0E94BD700E94D97801C0E0E3AA
:10ACE000EA930E941A630E943678E091430BE6349F
:10ACF000A9F441E050E00E944C620E2F0E940579B9
:10AD0000E13019F40E944C62AF011A930E94D96C91
:10AD1000E05FF84D0E94B6760E94AB1DE091430BB8
:10AD2000E33591F40E9409790E940270E83131F410
:10AD3000E091890BEA930E945D1806C0E885EA93CA
:10AD4000EFEFEA930E94D826E091430BE134A9F497
:10AD5000EEEEF9E10E94FF720E940979EA930E94E7
:10AD60005C190E941726E03011F0E1E301C0E0E336
:10AD7000EA930E941A630E9436788DC0E63511F07E
:10AD80000C942357E091430BE33411F00C942257B9
:10AD90000E944C621E2F113010F40C942257A09187
:10ADA0001908A13091F50E940579E03021F0A091B9
:10ADB000A2061A1709F028C011500E944C62AF0178
:10ADC0001A930E94AC213E2F0E944D730E949071F5
:10ADD0000F010E944D730E94116E0E9410790E9413
:10ADE0000579E03071F00E944C62AF010E946173FE
:10ADF0000E9490710F010E9461730E94116E0E9467
:10AE000010791A930E9439121DC01630D8F41150CF
:10AE1000A12FEAE00E94267BA3E2EA9FF001E85519
:10AE2000F94FBF01A12FEAE00E94767BF0E0BB0161
:10AE3000AAE0B0E00E94F47ADB01AE0FBF1F1496C7
:10AE40000E94277128C0E93431F5E091430BE035C9
:10AE500051F40E944C621E2FE0E0EA931A930E9484
:10AE60002F19E0932E06E091430BEC34A1F40E94DD
:10AE70001062E09328060E940579E03021F00E94DC
:10AE80001062E09329060E940579E03021F00E94CB
:10AE90001062E0932A060E94B16131CD0E94A97D23
:10AEA0002B960895A091580BA03521F4A091590B31
:10AEB000A33608F005C0E091590BEA930E947C1973
:10AEC000A091580BA33521F4A091590BAA3008F09A
:10AED00005C0E091590BEA930E94A719A091580B65
:10AEE000AB3421F4A091590BA03808F005C0E091D3
:10AEF000590BEA930E94E519A091580BA63521F44D
:10AF0000A091590BA03108F005C0E091590BEA93CC
:10AF10000E94131AA091580BA43511F40E9498189E
:10AF20009CD60895E3EAF6E0FA93EA93E091420BA7
:10AF3000EA93E0E8F0E00E94397008950E941879E1
:10AF4000A0E0A083E091400BE093590BE091420B0D
:10AF5000E093580B08950E94A27D0E94F561E130B4
:10AF600010F40C94A55AE091580BA091420BEA17EB
:10AF700009F098DFE091420BE33239F5E091430BA1
:10AF8000EC3431F4CFDFE4E0E09318080E941E793E
:10AF9000E091430BE435C1F4C5DFE091630CE03090
:10AFA00029F0EF77A9E0B0E00E94027CE091640C08
:10AFB000E03029F0EF77AAE0B0E00E94027C0E9426
:10AFC0001E79E7E0E093180802C0EB34E1F5E09168
:10AFD000430BE13211F4A6DF35C0E53211F462DF34
:10AFE00031C0E33299F40E94247921F00E942F7934
:10AFF0000E94B1190E941879E081EB3429F4E0E055
:10B00000E093340CE093350C99DF1CC0E134D1F4AB
:10B010000E944C629F012093340C0E94357991F07C
:10B020000E944C629F01A091340CF901E270F07013
:10B03000EA2BE093340C0E94357921F00E944C6297
:10B04000E093350C7FC2E33581F5E091430BE132AB
:10B0500011F468DF29C0E33299F40E94247921F0C9
:10B060000E942F790E948B190E941879E081E335A4
:10B0700029F4E091400BEA930E94D41B5FDF14C0D7
:10B08000EE3491F40E94B67410E01A3068F4A3EB29
:10B09000BBE0EE27A10FBE1F0E947671EC5BF44F60
:10B0A000E081EC931F5FF1CF4DC2E63511F00C94B7
:10B0B000A158E091430BE13211F434DF41C0E33297
:10B0C00099F40E94247921F00E942F790E94F319AB
:10B0D0000E941879E081E63529F4E091400BEA936B
:10B0E0000E94261A2BDF2CC0E63531F40E944C62F8
:10B0F0009F012093300C24C0E53471F40E944C620F
:10B100009F0120932F0C0E94357929F00E944C62F8
:10B110009F012093320C14C0E43591F440E050E0DC
:10B120000E944C629F01022E032A11F042E050E07F
:10B130000E94357919F00E944C62AF014093310CA6
:10B1400001C2E43511F00C945B59E091430BE332FA
:10B1500031F40E944C623197E093400BABC0E03574
:10B1600011F00C945A5910E00E94F97850F00E94A6
:10B170000D73AC91AD3329F00E94FD7811F01E30B3
:10B1800008F005C00E9476710E943B79EDCF0E94C5
:10B1900076710E944479EDE30E94497911F00C9494
:10B1A0005A59E4E5E093580B10E00E949B703496E6
:10B1B000E491EF3F11F40C945A590E94BA740E9422
:10B1C0009B700E94C16D0E94F868E03011F00C94F1
:10B1D00058590E949B703496E491E03851F40E94D3
:10B1E0004C62E058FF4FE093630CE0E8E093640C9E
:10B1F0005FC0E23839F40E944C62E058FF4FE093A0
:10B20000640C56C0E13839F40E944C62A8E0B0E00A
:10B210000E94027C4DC0E03011F0E13051F40E94F8
:10B220009170FF93EF930E944C62AF91BF91EC93AA
:10B230003FC0E23059F40E949170FF93EF930E9457
:10B240004C62AF91BF91ED93FC9332C0E33051F467
:10B250000E949170FF93EF930E942B62AF91BF9178
:10B26000EC9326C0E43021F50E949B703596E49162
:10B27000EA930E94FA620E949170E093610CF0934D
:10B28000620C00E00E949B703596E4910E1780F4EA
:10B290000E94D96CEC5BF44FE081A091610CB091FD
:10B2A000620CEC93A1E6BCE00E94B36E0F5FEACFA4
:10B2B0001F5F7BCF47C1E03511F00C94A25AE0919B
:10B2C000430BE33299F40E94247921F00E942F79F4
:10B2D0000E945C190E941879E081E03529F4E09120
:10B2E000400BEA930E94E91B29DE2CC1E13211F4E4
:10B2F00019DE28C1E134D1F40E944C621E2F00E017
:10B300000D3098F40E94DF74EA0FFB1F3396E4912E
:10B31000E11749F40E94DF740E94E374A0919A0B34
:10B32000EA2BE0939A0B0F5FEBCF0CC1E63559F592
:10B33000E0E0E093410BADE9BBE00E944E79FF9362
:10B34000EF930E944C62AF91BF91EC93EBE2EA93D2
:10B350000E94C161E03059F0A0EABBE00E944E7942
:10B36000FF93EF930E944C62AF91BF91EC930E94C8
:10B370005179A091410BA33018F40E94357909F45A
:10B3800001C0D9CFDFC0ED34D1F4E0E0E093410B50
:10B39000A9EABBE00E944E79FF93EF930E944C62B2
:10B3A000AF91BF91EC930E945179A091410BA330D2
:10B3B00018F40E94357909F401C0EACFC3C0E7351B
:10B3C000D1F4E0E0E093410BA0EBBBE00E944E79AA
:10B3D000FF93EF930E944C62AF91BF91EC930E9458
:10B3E0005179A091410BA23018F40E94357909F4EB
:10B3F00001C0EACFA7C0E434C9F5E0E0E093410B17
:10B400000E944C629F01E2E0EA930E94CE61AF018C
:10B41000E3E70E94497959F40E945779BF01D901A5
:10B420000E941872E40FF51FDB01ED93FC93E9E431
:10B430000E94497979F40E94577920833183AAE9DF
:10B44000BBE00E944E790F010E945E79EC91E160B1
:10B45000D001EC930E945179A091410BA33018F4D4
:10B460000E94357909F401C0CBCF6CC0EE3499F459
:10B470000E94B67410E01A3068F4AAE8BBE0EE2728
:10B48000A10FBE1F0E947671EC5BF44FE081EC933C
:10B490001F5FF1CF57C0E33449F40E94F5780E9452
:10B4A0004C62E093950BF093960B4CC0E33589F416
:10B4B0000E944C629F0100240216030624F42B30E4
:10B4C000E0E03E070CF004C0F9013197E093970BE0
:10B4D00039C0E53529F40E944C62E093990B32C0E3
:10B4E000EF3491F40E944C621E2FECE2EA930E942A
:10B4F000C161E12FE295E07FEF930E944C62AF9132
:10B50000EA0FE093980B1EC0E035E1F4E0E0E09331
:10B51000410BACEABBE00E9464790E949071FF93FA
:10B52000EF930E94DA62AF91BF91ED93FC930E947A
:10B530005179A091410BA23018F40E94357909F499
:10B5400001C0E7CF0E94B16108CDE0E0E093430A7B
:10B550000E94A97D269608950E94A47D0E94F5610F
:10B56000E13010F40C945E5DE091420BE332A9F4FB
:10B57000E091430BE03519F4E1EFF9E109C0E8345B
:10B5800019F4E2E1FAE104C0E33531F4EDE2FAE165
:10B59000FA93EA930E942B638EC2E43511F00C9467
:10B5A000695BE091430BE43229F4E8E2F0E00E94A9
:10B5B00068798EC0E33211F402D98AC0E03511F007
:10B5C0000C94685BE7D8A091400BA83210F00C9463
:10B5D000685B0E946C790E94C16D0E942B63EDE351
:10B5E000EA930E941A630E946C793496E491E038E1
:10B5F00039F40E94236E0E9493740E944D6368C0C8
:10B60000E23839F40E948C700E9493740E944D635A
:10B610005FC0E13839F40E948E740E9493740E94D6
:10B620004D6356C0E03011F0E13051F40E946C7966
:10B6300032960E94CF7B0E9495710E94707948C01B
:10B64000E23059F40E946C7932960E94CF7BDF0180
:10B650000E9401740E944D633BC0E33051F40E948C
:10B660006C7932960E94CF7BE081EA930E945B6303
:10B670002FC0E43069F50E946C7932960E94CF7B2E
:10B68000E093610CF093620C10E00E946C793596A7
:10B69000E4911E1790F40E947671EC5BF44F0F0159
:10B6A000A091610CB091620CEC91D001EC93A1E6F9
:10B6B000BCE00E94B36E1F5FE8CF0E946C793596A4
:10B6C000E491F0E00E9444790E94BA740E94A4635D
:10B6D000F2C1E33579F5E091400BEA930E948B19B2
:10B6E000E091430BE43229F4EAE0F0E00E9468794B
:10B6F00020C0E33211F463D81CC0EE34D1F44AD830
:10B7000010E01A3068F40E947671EC5BF44F0F0180
:10B71000A3EBBBE00E94A175D001EC931F5FF1CFBA
:10B72000E0E0E0934E0B0E94BA740E94A4630E9472
:10B730003678C1C1E635D9F5E091400BEA930E9415
:10B74000F319E091430BE43229F4E5E0F0E00E94C4
:10B7500068792CC0E33211F432D828C0E53451F4B2
:10B7600019D8E0912F0C0E9493740E947479E09193
:10B77000320C19C0E63529F40E94CA53E091300C0E
:10B7800012C0E43599F40E94CA53E091310CE030C4
:10B7900011F0E1E301C0E0E3EA930E941A630E9422
:10B7A0007A79E091310CF0E00E94C47884C1E035F0
:10B7B00011F00C94285DE091400BEA930E945C1913
:10B7C000E091430BE43229F4E3E6F0E00E9468796B
:10B7D0003EC1E33219F40E94DF5339C1E13411F064
:10B7E0000C94345C0E94CA5312E0A0919A0BECEDC9
:10B7F000EA233E2F00E00D3078F40E94DF740E94AF
:10B80000E374E31739F40E94DF74EA0FFB1F3396E9
:10B81000149102C00F5FEFCF0E94A66D0E942C789A
:10B82000E091980BE03089F0E8E4FAE10E94FF72C1
:10B830000E94856D0E9493740E947479E091980B28
:10B84000EF700E9493740E942C78E091990BE03085
:10B8500051F0EBE4FAE10E94FF72E091990B0E9433
:10B8600093740E942C78F3C0E43479F50E947E79B9
:10B87000A091410BA33040F5E091410BE03011F075
:10B880000E947A790E945E79EC91E17061F4A3EAFA
:10B89000BBE00E9464790E94116E0E9401740E94B4
:10B8A000AF63E3E70BC0A3EABBE00E9464790E94A8
:10B8B000116E0E9401740E944D63E9E4EA930E94B4
:10B8C0001A630E945179D4CFBEC0ED34C9F40E94EE
:10B8D0007E79A091410BA33090F4E091410BE030D0
:10B8E00011F00E947A79A9EABBE00E948479EC9178
:10B8F0000E9493740E944D630E945179EACFA3C0C5
:10B90000E735C9F40E947E79A091410BA23090F4F2
:10B91000E091410BE03011F00E947A79A0EBBBE09E
:10B920000E948479EC910E9493740E944D630E945E
:10B930005179EACF88C0E63531F50E947E79A09131
:10B94000410BA330F8F4E091410BE03011F00E947C
:10B950007A79ADE9BBE00E948479EC910E949374FE
:10B960000E944D63EBE2EA930E941A63A0EABBE0F7
:10B970000E948479EC910E9493740E944D630E940E
:10B980005179DDCF60C0EE34D1F40E94CA5310E08B
:10B990001A3068F40E947671EC5BF44F0F01AAE84C
:10B9A000BBE00E94A175D001EC931F5FF1CFE0E0F6
:10B9B000E0934E0B0E94BA740E94A46344C0E33427
:10B9C00099F40E94CA530E94BA74E3E5FAE1FA932B
:10B9D000EA930E9407700E941A740E949C750E944C
:10B9E000BA740E94A4632FC0E035A9F40E94CA5320
:10B9F000E091AC0BF091AD0BFA93EA930E94C76310
:10BA00000E947A79E091AE0BF091AF0BFA93EA9332
:10BA10000E94C76318C0E33531F40E94CA53E09115
:10BA2000970BEF5F0DC0EF3491F40E94CA530E9450
:10BA3000856D0E9493740E947479E091980BEF7069
:10BA4000F0E00E947079EBE3EA930E941A6333C03E
:10BA5000EB3489F5E091400BEA930E94B119E09133
:10BA6000430BE43229F4E0E8F0E00E94687923C057
:10BA7000E33219F40E94DF531EC0E134E1F40E9466
:10BA8000CA53A091340CE1E0EA230E9493740E940F
:10BA90007479A091340CE3E0EA230E9493740E942D
:10BAA0007479E091350C0E9493740E944D63E6E531
:10BAB000FAE10E94FF720E94B16150CD0E94D278DB
:10BAC0000E94AB7D249608951A930E944D72E0E483
:10BAD000F9E00E9419730E94D2780E948879E1816E
:10BAE000E43471F40E94887902800E94236EE05D44
:10BAF000E01529F00E948879E281EA3209F401C058
:10BB000057C00E948D790E948879E1810E949179C5
:10BB10000E948879E2810E9491790E940D731C91A4
:10BB20000E94887933960E941973E12FE23131F433
:10BB30000E949779E6E0EC930EDA3AC0E13131F4F5
:10BB40000E949779E2E1EC9307DD32C0EF30A9F46F
:10BB50000E949779EEE0EC930E94F353E13039F4C0
:10BB6000A0913508A03019F00E94F97709F402C0BD
:10BB70000E94E41C0E949D791BC0EE30C9F40E9413
:10BB80009779EFE0EC930E94F353E13089F4A091B0
:10BB90003508A03019F00E94F97709F402C00E941C
:10BBA000E41CE0E0E0933508EFEFEA930E947A545A
:10BBB00063C21A930E9415740E946970EAE7EA93BF
:10BBC0000E941A630E940D7311971C91E12FE231BC
:10BBD00031F4E6E0EA930E941A63BDD937C0E1313F
:10BBE00031F4E2E1EA930E941A63B6DC2FC0EF3031
:10BBF00099F40E94A1780E94F353E13039F4A091A6
:10BC00003508A03019F00E94F97709F402C00E94AB
:10BC1000E41C0E949D791AC0EE30C1F4EFE0EA9373
:10BC20000E941A630E94F353E13081F4A091350819
:10BC3000A03019F00E94F97709F402C00E94E41CB8
:10BC4000E0E0E0933508EA930E947A54A091380826
:10BC5000AA3211F00E94F3630FC2EFEFE093580B8A
:10BC6000E093590B0895AC81A03310F0AA3308F08B
:10BC700006C00E94A479E0530E94AC7999C4AC81BB
:10BC8000A13410F0A73408F006C00E94A479E7534D
:10BC90000E94AC798DC4A881B981E0E0EC9388C49E
:10BCA000AA93EA93FA93EFB7EA931A930A931BB114
:10BCB0000CB1E0919D0CF0E0E559F34F0083A091A9
:10BCC0009D0CAF5FA0939D0CA23319F4E0E0E093CC
:10BCD0009D0C09911991F3C21A93E0919E0CA091C9
:10BCE0009D0CEA17D1F3F0E0E559F34F1081A091D4
:10BCF0009E0CAF5FA0939E0CA23319F4E0E0E0939A
:10BD00009E0CB9C1A0919D0CAE5CE0919E0CAE1B47
:10BD1000E2E30E94767B08950A921A92FA926A935D
:10BD20007A938A939A93AA93BA93EA93FA93EFB782
:10BD3000EA930E94B17949F0A0913909A03021F02D
:10BD40000E94700DE13009F401C011C0E091040DB2
:10BD5000F0E0E156F34FE081ECB9A091040DAF5F44
:10BD6000A093040DA43619F4E0E0E093040DE991EA
:10BD7000EFBFF991E991B991A9919991899179913F
:10BD80006991F9901990099018951A930E94B179C8
:10BD900059F45D9B09C0A0913909A13021F40E949A
:10BDA000700DE03009F013C01091030D0E94767100
:10BDB000E156F34FA981A0831F5F143609F410E008
:10BDC000E091040DE117E1F31093030D02C0E98146
:10BDD000ECB9A1C20E94B17921F40E94700DE1304A
:10BDE00009F001C019C350C10E94A47D8BDFE0306F
:10BDF00011F40C94F25F70DF1E2FA091680CA53631
:10BE000018F0E0E0E0933A0930913A09E0913A09FC
:10BE1000E03011F00C94595FA091E40BA13021F0B7
:10BE2000A091E40BA23031F4E12FEF77E0934009C9
:10BE3000EBE4CEC01A3521F4E1E0E0933A09CAC040
:10BE4000123049F4E4E1E0933A09E0E0E0933B0981
:10BE5000E0933D09BFC0A091E40BA33069F417370C
:10BE600029F01A3310F4103308F402C0E7E001C0DF
:10BE7000E0E0E0933C0905C01A930E94764EE093FF
:10BE80003C09A0913C09AF3F99F010934009E1E0D3
:10BE9000E0933B0910933D09E0913C09E03011F437
:10BEA000E5E404C0EAE0E0933A09E0E0E0933F090A
:10BEB00091C0E13069F4103039F4E2E0E0933A09DE
:10BEC000E0E0E0933F0903C0E0E0E0933A0982C07C
:10BED000E23059F410933C0910933D09E0E0E093FF
:10BEE0003B09E3E0E0933A0975C0E330F1F40E94C6
:10BEF000B7790E94BD79EA0F0E94C779A9F4E09151
:10BF00003D09E03071F4E4E0E0933A09E0913B0947
:10BF10000E94B16F0E94D0790E94B779A0E0A083FF
:10BF200003C0E0E0E0933A0955C0E43049F41D3025
:10BF300019F4EAE5E0933F09E0E0E0933A094AC0EA
:10BF4000EA3079F40E94B7790E94BD79EA270E940D
:10BF5000C77931F4E0E0E0933A09E5E4E0933F0982
:10BF600039C0E431B9F40E94B7791083E12FA09170
:10BF70003D09EA27E0933D09E0913B09EF5FE0933B
:10BF80003B09E0E0E093670C133019F4E5E1E0933E
:10BF90003A0920C0E53111F0E63159F41A93E7E689
:10BFA000FCE0FA93EA93EAE3F9E0FA93EA935BDEC2
:10BFB00011C0E73179F4E0E0E0933A09173131F448
:10BFC000E091670CA0913D09EA1709F003C0E3E492
:10BFD000E0933F09A0913A093A1719F0E0E0E093A5
:10BFE000680C04CF0E94AB7D44C4AA93BA93EA9331
:10BFF000FA93EFB7EA931A930A9310919B0000917A
:10C000009C00E12FEC71A9F4E091CD0DF091CE0DE3
:10C01000EB5FF24F0083ADECBDE00E94B36EE83CF5
:10C02000A0E0FA0731F4E0E0F0E0E093CD0DF0930A
:10C03000CE0D09911991E991EFBFF991E991B9916B
:10C04000A99118951A930E94D5790E94DA79D9F3AB
:10C050000E94D579EB5FF24F1081AFECBDE00E94FA
:10C06000B36EE83CA0E0FA0731F4E0E0F0E0E093E2
:10C07000CF0DF093D00DE12F199108950E94D5793D
:10C080000E94DA7909F0C8C1E0E008950E94A47D19
:10C09000F5DFE03021F0A091660CA03009F0E5C09A
:10C0A000D1DF1E2FA091D90DA53618F0E0E0E09366
:10C0B000D30D3091D30DE091D30DE03059F4113010
:10C0C00019F4E4E0E093D30D1A3519F4EAE0E093B3
:10C0D000D30DC3C0E430C1F4E0E0E093D30D1A32D5
:10C0E00029F00E94236EE05DE11769F4109338088F
:10C0F0001093D40DE5E0E093D30DE0E0E093660CFF
:10C10000E1E0E093D60DA9C0E530A9F4E0E0E093CA
:10C11000D30D0E94236EE05DE11761F00E94E1798A
:10C120000E94EA79E091D60DEF5FE093D60DE6E04C
:10C13000E093D30D92C0E63091F4E091D60D0E94C9
:10C14000EA790E94E179EF5FE093D60DE0E0E093B9
:10C15000D70D133019F4E7E0E093D30D7EC0E7303C
:10C1600011F0E83059F41A93E7EDFDE0FA93EA9301
:10C17000E3EDFDE0FA93EA9376DD6FC0E93081F4F8
:10C18000E0E0E093D30D173131F4E091D70DA091A9
:10C19000D40DEA1709F003C0E4E5E093660C5DC036
:10C1A000EA3041F4103011F4EBE001C0E0E0E0933C
:10C1B000D30D53C0EB3071F4E0E0E093D60D109353
:10C1C000D50D1093D40DECE0E093D30DE0E0E093B7
:10C1D000660C43C0EC30A1F5E091D60DF0E0E05CD8
:10C1E000F64F10830E94E179EF5FE093D60DE09166
:10C1F000D50DE150E093D50DA091D50DA03021F4DF
:10C20000A091D40DA03009F00EC0EDE0E093D30D65
:10C21000E091D60D0E94B16F0E94D079E091D60DC9
:10C22000F0E00E94D079A091D50DA03021F4A0912A
:10C23000D40DA03009F403C0E0E0E093D30D0DC0AD
:10C24000ED3059F4E0E0E093D30D1D3031F4EAE530
:10C25000E093660CEFEFE093650CE091D30DE317EC
:10C2600019F0E0E0E093D90D13CF0E94AB7D01C33C
:10C27000AA93EA93FA93EFB7EA93E091DB0EA091C9
:10C28000DA0EEA1791F0E0913708E03019F0E894FF
:10C2900026F80AC00E94EF79F0E0E030A1E0FA074A
:10C2A00019F4E0E0E093DB0E03C0E89425F826F8EB
:10C2B000E091650CE03019F0E0E0E093D30DE991F6
:10C2C000EFBFF991E991A99118951A93E091DB0ECE
:10C2D000A091DA0EEA1721F4E0919B00E072C1F41C
:10C2E000E091DA0EF0E0E652F24FA981A0831091BE
:10C2F000DA0E1F5F0E94F46CA030E1E0BE0709F483
:10C3000010E0E091DB0EE117E1F31093DA0E03C0C9
:10C31000E981E0939C00188122960895E0E0E09383
:10C32000DB0EA091DA0EA13020F00E94EF79689424
:10C3300026F80895AA93BA93EA93EFB7EA93E091A7
:10C34000650CE03041F4E0E0E093DB0E0E94236EE8
:10C35000EF5FE0933708E991EFBFE991B991A991B7
:10C3600018950E94F97818F00E94FD7809F403C02E
:10C370000E940674F6CF0E94FD7811F40E940674A4
:10C3800008950E940D73AC91E881EA1729F40E9488
:10C3900006743197E1E05DC1E0E05BC10E94A47DDD
:10C3A00000E010E0EEE20E944979E9F420E030E09C
:10C3B000EC810E94F177BCF4D8010E94C9748F010E
:10C3C0000E94CE7818F00E94FD7908F009C00E9402
:10C3D0000D73EC910E948B730E0F1F1F0E94067449
:10C3E0002F5F3F4FE5CFF801E1C00E94F97828F0B8
:10C3F0000E948879E181E03208F410C00E940D7338
:10C40000EC91E093420B0E9406740E940D73EC9134
:10C41000E093430B0E940674E1E008950C94C66615
:10C420000E9447760E9401790E946468EF3F89F07C
:10C43000F8010E94CF7AFF93EF930E9401790E9446
:10C440006468AF91BF910E94DB748F010E940674F3
:10C45000E9CFF8011EC01A930A9310E00E940D73F1
:10C460000C910B3311F0003208F412C0013310F0BC
:10C47000093308F007C0E02F0E948B73E255FF4F8D
:10C48000E4911E2B0E9406740E940D730C91E9CF5B
:10C49000E12F0991199108950E94A47D00E010E018
:10C4A0000E940D73AC91AD3221F40E94067431E00C
:10C4B00001C030E00E94CE7818F00E94FD7908F0AB
:10C4C00009C0D8010E94C9740E94017A8F010E949C
:10C4D0000674F0CF303021F4F8010E94AB7DC9C161
:10C4E000F8010E94BB7A0E94AB7DC3C124971A93C6
:10C4F000E0E0E983EA83EB83EC830E940D73AC9167
:10C50000AD3221F40E94067411E001C010E00E94D7
:10C51000CE7818F00E94FD7908F022C0A981BA8176
:10C520008B819C81EAE0F0E060E070E00E94217B7A
:10C530007F936F93FF93EF930E940D73EC91E05301
:10C54000AF91BF918F919F91FF27662777270E9418
:10C55000B17AE983FA836B837C830E940674D7CF18
:10C56000103031F4E981FA816B817C81188120C01F
:10C57000E981FA816B817C810E94BF7A188118C0A1
:10C580000E94A47D20E030E000E010E0EC810E94F9
:10C5900058765CF4D9010E94C9740E94017A9F0107
:10C5A0000E9406740F5F1F4FF1CFF9010E94AB7D0F
:10C5B000259608950E94A47D6FDF8F0120E030E072
:10C5C000EEE20E94497911F467DF9F01112322F402
:10C5D000F9010E94BB7A9F01A0911B0CA13030F0A1
:10C5E000D8010E941872E20FF31F8F01F8010E9418
:10C5F000AB7D3FC11A9310E00E94F578E030A1F0C6
:10C600000E94F97858F00E940D73AC91A23231F07B
:10C610000E94FD7819F0E9811E1708F005C00E94FC
:10C6200076710E943B79ECCF0E9476710E9444792A
:10C630000C942267E8810E949179E881A0915C0BBB
:10C64000EA0FE0935C0BE881A0915D0BEA27E09391
:10C650005D0B219608951A9310E0E12FA981BA810C
:10C660000E94DB74E491E03049F0E12FA981BA81A6
:10C670000E94DB74E4910E94077AEFCF0BC01A93FB
:10C6800010E00E944476E03029F00E9444760E9437
:10C69000077AF7CF18812396089564970E945E75F4
:10C6A0000E940C7AE88DF98D0E941A740E948E7592
:10C6B000E6DF669608951A93ECE3EA93BBDF11E098
:10C6C000193080F40E947671E255FF4FE491A98100
:10C6D000EA2319F0E12FE05D01C0E0E2EA93AADF6E
:10C6E0001F5FEECFEEE3EA93A5DF0C942267649719
:10C6F0001A930E94117A0E940C7AEA8DFB8D0E9497
:10C700001A740E949C750E94117A0E9420691E2F43
:10C71000ED891E1720F40E9432781F5FF9CF0E9426
:10C72000117AADDF18810EC064970E945E750E9479
:10C730000C7AE88DF98D6A8D7B8D0E9467740E945A
:10C740005E759DDF68960895E2E2EA9373DF0E94CA
:10C75000DA7795DFE2E2EA936DDF0C942367A88134
:10C76000B981E4E6F0E00E94477B0E947079EEE236
:10C77000EA9360DFA881B981E4E6F0E00E94797B6A
:10C78000FA93EA93E2E0EA93B2DF0C942367A09174
:10C790001B0CA13020F00E94DA77E1DF07C00E9475
:10C7A000DA777BDFE4E6FAE10E94FF720C942367FC
:10C7B00025FE06C0E5E0F0E00E94936EA895F8CF54
:10C7C000EAEDFDE0E0935E0BF0935F0BE1E00E9489
:10C7D0005472E0935C0B0E94167A0E94236E0E94B2
:10C7E00095780C9461691A930A93E091650CE03096
:10C7F00011F00C949568E3E0EA931CDFE0915C0B88
:10C80000E295EF70EA930E947B681E2FE0915C0B2B
:10C81000EF70EA930E947B680E2F1A930BDF0A9346
:10C8200009DFE7E1EA9306DFEAEDFDE0A0915E0BA8
:10C83000B0915F0B0E94E37BEA1BE093DA0E6894F1
:10C8400025F80C949568EE81EA93B2DFEC81FD81C6
:10C850000E94FF720E941A7A67DFC5DF0C94886914
:10C86000EB81EA93A5DF0E947171F5DE0E94167AD2
:10C87000BADF24960895ED81EA939ADFEB81FC817B
:10C880000E94FF72EA81EA93D5DEE981E03011F07F
:10C89000EA93D0DEE881E03011F00E94167AA3DF3F
:10C8A000269608950E94A27D10E0E8E6FAE1A885A8
:10C8B000B985EA17FB0719F444E150E002C048ECDF
:10C8C00050E0EA85E0933809E89431F8EA93E98585
:10C8D000FA85FA93EA93EA85EA93EA85EA93E0E037
:10C8E000EA93C9DF0E948C689F010E94B7150E94DD
:10C8F00090760E9498680E2F31FC02C0003009F03B
:10C9000001C0F3CF31FE04C0E89431F8E1E004C087
:10C910001F5F1230B0F2E0E00E94A97D2B960895CF
:10C920001A930A93E091400AE03011F40C94956850
:10C93000E0E0E0933909E2E0EA9327DA10E003E06F
:10C940000E9476710E94217A61F00E9476710E94A5
:10C95000F6770E947671E05CF54FE0810E271F5F4D
:10C96000EFCFE3E0EA9311DAE02FE295EF700E9457
:10C97000267AE02FEF700E94267AE7E1EA9305DA43
:10C980000C9495681A930A93E091400AE03011F4F0
:10C990000C9495680E948C70E03021F0E091420A7E
:10C9A000EA3209F405C00E948C70E05DE093420A0F
:10C9B000E0E0E0933909EAE5EA93E7D9E0E0EA93B9
:10C9C000E4D910E00E9476710E94217A11F01F5F75
:10C9D000F9CF1F5F012F0A93D8D910E00E9476711A
:10C9E0000E94217A61F00E9476710E94F6770E947F
:10C9F0007671E05CF54FE0810E0F1F5FEFCFE02F07
:10CA0000E195EA93C2D9EDE0EA93BFD90C94956819
:10CA10001A930A93F894E0E0E0933708E091DB0E74
:10CA2000E093DA0E7894E091400AE03011F40C942F
:10CA30009568EAE5EA9349DCE0E0EA9346DC10E039
:10CA40000E9476710E94217A11F01F5FF9CF1F5F5B
:10CA5000012F0A933ADC10E00E9476710E94217A3D
:10CA600079F00E947671E05CF54FE081EA932DDC6D
:10CA70000E947671E05CF54FE0810E0F1F5FECCFF6
:10CA8000E02FE195EA9321DCEDE0EA931EDC0C94C3
:10CA90009568E881EA938CDEEAE5EA93CBDDE091E4
:10CAA0004009EA93C7DD0E940D73EC91E03031F04C
:10CAB0000E940179BFDD0E940674F5CF94DE0C94CC
:10CAC00061691A930E944D72E0913B08EA93B2DDCE
:10CAD000E4E4EA93AFDDE0913908EA93ABDD14E0DA
:10CAE0000E947671E85CF74FE081E43040F00E94EC
:10CAF0007671E85CF74FE0810E94077AF1CFE0E0C1
:10CB0000EA9398DD3FDF3DC11A930A936DD9E09116
:10CB10003F09E03011F40C940166A0913F09AA3559
:10CB200041F4A0913B09A33020F0E0914109E434A5
:10CB300009F04BC00E948C70E03021F0E091420976
:10CB4000EA32C1F40E94236EE05DA0914209EA1727
:10CB500021F0E0914209EA3221F40E94645D12DF83
:10CB600008C0E3E4F9E00E941973E09142090E94D1
:10CB70002C7A2BC00E948C70E05DA0914209EA17CC
:10CB800021F50E94236E1E2FE0914309ED3421F41C
:10CB9000E0914409E33209F007C0E5E4F9E00E94BE
:10CBA00019737ADC1E2FDDDB0E94236EE11729F05A
:10CBB000E12FE05D0E942C7A08C00E94236EE05DA8
:10CBC000E09342090E94645DDDDEA0913F09A53437
:10CBD00049F4A091E40BA33019F40E945F2B02C02A
:10CBE0000E94E94EA0913F09A33411F40E94172B33
:10CBF000A0913F09AB3411F40E94122BE0E0E093C6
:10CC00003F09A091E40BA33011F40E945F2BE0E0F8
:10CC10000C9495683BDAA091660CA43529F4A0E049
:10CC200025FCA1E0A03009F03AC0E0913A08E035D7
:10CC300081F4E0913B08EA93E6E0EA930E946B43BB
:10CC4000A0913B08A03820F0E0913B08E0936505F7
:10CC500023C0E03721F4E0E0E09365051DC0EA352C
:10CC600019F40E94D95D18C0EA3711F42ADF14C004
:10CC7000E23519F40E94FC500FC0E23719F40E940B
:10CC800031510AC00E94E330E0913908A09138097F
:10CC9000EA1711F4689431F8E0E0E093660CA09193
:10CCA000660CAA3531F40E94645DB2DEE0E0E093E8
:10CCB000660C6CC0A091690CA13050F0E091690C39
:10CCC000E150E093690CE03019F4E1E0E0936A0C84
:10CCD000A0E025FCA1E0A13049F4A0E026FCA1E001
:10CCE000A03021F4A0913708A03009F001C016DB74
:10CCF000E0913708E03019F0E150E09337080895EB
:10CD0000E091D90DEF5FE093D90DE091680CEF5FF2
:10CD1000E093680CE091650CE03019F0E150E0938D
:10CD2000650C0895A091E40BA13021F0A091E40BD3
:10CD3000A23029F4E3E0E0939000E8E3E9B9089534
:10CD4000E0E00E94166CE1B3E360E1BB85E38A9505
:10CD5000F1F7E1B3EC7FE1BBE4E4E09374000E94FF
:10CD60002D6C08951A9314EAE4EA0E94337A41F490
:10CD70000E94387A183011F0103111F4E0E001C04F
:10CD8000E2E019910895E4E9E0937400E0E0089589
:10CD90001A93E981E1600E943D7A31F40E94387A69
:10CDA000103411F4E0E04EC04CC01A93E9810E94A7
:10CDB0003D7A31F40E94387A183111F4E0E042C033
:10CDC00040C01A93E9810E943D7A31F40E94387A7A
:10CDD000183211F4E0E036C034C01A93E981E03033
:10CDE00011F0E4EC01C0E4E80E94337A79F40E9487
:10CDF000387AE0917300AA81BB81EC93103511F071
:10CE0000183521F4E0E018810C94DE6BE1E0188124
:10CE10000C94DE6B1A93E981E093740010E0E091CA
:10CE20007400E07811F4163908F005C08BE18A959A
:10CE3000F1F71F5FF4CFE0917400E07811F0E0E0CB
:10CE400001C0E1E01881229608950E94A47D3D81F1
:10CE50000C8120E087DFE03011F5EE810E943E6F0B
:10CE6000F1F43A93AEDFE030D1F40E94417AB9F4A4
:10CE700079DFE030A1F4EE810E94246C81F4EDB7FB
:10CE8000FEB7FA93EA931F930E94296C1F91E0303A
:10CE900031F479DFE12F0E94AB7D0C94886950DF7B
:10CEA000D9CF0E94A47D30E00E811D815BDFE03090
:10CEB00099F4EF810E943E6F79F40E94417A61F407
:10CEC0001A937FDFE03041F4EC81EA937ADFE030BF
:10CED00019F459DFE0E002C033DFE8CF0E94AB7DF8
:10CEE0002896089522970E94A27D50E02B853A85CE
:10CEF000A89538DFE03011F00C94D467EE850E94DD
:10CF00003E6F11F00C94D4672A935BDFE03011F090
:10CF10000C94D4673A9355DFE03011F00C94D46749
:10CF200021DFE03011F00C94D467EE850E94246C70
:10CF3000D9F5E0E0EE83EF83EC85FD8531970E9423
:10CF4000187649F4EDB7FEB7FA93EA931F930E945F
:10CF5000296C1F9109C0EDB7FEB7FA93EA931F93AE
:10CF6000E1E0EA933ADF1F910E2FEE81FF81A88561
:10CF7000B985EA0FFB1F1083EE81FF813196EE83A6
:10CF8000FF83003039F4EC85FD85AE81BF81AE179B
:10CF9000BF0708F001C0D0CFEC85FD850E94187650
:10CFA00019F4F1DEE0E002C0CBDEA3CF0E94A97D40
:10CFB0002F96089568970E94A27D20E0E0E0EC8F14
:10CFC000ED8F31E0A895E9A1FAA1662777270E94A5
:10CFD000797CEA87FB876C877D87EE8D0E94467A95
:10CFE000EE83FF8368877987AA85BB858C859D85BD
:10CFF0000E944F7DEA8BFB8B6C8B7D8B0E94D37BD9
:10D00000FE017296FA93EA930E94E06BEE8BFF8B1F
:10D01000688F798F0E944C7A0E94407CAF010E94F9
:10D020004C7AAE8DBB27882799270E94DA7B0E9415
:10D030005F7ADE015A960E94407CED93FC930AA130
:10D0400019A190DEE030D1F5EDA10E943E6FB1F55F
:10D050000E94417A99F51A93B4DEE03079F53030C8
:10D0600051F14F5F5F4FEC8DFD8D3196EC8FFD8F51
:10D07000AC8DBD8D1197EBA1FCA1EA17FB0711F454
:10D0800030E018C0EC8DFD8D3197AF8DB8A10E94B6
:10D090005D7697DEEE8DDA01F0E0EA17FB0751F4DA
:10D0A00072DEEA8DFB8DA9A1BAA1EA0FFB1FE9A3ED
:10D0B000FAA389CFD4CF67DEE0E002C041DEC1CF62
:10D0C0000E94A97DA6960895A881A03310F0AA33E6
:10D0D00008F004C0E881E0530C946169A881A13490
:10D0E00010F0A73408F004C0E881E7530C9461699C
:10D0F000EFEF0C946169A881AA3020F4E881E05D2B
:10D100000C946169A881AA3020F0E881E95C0C9454
:10D110006169E8E50C9461691A930A93F8940091A7
:10D12000620B1091630B7894F8010991199108959D
:10D130001A930A93F1DF8F01EA81FB81AC81BD81F3
:10D14000EA0FFB1FE01BF10BDF010E94987D2CF41E
:10D15000E0E0198108810C940C6CE1E019810881F0
:10D160000C940C6CECE9F4E1FA93EA93E8E2F0E059
:10D17000FA93EA930E94AB6DE4E1EA93EBE1EA9360
:10D18000EFE0EA930E94134EE8EBF6E1FA93EA939C
:10D19000E0E7F0E0FA93EA93EDE1F0E0FA93EA9346
:10D1A000E9E0EA93E2E1EA93EFE0EA930E94134EAA
:10D1B0000895089599818881009641F0BD81AC81E0
:10D1C000FB81EA8105900D920197E1F7FD81EC81E9
:10D1D0000C940C6CB981A881109631F0FC81EB8124
:10D1E0006A8161931197E9F7EB81FC812596089597
:10D1F000E991F991A991B9911D900590011421F43B
:10D200000020D1F7EE2708951018E1F3E1E008F4CB
:10D21000E2500895E991F991A991B991CD016191F7
:10D220006D936623E1F7FC010895E991F991A991C5
:10D23000B991CD0105900D920020E1F7FC01089510
:10D24000A991B991EE27FF276D91662311F03196D0
:10D25000FBCF0895AA27BB27E991F99105900020FB
:10D2600011F01196FBCFFD0108957991E991F991A3
:10D27000A991B991CD01772351F07A9561916D9380
:10D280006623C9F7772319F07A956D93FBCFFC01DC
:10D2900008956991E991F991A991B991CD01662318
:10D2A00051F06A9505900D920020C9F7662319F098
:10D2B0006A950D92FBCFFC0108955D9BFECFE8813E
:10D2C000ECB9219608951A930A93AC81BD810E940E
:10D2D000C07B3097C1F0AA81BB810E94C07B8F01C7
:10D2E000309749F00230E0E01E0760F0F801319716
:10D2F0008F01ED93FC93AC81BD810E94B36E319799
:10D30000AE81A08303C0EE81EA93D7DF1981088143
:10D31000279608952C970E94A27D10E0E88DF98D44
:10D320003196E88FF98F3197E4912E2FE03011F488
:10D330000C94486BE12FE03039F4253211F411E000
:10D3400002C00E94647AA3C1E130C1F4253219F40D
:10D350000E94647A9BC112E0E0E0E98B00E02D328C
:10D3600011F401E094C12B3219F4EBE2E98B8FC187
:10D37000203219F4E0E2E98B8AC102C0E23039F4CC
:10D3800050E013E0203311F4006881C102C0E330A3
:10D39000A1F4203310F02A3308F009C0A52FEAE0E9
:10D3A000EA9FF0015E2FE22FE0535E0F70C140E074
:10D3B0002E3211F414E06BC110C0E430A1F420331C
:10D3C00010F02A3308F009C0A42FEAE0EA9FF00128
:10D3D0004E2FE22FE0534E0F5AC12C3619F4026043
:10D3E00015E055C104C0E53011F00C94476BE22FF5
:10D3F000E33649F40E946F7AEE89FF89A481AA93EB
:10D400000E94757A43C1E33741F40E946F7A0E940B
:10D410007F7A0E9420691E2F0AC0E037A1F40E9483
:10D420006F7A0E947F7A0E942A691E2F08600F7708
:10D43000403011F0411708F001C0142F40E0E0E047
:10D44000E88B30E076C0E43611F0E93611F4046080
:10D4500002C0E537A1F4EAE0E88B01FF08C0E0E094
:10D46000FAEC6AE97BE30E94726E1AE023C0E0E105
:10D47000F7E260E070E00E94726E15E01BC0E835D4
:10D4800011F4086004C0E83711F00C94466BE0E139
:10D49000E88B01FF08C0E0E0F0E060E070E10E948E
:10D4A000726E18E007C0E0E0F0E160E070E00E941A
:10D4B000726E14E0403011F00F7701C041E001FFBF
:10D4C00008C00E946F7AAE89BF8914960E94C47BFF
:10D4D00013C002FF08C00E946F7AAE89BF891496FC
:10D4E0000E94166E09C00E946F7AAE89BF89149699
:10D4F0000E94C07B66277727EC87FD876E877F8732
:10D5000002FF16C0AF85AA2362F4EC85FD856E8507
:10D510007F850E94BF7AEC87FD876E877F87EDE26B
:10D52000E98BE989E03019F01F5F4F5F01C00B7F85
:10D53000342F00FD14C0151710F4351708F00FC074
:10D5400007FF08C002FF04C00B7F2989115001C0EA
:10D5500020E301C020E20E94647A5150ECCF1417FE
:10D56000B0F4006102FF0AC00B7FE989EA930E94D0
:10D57000757A503009F0515011504150E0E3EA9370
:10D580000E94757A503009F051504150E8CF312F48
:10D59000E889E030D1F43030B9F003FF08C0EE8103
:10D5A000FF813196EE83FF833197E49105C0AE8110
:10D5B000BF81ED91AE83BF83EA930E94757A5030AC
:10D5C00009F051503150E7CF57C00E94877A0E942E
:10D5D0004C7B2E2F2A3030F003FF02C0295C01C0A3
:10D5E000295A01C0205D04FD25C0213360F4A885BF
:10D5F000B9858A859B85A130E0E0BE07E0E08E0713
:10D60000E0E09E0709F40BC0431740F4531710F0F5
:10D6100000FF01C014C020E207FF0CC020E300613E
:10D6200002FF08C00B7FE989EA930E94757A5030A7
:10D6300009F051500E94647A503009F05150315035
:10D640000E94877A0E94877BEC87FD876E877F87A1
:10D65000E889A885B9858A859B85FF27662777276E
:10D660000E944C7B0E94726EE885F9856A857B85F5
:10D670000E94947D09F0A9CF00FF08C0503031F01E
:10D680005150E0E2EA930E94757AF8CF10E046CE5E
:10D690000E94A97D6A960895FF92F82E22971A9308
:10D6A0000A93DE010E94AD7A8D01DE0116960E947A
:10D6B000AD7A0E94C07BEA83FB83DE0114960E9450
:10D6C000AD7A0E9401741A930A93FE0136960E9465
:10D6D000976C20DEAA81BB81E0E0EC931981088180
:10D6E0002496FF900895A991B991EE27002460E84F
:10D6F000E894162E169407941E2A1EF0A015B10564
:10D7000018F0A019B109E62BB7FBAA0FBB1F66954D
:10D7100080F708957B816A81F981E88177FB770F33
:10D7200067FD7160972F9E5781F078F0983190F4E3
:10D73000AA27BB27882708948795B795A7959A9518
:10D74000D1F7EA23FB23682305C0E8947727EE2767
:10D75000FF2766276F77769508F4606877F9A991B7
:10D76000B99189919991EA17FB076807790797FBA7
:10D7700008950E941A7A0E94907A19F40E94977A6A
:10D780001DC0E6F7A881B9818A819B81E0E0F0E0C5
:10D7900060E87FE30E945F7A11C00E941A7A0E94BB
:10D7A000907A19F40E94977A09C0E6F30E94977A5A
:10D7B000A0E0B0E080E89FE30E94B37C2496089547
:10D7C0000E949C7A0E94947D39F4A881B9810E94BC
:10D7D0003D700E94CA7B20C0AA81BB818C819D8143
:10D7E0000E949C7D34F40E949C7A0E94D37BC1DF0E
:10D7F00005C00E949C7A0E94D37BCFDFA881B981AB
:10D800000E94CA7BA881B9810E94C47BAA81BB8186
:10D810008C819D810E945F7A26960895E991F99105
:10D8200030971AF4E095F09531960895E0937100E1
:10D83000E0E0E0937400E2B3E360E2BB089588ECBB
:10D8400090E00197F1F70895EA930E94C866E030EE
:10D850000895E0E0EA930C94ED6680E991E0019789
:10D86000F1F708951A930A930C944047EA9FF00148
:10D87000F0E00895FA93EA93A02FB0E00895ECE366
:10D88000F0E00E941C7B0895ECE3F0E0FA93EA9349
:10D890000895EAE3F3E0FA93EA930C941C44E0E081
:10D8A000E0930F04EFE0E09310040895E0E0F0E06F
:10D8B000FA93EA930895FA93EA93E8E2F0E0FA9390
:10D8C000EA93E0E0EA930C942F4CE0915905F09133
:10D8D0005A05FA93EA930895E0915B05F0915C058F
:10D8E000FA93EA930895FA93EA930C949943EFEE2E
:10D8F000F0E0FA93EA930895FA93EA93E0E0EA936A
:10D900000C942F4CFA93EA930C941C44E12FA0E45E
:10D91000B2E0F0E00E94D37AEA0FFB1F0895A12F36
:10D92000B0E0ADCFFA93EA93E2E3F0E00895FA9322
:10D93000EA93BCCFE0911004E0930F0408950E9495
:10D94000070E0C94C849E32FF0E0E05BFD4FE49133
:10D950000895EA930E941D0EFE013696FA93EA930B
:10D960000895FF27662777270E94D37B84E00E94D3
:10D970004C6B28960895FE017196FA93EA930C94E5
:10D980003C440E94A47D0C944047E8E0F0E0FA9308
:10D99000EA930895E4E0F0E0FA93EA930895FA93A5
:10D9A000EA93E8E3F0E0FA93EA9308950E94CF7BCC
:10D9B000BECFE02FF0E00895A0913A0CB0913B0C5F
:10D9C000BD01A3E0B0E00E94F47AE60FF71FE491F6
:10D9D000E0300895E091C005EE0FEE0FEF5F3E2FAF
:10D9E0000895E32FF0E00895A12FB0E00895A091ED
:10D9F0003A0CB0913B0CBD01A3E0B0E00E94F47A78
:10DA0000E60FF71F08950E94D17AE05AFD4F08955E
:10DA1000FA93EA93E22FF0E008950E94A27DA0918C
:10DA200019080895E091C20BF0E00895AFE3B1E06A
:10DA30000E94477B089530911E08E1E0E0930D04B9
:10DA4000E2E0E0930E043A930E945C19E091980B97
:10DA5000E295EF70E0930F04E091980BEF70E09384
:10DA600010040895FA93EA93E52FF0E0FA93EA930D
:10DA70000895E7E3F0E0FA93EA930895E22FE45083
:10DA8000F0E0FA93EA930895FA93EA93F7CFE32F3D
:10DA9000E058EA930BCFEAE8FBE0FA93EA930C94A0
:10DAA0003C443A930E945C19A0918A0BAD320895D0
:10DAB000E091980BE295EF70E0930F04E091980BE2
:10DAC000EF700895E52FF0E00895EA0FFB1FFA9339
:10DAD000EA930895EF5EFC4FBF01E081E058DB015F
:10DAE000EC930895E0E0EC93AE81BF810895E3E00C
:10DAF000F0E0FA93EA930895E52FE450F0E0FA930A
:10DB0000EA930895E550F0E00895E091980BE295CE
:10DB1000EF700895EA1BA2E5B7E0F0E00E94D37A27
:10DB20000895F0E0EE0FFF1FEA5CFD4F0895A4E3B7
:10DB3000B2E0F0E0EE0FFF1FEA0FFB1F0895FA932B
:10DB4000EA93E12FF0E0FA93EA930895E12FF0E0F1
:10DB5000FA93EA930895E2E0F0E0FA93EA930895E5
:10DB6000EAE8FBE0FA93EA93EAE0EA930C94E346EE
:10DB7000E1E0F0E0FA93EA930895FA93EA930C94C3
:10DB8000CE460E94CF7BFA93EA930895ABE0EA9FDA
:10DB9000F001E252FA4F0895ED85FE85FA93EA937B
:10DBA00008951A930A933ECF1A930A93E0E0EA93FA
:10DBB0000E942F4CDDCFE1E0E0933C0C0E948C688A
:10DBC000E0933D0CF0933E0C0895BD01AAE0B0E057
:10DBD0000E94F47AE60FF71F0895FA93EA93EAE0B9
:10DBE000EA930C94E346E1E0E0930E045FCE0E94DA
:10DBF00019470C94FC46E0E2EA930C94B746A6E47D
:10DC0000B7E0E881F0E0EE0FFF1FAE0FBF1F0E94EC
:10DC1000C07B0895FA93EA930C94D241E881F0E036
:10DC20000895EE0FFF1FAE0FBF1F08950E94C07B27
:10DC30000E94DE7A08950E94D37B0C94B341FA933C
:10DC4000EA930C941947A9E0B0E00E94EE7B089596
:10DC5000A7E11A9FF001EF5CF94FE0810895E12FF1
:10DC6000EF5FEA930C94E841F0E0D4CFE8E0F0E015
:10DC70005ECEEA93E6E0EA930E949E4186CEE09172
:10DC80006D05F0916E050895E0916905F0916A05C2
:10DC90000895AE0FBF1FE3E0F0E00E94477B0895B8
:10DCA000FA93EA931A930A930C944013FA93EA9323
:10DCB0003A932A930C944013A0917105B091720588
:10DCC0000895A0917305B09174050895A0E0B0E0A7
:10DCD0000E94EA7B08950E94E37BEA1BFB0B0E94F3
:10DCE000DE7A0895E887F9876A877B870895A88593
:10DCF000B9858A859B85EFEEF0E060E070E00895DD
:10DD00000E94DE7A0E94717B0895A4E0B0E00E9438
:10DD1000EA7B0895EC83FD836E837F830895FA93F5
:10DD2000EA930C943447FA93EA930C94A17AA9E00D
:10DD30001A9FF001E058FC4F089537960E94CF7B60
:10DD4000DF010E94C07B08950A921A92FA926A93A8
:10DD50007A938A939A93AA93BA93EA93FA93EFB732
:10DD6000EA931A930895ED91FD913196FE93EE9307
:10DD70000895ADE01A9FF001EB5FFC4FE08108953C
:10DD80001A93E1E0EA930C94A247ADE01A9FF001E8
:10DD9000DF01EB5FFC4FE081E0300895E2E0EA93C1
:10DDA0000C94A247FA93EA93E4E6F0E0FA93EA933C
:10DDB0000E949868E0300895E1E0E0930D04E0935C
:10DDC0000E040895E0912908F0912A0860912B082B
:10DDD00070912C080895E0912108E150A3EAB6E083
:10DDE000F0E00E94D37AAE0FBF1F0E94C47B08955B
:10DDF000E12FEF5FF0E023CFE0912208EA93E0917A
:10DE00001E08EA930E94761BA0911E0CB0911F0C75
:10DE100010970895A091200CB091210C8091220CB4
:10DE20009091230C0E949C7D0895E0911E0CF0912E
:10DE30001F0C0895E091200CF091210C6091220CB0
:10DE40007091230C0895E2E3F0E06DCF1A93E0EABD
:10DE5000EA93EA81F0E0E050F84FFA93EA930E94E7
:10DE600025671E2F0895E0EAEA93EA81F0E0E0508A
:10DE7000F84FFA93EA931A930C945167EA930E942D
:10DE8000D566E0300895E0EAEA93EEE5F0E0FA9333
:10DE9000EA93E0E0FFE0FA93EA93EEEBFBE008950B
:10DEA000FA93EA93E0E2EA930C94DA67E0EAEA9301
:10DEB000E981FA81E050FC4FFA93EA930895EA81F0
:10DEC000F0E0A8E2B0E00E941C7B0895E0EAEA934B
:10DED00042CEFA93EA930C947267FA93EA930C9405
:10DEE0002567E0EAEA93E8E2F0E0FA93EA931A930E
:10DEF0000A93EAE8FBE00895EAE8FBE0FA93EA9384
:10DF00000895EDE2EA93EAE0F0E0FA93EA930E94E2
:10DF1000EA68E0E00895EA81F0E0ABE0B0E00E945A
:10DF20001C7BE050F24F8F01AA81AA300895E0EAED
:10DF3000EA93EBE0F0E0FA93EA931A930A93E2EBA8
:10DF4000FBE00895E3EBFBE0FA93EA930895EA819E
:10DF5000F0E0EE0FFF1FE050F04F8F01AA81A038D4
:10DF60000895E150F0E00895EA81F0E00E94D37A4C
:10DF7000E058F14F8F01AA81A5300895EFE2FCE04F
:10DF8000FA93EA93E0E0EA9305CDECE1FCE0FA9342
:10DF9000EA93E0E0EA93F9CC0E941C7BDF01EA857A
:10DFA000F0E0AE0FBF1FE8E0F0E00E941C7BE05005
:10DFB000F04D8F01E0EAEA93E8CC1A930A93ECE182
:10DFC000FCE087CFAE81BF81888599850E94B17AB8
:10DFD000EE83FF8368877987089540931E0C5093E2
:10DFE0001F0CEE81FF8168857985E093200CF0930A
:10DFF000210C6093220C7093230C0895F0E0AE0F77
:10E00000BF1F0895EA930E945C190C943020E091A0
:10E01000950BF091960B0895FA93EA930C94FB18E4
:10E02000ED81EA93ED81EA930895E091AC0BF091D4
:10E03000AD0B0E94DE7A0895F0E0A4E6B0E00E9405
:10E040001C7B0895EC81F0E0EA0FFB1F0895E0913E
:10E050002708F09128080895E093270CF093280CE6
:10E060000C94C71CE3EAF6E0FA93EA93E0E0EA9343
:10E070000895FA93EA930C94EA68E0E0F0E060E037
:10E0800070E00895E0932908F0932A0860932B0824
:10E0900070932C080895E091970BA3EAB6E0F0E0A6
:10E0A0000E94D37A0895AE0FBF1F0E94C47B0895CB
:10E0B000ED5EF94FE081E1300895FA93EA93E09143
:10E0C0002208E05DEA930895EA930E945264E130E9
:10E0D0000895ECE3F8E0E093600BF093610B089592
:10E0E000E12FA3EAB6E0F0E00E94D37A08950E94FF
:10E0F000DA68A881AF5FEAE00E94267BE05D0895C0
:10E10000A881AF5FEAE00E94767BE05D0895FA9314
:10E11000EA93E0E0EA930895AAE0B0E00E94EE7B83
:10E120000895E12FF0E00E94D17AE854FF4F329633
:10E130000E94CF7B0895E12FF0E00E94D17AE8544D
:10E14000FF4F08953696E491D901EC930895E0EAE3
:10E15000EA93E5E0F0E0FA93EA930895EA930E94E7
:10E16000B81CFA93EA93E4E2FCE00895FA93EA9388
:10E17000EFEFEA93E5E0F0E07CCFE093250CF0933D
:10E18000260C08950E94E37BEA1BFB0B0895A091E7
:10E190002A0CB0912B0C0895E0E0E093380CE0934A
:10E1A000390C0895A0912C0CB0912D0C0895E0919C
:10E1B0002C0CF0912D0CAC81BD81EA0FFB1F089552
:10E1C000E0932C0CF0932D0C08951A930E94521D8D
:10E1D0001E2F0895E0932A0CF0932B0C0895FA93C8
:10E1E000EA930E949868E0300895ABE01A9FF0012E
:10E1F000E452FA4F08951A930E943E1FD3CFE09144
:10E200002A0CF0912B0C0895EA930E943E1F0E9465
:10E21000DB1EE0300895EB81EA930E94791DFA93AA
:10E22000EA93E9E2FCE00895E0E0E0934D0CE0932E
:10E230004C0C08951A930A93E0911208ABE0EA9F00
:10E24000F001E752F84F8F01D80111960895E0E0F0
:10E25000F0E0ED93FC930895EA81D801EC93E2E1BC
:10E26000F8E0FA93EA930E94143419810881089522
:10E27000E12FACE8B0E0F0E0EE0FFF1FEA0FFB1F6C
:10E280000E94CF7B0895ACE8B0E0F0E0EE0FFF1FF6
:10E29000EA0FFB1F0E94CF7B0895A0911608B09152
:10E2A0001708EA2BFB2BE0931608F0931708089544
:10E2B000E150A7E1EA9FF0010895A7E10A9FF0016C
:10E2C000E15DF94FAF010895A3E21A9FF001ED550A
:10E2D000F94F0895EC93EC81E150ADE0EA9FF00135
:10E2E0000895E981FA81FA93EA930895E12FF0E025
:10E2F0000895E2E0F0E00E94477B0895AAE9BBE0C0
:10E30000E0911A080895ADE9BBE0E0911A0876CED5
:10E31000A0EABBE0E0911A0871CEA6E4B7E0D2CB48
:10E32000EE0FFF1FEA0FFB1F0895E081F0E0089554
:10E33000A7E11A9FF001E15DF94FEE83FF83AE8103
:10E34000BF810895EE81FF81A481AA930C94772068
:10E350000D901C90AE81BF811296EC91F0E0E00D23
:10E36000F11DDB01ED93FC930895ED91FD91319743
:10E37000FE93EE9308950E940D220E2EAA85BB8572
:10E38000EC91E0150895A3E20A9FF001E855F94FDA
:10E390000895E0911208ABE0EA9FF001E752F84FD0
:10E3A000EC87FD87AC85BD85119608951296EC919A
:10E3B000AC85BD851696EC930895D001F0E00895E4
:10E3C000A885B98518960E94C07B0895AC85BD8547
:10E3D000EC93E2E1F8E0FA93EA930C941434E885C4
:10E3E000F985A281AA9308950A930E946720E030DC
:10E3F0000895AA85BB85EC91EA93E3E0EA930C9437
:10E400006B43AA85BB85E0E0EC93E2E0E093240651
:10E410000895BF0100801180AE81BF811296EC91FA
:10E420000895DB01ED93FC93AE81BF8112965ACB28
:10E43000E4E6F0E00E941C7B0895F0E0ED93FC938D
:10E440000895E2E1F8E0FA93EA930C941434E09131
:10E450001908A0911808EA170895F0E0E00DF11DE1
:10E460000895A3EABBE042CFADE9BBE0EE27A10FE0
:10E47000BE1FEC910895A0EABBE0EE27A10FBE1FDE
:10E48000EC910895BD01AAE0B0E00E94F47ADB01AE
:10E490000895E081EA930C94C55EE0E4FAE0E0932D
:10E4A0005E0BF0935F0B0895EA930E941A63E0E01D
:10E4B0000895EA930E941A630C949064ADE9BBE05E
:10E4C000EE27A00FBE1FEC910895A0EABBE0EE2757
:10E4D000A00FBE1FEC910895AAE9BBE0EE27A00FA4
:10E4E000BE1FEC91E1700895A3EABBE062CAA0EB05
:10E4F000BBE0EE27A00FBE1FEC910895A9EABBE098
:10E50000EE27A00FBE1FEC910895ADE0EA9FF00149
:10E51000E15FFC4F0895ADE0EA9FF001EB5FFC4F37
:10E520000895ABE00A9FF001E452FA4F0895ABE082
:10E530000A9FF001EE51FA4F0895FA93EA930C9472
:10E540009F35FA93EA930E94DD433A9327CCE091FA
:10E550002C0CF0912D0C30970895AFEFBFEFA083F6
:10E56000B18308950E948C68E093520CF093530C91
:10E570000895FA93EA93E0E0F0E80895E091120834
:10E58000ABE0EA9FF001E752F84FFA93EA930E945A
:10E59000732957CFE0911008ABE0EA9FF00108958E
:10E5A000E0E1F8E0FA93EA930C941434FA93EA93D6
:10E5B0000C94A553E88DABE0EA9FF0010895FA931F
:10E5C000EA93F7C9E0E1EA93E0912506EA930E9415
:10E5D0002F191E2F08953BDDFA93EA930895FA93BD
:10E5E000EA930C94091FE0932506E0E0E0934F0CBA
:10E5F000E1E3E093500C0E94B22A0C949026FA9327
:10E60000EA930C942B63E1E4F9E0E093600BF09360
:10E61000610BE3E0EA930C94C062A091600BB091AF
:10E62000610B08950E948C68E093470CF093480CAE
:10E630000895E093600BF093610B0895E3E0EA9393
:10E640000C94C062E0932708F093280808950E9474
:10E650004047E0E0EA930C941A0FE0E0F0E0E0932A
:10E660002508F0932608E2E0E0930E040895E09177
:10E67000130448CAE0912508F0912608CBCAE0911E
:10E680005D05F0915E0531970895FA93EA930C9435
:10E690001246EF5CEA930C94B746A6E0B7E0A1C936
:10E6A000A3EABBE0E0911A08F0E03ACE0E94C07BFA
:10E6B000D001ED93FC9322CEF0E0EA0FFB1F0F0197
:10E6C0001DCEA6E4B7E08DC9E7E0E0931808EA9311
:10E6D000E0E0EA93EBC8EA930E9447410E947E4340
:10E6E0001E2F0895EAE2EA93E7E7F8E110CD0E94D1
:10E6F0005E2CE1E0EA930C94462C1F771A930C945D
:10E700005C19A0912508B09126080895E8EEF3E081
:10E710000E94797B0895E053F0E00895A0E024FC86
:10E72000A1E0A0300895E0E0EA93C0C8E09133088A
:10E73000F0913408FA93EA930895FA93EA930E94C9
:10E740009868E13008950E948C68E0933308F09354
:10E7500034080895E0E0E0934C0C0895D2DFEA1706
:10E76000FB070895E0931808E0E0E093300808956F
:10E770000E9430640E94C72DE093240808950E94EF
:10E780005C190C944047E0911908EA93E0E0EA93A1
:10E790000E94712D0C9425290E947E431E2F1A93EE
:10E7A0000E94F72D103808951A93E091C605EA9358
:10E7B0000895E091890BEA930E946718E03008956C
:10E7C0000E948C68E093540CF093550C0895D90185
:10E7D00018960E94C07B0895E4E6F0E060E070E0E7
:10E7E0000E94717B08950E945C1911CC0A93E091FC
:10E7F000C605EA930895E0912F08EA930A930C94D2
:10E80000951A0E94C07BFA93EA930895A0E6BBE0B4
:10E81000AACAE0913C08E053E09322080895FA93D5
:10E82000EA93E0E3EA930C943064E0913908EA93C8
:10E830000C94D8630E94DE7A0E94D37B08950E94D4
:10E840009463EBE3EA930C941A63E89423F8E0E012
:10E85000F0E0F8DE0A93E1E0EA930C94712D0A935C
:10E86000E1E0EA930E94712DE1E00895E091120841
:10E87000ABE0EA9FF0010895A881B981EC91EF5FC8
:10E88000EC930895ABE00A9FF001E352FA4F08952C
:10E89000A083ABE00A9FF0010895ABE00A9FF0016E
:10E8A000E152FA4F0895E7EAF8E1FA93EA93EA852C
:10E8B000ABE0EA9FF0010895AC81BD81EE27A00F87
:10E8C000BE1F0895E02FAC81BD81F0E008950E9445
:10E8D000D37B84E00E944C6B28960895EE27A30F0B
:10E8E000BE1FEC91D001EC930895A2E5B7E079C882
:10E8F0000E94D37AEA0FFB1FAF010895E0912C0C20
:10E90000F0912D0C0895E32FA0911E08EA0F0895B1
:10E91000ADE02A9FF001E35FFC4F0895A8E0B0E06E
:10E920000E94EE7B0895F0E0FA93EA9308950E9426
:10E93000EF420C94BE42F0E00E94D37A08950E9408
:10E94000D37B0E94D9420C94BE420E94EF42EBEC72
:10E95000F8E1DDCB0E94BE420C94BE4220E030E0E4
:10E96000E12FE05DEA93EEECF8E1A7CBEAE0EA9371
:10E970000C94FA62E4E4FBE0FA93EA9308951091B0
:10E980005D0500915F0508950E947E433E2F0C9423
:10E990006046EAE0F0E00E941C7B0895DF01EE276C
:10E9A000A30FBE1F0895FA93EA9321C9EF81F8855A
:10E9B000FA93EA930895F0E0EA0FFB1F0895E02F21
:10E9C000A0E0B2E0B8CFEA0FFB1F3296E4910895C1
:10E9D000FA93EA93E0911B0CEA930E94E638E13245
:10E9E0000895EA930E948C38E1320895E6E0F0E061
:10E9F0000C94976C0E941947AAE9BBE0EE27A10F7F
:10EA0000BE1FEC91E1700895EE0FFF1F5EC8EA9300
:10EA10000E94E638E13208950E94300E0C94566C44
:10EA2000EAE3EA930C94B7460E94D37B0C94C74167
:10EA3000E3E7EA930C94B746EA23EA930E94EE4197
:10EA4000DAC8EA930E94EE41D6C8DF01329699C82F
:10EA50000E94D17AE854FF4F0895EAE4F6E0E0938B
:10EA60003A0CF0933B0C08950E94FA1AE0E0E09310
:10EA700021080E9445160E94300EE1E0E0931B0839
:10EA800008950E9440470E94CC100E947E430E2FA2
:10EA90000D330895EE81FF81FA93EA930895EAE237
:10EAA000EA93E6E7F9E10895EA930E9495160C943B
:10EAB000300EE093C105F093C2050895FE01FA936C
:10EAC000EA930895EEE8F9E1FA93EA93EE85FF857B
:10EAD00068897989FCCEE2E9F9E1FA93EA93AE8597
:10EAE000BF858889998978CE0E94D37BAA89BB8902
:10EAF0008C899D89E4E6F0E060E070E00E948B7B09
:10EB00000E94D37B88E00E944C6B2C960895EBE921
:10EB1000F9E1FA93EA93EE85FF858CCE84E00E94BA
:10EB20004C6B2896CBCFFA93EA93EE85FF85089538
:10EB30000E94F3630C948C6884E00E944C6B2896CE
:10EB40000895EE27A10FBE1FEC910895EA930E944D
:10EB500059421F5F0895E091C405A7ECB5E0F0E0CD
:10EB60000895AF5FEAE00E94767B0895E091C305C7
:10EB7000A7ECB5E0F0E0D4CBE981ADE0EA9FF0018D
:10EB8000E05FFC4F0895EF73A5E1EA9FF001E051CB
:10EB9000FB4F0895EF73ABE0EA9FF001EC5EFB4F93
:10EBA0000895AC81BD81EE27A30FBE1FAC91A030AC
:10EBB0000895ABE00A9FF001EC5EFB4F0895EA0F69
:10EBC000FB1F0F01AC81BD8189CEA5E10A9FF00139
:10EBD000E051FB4F0895EE81FF8101801280AE81EC
:10EBE000BF8115960E94C07BD0010895FE01389622
:10EBF000FA93EA930895EAA5FBA5FA93EA93089598
:10EC0000FA93EA93FE013A96FA93EA930E940A690C
:10EC100030E0E02F0895E091C105F091C20508951C
:10EC2000A1ECB5E0ED91FD913296FE93EE9308953F
:10EC3000AE81BF81EA17FB070895E0E0E093650528
:10EC4000E093660508951A930A933A932A930895D8
:10EC5000FA93EA93E0910E040895A0910003B09115
:10EC600001030895E0910003F0910103FA93EA9300
:10EC7000E0910203F0910303FA93EA930895E0937D
:10EC80000003F09301030895A981BA815ACF1A9322
:10EC90000A9300E010E00895F801AA81BB81EA0F11
:10ECA000FB1FE4910895AE0FBF1FAC91A0300895F3
:10ECB000D801F0E0AE17BF070895AE0FBF1FEC916B
:10ECC000EA930895EFEEF0E0EA1BFB0B0895A091A4
:10ECD0000E04E4E1EA9FF0012E2F3327C3CFE0E0DA
:10ECE000EA930E942F4C0E94AB7D0895ECE0EA9FCE
:10ECF000F001A0910D04EA9FF00108951A93E1E05C
:10ED0000E0930E04E0930D0410E00895ED81FE8180
:10ED1000FA93EA930895EF81F885EA1BFB0B0895B7
:10ED20003A932A935A934A930895EAA5FBA5E20FD2
:10ED3000F31FFA93EA930895ECA1EA930C94924C92
:10ED40003A932A93EEA1FFA1E40FF51F0895FA93D9
:10ED5000EA93EBCFEAA5FBA5E40FF51FFA93EA933C
:10ED6000EBCFE20FF31FFA93EA930895FA93EA9335
:10ED70005A934A930895EA9FF001AEA1BFA1F0E033
:10ED80000895E2E0E0930E04E0E2F0E0EAA3FBA3E2
:10ED90000895AE1BBF0BADCAEE8DF0E00895E20FF3
:10EDA000F31F3196FA93EA93ECA1FDA1E40FF51F4E
:10EDB00031960C948F6EECA1FDA1E40FF51F0C941D
:10EDC0008F6EE9A1F0E0DE0116960895ED8DEA93CD
:10EDD0000E946D46E9A1EF5FE9A30895ED8BFE8BDC
:10EDE000AB89BC8986CAA98DBA8DEA0FFB1FE98F52
:10EDF000FA8FEB89FC89AF89B88DEA0FFB1FEF8B87
:10EE0000F88FED89FE89AD89BE890E941C7B0E9426
:10EE1000DE7A0E94797CEE87FF87688B798BEB899D
:10EE2000FC89AB89BC890E941C7B0E94DE7A0E940F
:10EE3000797CAE85BF85888999890E944F7DEA8754
:10EE4000FB876C877D8700E010E00895F8010E9441
:10EE5000DE7A0E94797CEE83FF8368877987AE81B2
:10EE6000BF81888599850E94017DAA85BB858C8597
:10EE70009D850E94017DAE85BF85888999890E9404
:10EE8000DD7B0E94AC7C0E94427CAF015A934A9386
:10EE90000C94736BE98DFA8DE21BF30BFA93EA93F2
:10EEA0000895E98DFA8DE01BF10BFA93EA9308952A
:10EEB000F901AD8DBE8D0C94656DED8DFE8DE01B61
:10EEC000F10BFA93EA93EA8DEA930C94924CAD8D90
:10EED000BE8D0C94656DEFE3F1E0EA1BFB0B08952A
:10EEE000EB81FC81AF81B8850895E00DF11DFA93A7
:10EEF000EA930E94A44AE5E3EA930895E09365004B
:10EF00000C94236F0E94A27DEE81EA930E94D34A63
:10EF10008F010895E985FA85AD85BE8508950E9423
:10EF2000ED4AEB85FC85FA93EA930C94054BED854D
:10EF3000FE85A985BA85AE17BF070895EB85FC85C8
:10EF4000AF81B885AE17BF070895AD85BE85E98549
:10EF5000FA85EA1BFB0B0895FA93EA930C940E6C66
:10EF6000AB85BC85D8CEAF81B885EB85FC85EA1B27
:10EF7000FB0B0895D9010E941C7B0F010895D0015D
:10EF80000E94477BAF01FA01AD85BE850C94656D8B
:10EF9000ED85FE85E21BF30BFA93EA930895AD85A8
:10EFA000BE850C94656DA985BA85ED85FE85EA1B45
:10EFB000FB0B0895E881F981FA93EA9308955A9337
:10EFC0004A93EE85FF85AFCDFA93EA93EC85FD85F4
:10EFD000FA93EA930E94734DE0910E04AA85BB85D3
:10EFE000EACCD901F0E0AE17BF070895E05CF54F19
:10EFF00050CAE091370CA091360CEA170895E091C1
:10F000001108ABE0EA9FF0010895E3E0EA930E9463
:10F010007763F5CFE081E05DEA930C941A63A091E9
:10F02000250CB091260C0895E2E5EA930E941A633C
:10F030000C94604EF096EA930E94D863E2E7EA935C
:10F040000C941A63EA930E941A63EEE0EA930C941C
:10F050001A63EEEAF9E1D3CA0E944D63EBE3EA9347
:10F060000C941A63E0E3EA930C941A63EBE3EA93DB
:10F070000C941A635A934A930E94FB180E2F03367E
:10F080000895FA93EA930C9414341A93E985FA8557
:10F09000FA93EA930895E552F84FA885B985A083BD
:10F0A000B183E4CBE2E5EA930C941A631A93E091FE
:10F0B0003908E0531E2FEDE3F8E0BBCAE0911208D7
:10F0C000A0911308EA170895E3E1F8E0DACFE091A0
:10F0D0001308ABE0EA9FF0010895A091740B41CDB5
:10F0E000E093740BEAE2EA930E94D863DBCFE091ED
:10F0F000740BE05AA7CFD9011696EC9114CCF90104
:10F10000A281B381BA93AA9308950E944D63EAE362
:10F11000EA930C941A63D9011196E0E0EC930E94F3
:10F12000F363D2CFD901EC91FECBE05DEA930C946E
:10F130001A63E05DEA930E94D863B4CFEB58F44FB2
:10F1400069CFEEE0EA930C941A63EAE3EA930E9433
:10F150001A63F9010895E0935E0CF0935F0CE2E00E
:10F16000E0933608D9011196EC930895EA930E9432
:10F17000D86398CF0E944D63DBCCE091190CD9CFB6
:10F18000E091190CF0E0DACFFA93EA9365CF0E9490
:10F190004D63ECE2EA930E941A630CCF3EDAAC9125
:10F1A000A0330895A0915E0BB0915F0BE0E0EC936B
:10F1B0000895EE81FF81E093270CF093280C1093C3
:10F1C000240C0E94C71CE1E3089541E050E00E9436
:10F1D0004C62E887F987EAE3EA930E94C161E13073
:10F1E00008951A93E985FA85C1CDE2E2EA930C9479
:10F1F000C16113DAAC91A03208950FDAAC91AB3350
:10F2000008950BDAEC91EA930895EAE3EA930C94FB
:10F21000C1610E944C623197E887F987E8850895BB
:10F220000E94C07BE40FF51FD001ED93FC9308957D
:10F23000E091400BF0E0ED55F94F0895E0E0E093E8
:10F24000630CE093640C08950E944C623197E09344
:10F25000400BE091590BA091400BEA1708950E94D2
:10F260005257E091400BEA930895ECE2EA930E9432
:10F27000C161E0300895EC5BF44F0F01CED9EC9101
:10F28000D001EC931F5FC2CAEC5BF44FA0E0A083F7
:10F290000895EA930E94C161E1300895E091410B25
:10F2A0008ACBE091410BEF5FE093410B0895A3EA15
:10F2B000BBE0E091410BF0E00C949071AAE9BBE057
:10F2C000E091410B0C94FE6FE091410BF0E008954A
:10F2D000FA93EA930C94D553E091400BF0E0B8CB4D
:10F2E000FA93EA930C944D630E944D63ECE2EA9327
:10F2F0000C941A63ECE2EA930C941A630E94CA53CA
:10F30000E0E0E093410B0895E091410B0C94FE6F17
:10F31000E091600BF091610B0895AEE5BBE00C94B9
:10F32000B36EA0915E0BB0915F0BEC93F6CFA09102
:10F330005E0BB0915F0B13970895E0E0EA930E9493
:10F340002E54E09335080895AA81BB81EC91E29593
:10F35000E07FAE2FEC810895EA0FAA81BB81EC9388
:10F360008BCAE091040DA091030DEA170895E09176
:10F370003B09F0E0E05CF64F08951083E0913B0913
:10F38000EF5FE0933B09E12FA0913D090895E093E1
:10F390003D09E0913C09E150E0933C09E0300895DB
:10F3A000E05CF64FA0E0A0830895E091CF0DF091CE
:10F3B000D00D0895A091CD0DB091CE0DEA17FB07A9
:10F3C0000895E12FA091D40DEA0FE093D40DE091C0
:10F3D000D60D0895F0E0E85CF74F10830895E091B2
:10F3E000DB0EF0E0E652F24FE081E0939C00E0910A
:10F3F000DB0EEF5FE093DB0E08950FD9AC91AA33DB
:10F4000008950F010AD9EC91E0530C942D72EA9300
:10F410000E941A631F5F0895ECE5FAE1FA93EA93FC
:10F420000895FE013196FA93EA930895E881EA93EC
:10F430000C941A63E881F9816A817B810E94D37BF5
:10F440000895E05CF54FE081E0300895EA930E9472
:10F450007B68EA930C94C55EEA930E944965EAE5ED
:10F46000E0933E090895EA930E940A67E030089508
:10F47000E0917100E87F1E2F0895E0937300E4E8A7
:10F48000F2CF0A930E94E166E0300895FF276627D5
:10F4900077270E94797C0895EE8DAE85BF85888997
:10F4A0009989F4DF0E94017DA9A1BAA18827992733
:10F4B0000E94DA7B0E94DD7B0E94AC7C08950E9452
:10F4C000DD7B0E94AC7C08952A93ED89FE89FA9336
:10F4D000EA93FE017596FA93EA930C946369EE89B8
:10F4E000FF893497EE8BFF8B0895ED89FE89FA939F
:10F4F000EA93FE017596FA93EA930C946369AE89D8
:10F50000BF8914960E94C07BEE83FF83C3CAE8853F
:10F51000F9856A857B85AC85BD858E859F85089537
:10F520000E948A6BE883F9836A837B830895E8816C
:10F53000F9816A817B810895EA81FB816C817D81FB
:10F540000895E991F991309639F080EA9FE00197AA
:10F55000F1F7A8953197C9F708950024AF0DB01DB4
:10F560000895EA0FFB1F681F791F0895EA1BFB0B24
:10F57000680B790B0895F195E195F0400895F095A9
:10F5800060957095E195FF4F6F4F7F4F0895EE2383
:10F590000E2EEA2F19F0EE0F0A94E9F70895EE0FF8
:10F5A000FF1FEE0FFF1FEE0FFF1FEE0FFF1F08954F
:10F5B000FE2FFF0FFF0B6F2F7F2F08956F2F660F0A
:10F5C000660B762F0895BA2FBB0FBB0B8B2F9B2F8B
:10F5D00008958B2F880F880B982F0895EA17FB0743
:10F5E000E1E00CF0EE270895FA9FF02DEB9FF00D6F
:10F5F000EA9FE02DF10D08957A9F702D6B9F700D9D
:10F60000F89F700DE99F700D6A9F602D710DFB9F33
:10F61000600D711DE89F600D711D8827FA9FF02D08
:10F62000610D781FEB9FF00D611D781FEA9FE02DA3
:10F63000F10D681F781F089582D0D6DF0EF49BDF8E
:10F6400008958BD0D9DF0EF49ADF0895002498E056
:10F65000AA0F001C0E1A10F40E0E01C0A1609A959C
:10F66000B9F7EA2FA02D08950024112490E1AA0FE4
:10F67000BB1F001C111C0E1A1F0A18F40E0E1F1EB1
:10F6800001C0A1609A9599F7FD01D001089557D066
:10F69000EBDF0EF470DF08953F934F935F930024E8
:10F6A00011244427552730E2AA0FBB1F881F991F3A
:10F6B000001C111C441F551F0E1A1F0A460B570B26
:10F6C00028F40E0E1F1E461F571F01C0A1603A9559
:10F6D00059F7FD01BC01D001CA015F914F913F91E3
:10F6E00008953BD0D9DF0EF44ADF0895AFDFEA2F4B
:10F6F0000895E894B7FF04C0A095B095119668945A
:10F70000F7FD39DFB1DFFD010EF435DF0895C4DF09
:10F71000FD01BC010895E89497FF09C0A095B0953C
:10F7200080959095AF5FBF4F8F4F9F4F689477FD47
:10F7300026DFB2DFFD01BC010EF421DF0895E8945D
:10F74000F7FF02C018DF6894B7FF06C0A095B09518
:10F75000119600F8039400FA0895E89477FF02C028
:10F760000EDF689497FF0BC00024A095B09580959C
:10F7700090951196801D901D00F8039400FA08954D
:10F78000ED91FC9111970895ED91FD916D917C9112
:10F7900013970895ED93FD936D937C9308950590D1
:10F7A000F491E02D08957A936A93FA93EA93089579
:10F7B000689401C0E89401D09DD0182E862F612D49
:10F7C000192E972F712D1B2EBF2FF12D1A2EAE2F14
:10F7D000E12D0895119602D0FE2F1197E199FECFE9
:10F7E000FF93FFB7F894AEBBBFBBE09AEDB3FFBF8A
:10F7F000FF91089507D01196EF93EF2F03D0EF916B
:10F8000011970895E19B02C0A895FCCF9FB7F8948B
:10F81000AEBBBFBBE09A8DB3E81719F0EDBBE29A1F
:10F82000E19A9FBF0895552342F4503811F4E0FF48
:10F8300004C03196691F791F6BF050E8572711F407
:10F840005F93CDC05F3F31F0660F000C5795679511
:10F85000752F08955F9300200AF0CDC0C6C050E810
:10F86000192E1522880F991F9527550F879550E857
:10F87000072E0522660F771F7527550F6795089588
:10F88000689401C0E8945F93F2DF703818F07F3F0E
:10F8900008F4A5C056E1571BAAF4519558300EF450
:10F8A000593030F0EFEFFFEF6FEF7FE777F91AC0D5
:10F8B00077275523B9F0EE0FFF1F661F771F5A9564
:10F8C000D1F710C07727583028F0EF2FF62F672F89
:10F8D0005850F9CF552331F076956795F795E79510
:10F8E0005A95D1F700200AF44ADE5F910895689492
:10F8F00001C0E894309760407040B1F0002426F0D9
:10F90000772312F400943BDE172E7EE1112032F0B3
:10F910007A95EE0FFF1F661F111CF9CFEF2FF62F00
:10F92000612D5F938ADF5F9108954F93AF01FD01D1
:10F93000DA01AB01BC01CA01402D012C142E4F91FC
:10F940000895EA0FFB1F681F0895E095F0956095F4
:10F95000EF5FFF4F6F4F08955F9381DF903871F134
:10F9600050E8152604C05F937ADF903839F170387B
:10F9700021F1572F591B13F112F4D7DFFACF583169
:10F9800018F0AA27BB278827583028F0AB2FB82FAC
:10F9900088275850F9CF552329F08695B795A79514
:10F9A0005A95D9F7502D512562F0CBDF38F4679581
:10F9B000F795E795739513F41EC0B7DF3EDF5F91AF
:10F9C0000895EA1BFB0B680B51F010F40094BDDFA7
:10F9D0006623A2F3EE0FFF1F661F7A95CBF7EE2783
:10F9E000FF27662777275F910895EFEFFFEF6FE717
:10F9F0007FEF5F910895EFEFFFEF6FE77FE75F9194
:10FA000008955F932CDF703851F3903841F301244F
:10FA10000894791F23F41CF300203AF3ECCF0F92E3
:10FA20001F932F933F934F93112722279927689F66
:10FA3000A0018F9F302D410D591F6B9F300D411D2F
:10FA4000591F8E9F27D0BF9F25D06A9F23D0BE9F6E
:10FA50001DD0AF9F1BD0AE9F110D291F391F491F0D
:10FA6000591FE32FF42F652F522F4F913F912F9164
:10FA70001F910F9066232AF0550FEE1FFF1F661F80
:10FA800002C073954BF2CFDE5F910895100D211DDA
:10FA9000391F02C0200D311D491F591F08955F9362
:10FAA000DEDE703821F411200AF49FCFA4CF903805
:10FAB00009F495CF01240894970B1BF4D4F300208C
:10FAC000F3CF792F1F932F933F934F931124112737
:10FAD000222733274427552790E2AE17BF07860712
:10FAE000410730F0AE1BBF0B860B410B089401C0E1
:10FAF0008894551F221F331F111CAA1FBB1F881F6C
:10FB0000441F9A9551F7F901612D4F913F912F9123
:10FB10001F91662332F0550FEE1FFF1F661F7A9567
:10FB200043F281DE5F910895309760407040089500
:10FB300000240A160B06089500240A160B06080670
:10FB4000090608955A934A933A932A931A930A936B
:10FB500008955D814C813B812A8119810881089536
:00000001FF
